:1000000000000320D10100007DF1010035F1010065
:1000100035F1010035F1010035F1010035F1010044
:1000200035F1010035F1010035F101007DF10100EC
:100030007DF1010035F10100111C0200151D0200C7
:100040007DF101007DF101007DF101007DF10100F4
:100050007DF101007DF101007DF101007DF10100E4
:100060007DF101007DF101007DF101007DF10100D4
:100070007DF101007DF101007DF101007DF10100C4
:100080007DF101007DF101007DF101007DF10100B4
:100090007DF101007DF101007DF101007DF10100A4
:1000A0007DF101007DF101007DF101007DF1010094
:1000B0007DF101007DF101007DF101008DFC010069
:1000C0007DF10100FD0302007DF1010091090200B4
:1000D0007DF10100B52A02007DF101007DF10100F2
:1000E0007DF101007DF1010059E901007DF1010080
:1000F0007DF101007DF101007DF101007DF1010044
:100100008521020099210200AD210200C1210200D7
:100110007DF101001D0C02007DF101007DF1010067
:100120007DF101007DF101007DF101007DF1010013
:100130007DF101007DF101007DF101007DF1010003
:100140007DF101007DF10100AD2B02007DF1010088
:100150007DF101007DF101007DF101007DF10100E3
:100160007DF101007DF101007DF101007DF10100D3
:100170007DF101007DF101007DF101007DF10100C3
:100180007DF101007DF101007DF101007DF10100B3
:100190007DF101007DF10100A52C02007DF101003F
:1001A0007DF101007DF101007DF101007DF1010093
:1001B0007DF101007DF101007DF101007DF1010083
:1001C0007DF101007DF101007DF101007DF1010073
:1001D0005C4B4CF2205210B51A804DF628121A8052
:1001E00000BF00BF1EF0CEFF574B4FF030621A60C9
:1001F000564A9A60564ADA60564B4FF470021A60BB
:10020000554B564A1A60564B1A78110703D51A787F
:1002100042F008021A70534B5349AA221A70534AEB
:10022000534B8B4204D252F8040F43F8040BF8E707
:10023000504B514900228B4202D243F8042BFAE77B
:100240004E494F4A002352F8230041F8230001335E
:10025000742BF8D14B4B4C4A802103F8011B93427D
:10026000FBD14A4B454A1A60494B8A221A70A3F5C2
:10027000805324225A70A0221A709A799207FCD5D2
:100280009A79D406FCD4434A937903F00C03082BE3
:10029000FAD1414B60221A7002331A78802AFCD1BD
:1002A0003C4B01221A715D225A719A799006FCD555
:1002B0009979384A4906FBD5384B394919600021EC
:1002C000596020231370937903F00C030C2BFAD19F
:1002D000344B354A1A60354A354C136813F4807331
:1002E00003D123604FF4A8531360324B324A1A6093
:1002F00000225A60072243F8042C304AC3F80C2D20
:1003000062B61FF091F82368DA0705D52C481FF074
:100310000DF82C4B2C4A1A602C4B1B785B0609D528
:10032000284C294B22689A4204D125481EF0FEFF32
:100330000023236024F0B2FE1EF02AFF21F04AFFC2
:10034000FEE700BF0E20054030800440823F0400DD
:100350000100002B88ED00E0002008E0030000858C
:1003600002D0074000E007408812FF1F0CCA0200BD
:100370003007FF1F8812FF1F8420FF1F0002FF1F8E
:100380000000000000E400E064E400E008ED00E0AC
:10039000005006400040064001E007404480044011
:1003A0000000060204800440C010070010D0034083
:1003B00014D0034014E000E01FBF02000000202022
:1003C000CB0D29611CE00340A5C3945A00F00740FF
:1003D000FFFFFFFFFFFFFFFFFFFFFFFFFFFFFFFF2D
:1003E000FFFFFFFFFFFFFFFFFFFFFFFFFFFFFFFF1D
:1003F000FFFFFFFFFFFFFFFFFFFFFFFFFFFFFFFF0D
:10040000FFFFFFFFFFFFFFFFFFFFFFFFDEF9FFFF23
:1004100010B5054C237833B9044B13B10448AFF33E
:1004200000800123237010BD8812FF1F0000000010
:1004300008CA0200084B10B51BB108490848AFF3C1
:1004400000800848036803B910BD074B002BFBD0A0
:10045000BDE81040184700BF000000008C12FF1FCD
:1004600008CA02008812FF1F0000000000690B6923
:100470009842D4BF00200120704700BF80698B697B
:100480000028B8BF4042002BB8BF5B429842D4BF9F
:1004900000200120704700BFF0B586460120DEF83D
:1004A0005870DEF83030BA6A106079683A680A44E9
:1004B0007A600EF1300493B15A69002A08DB9A6A17
:1004C00010605E6819683D695A6931445960521B71
:1004D00019690A445A6154F8043F002BECD1DEF844
:1004E0002430144ADEF81840DEF86C000021116058
:1004F000DB00516803F1804303F5603321440D2490
:1005000019611460DA68502122F08002DA60D96043
:1005100000B1F0BD7A68FB689A4200D0F0BDDEF809
:100520005C3001228EF82820002BF7D0BDE8F04087
:10053000184700BF00800340C36A00F12C0233B1AA
:100540000120D96A52F8043F0860002BF9D17047A6
:100550000C4BD3F8902072B9596A1A6AD3ED0A7A13
:1005600002FB01F207EE102A60EE277AB8EE477A16
:1005700087EE870A7047D3F89810D3F89420D3ED0C
:10058000277AEDE7E815FF1F836D012280F89020A0
:100590005B6872B6DFED0B6AD0ED207A90ED1F7AC2
:1005A00067EEA67AF4EEC77AC0ED1E7AD0ED227A15
:1005B000F1EE10FAD8BFF1EE677AC0ED237A62B699
:1005C000704700BF00000000036A8B4210B523D0C3
:1005D000C369994200D010BD8369002BFBD072B66D
:1005E000194AC369846900211160DB00516803F175
:1005F000804303F5603321440D2419611460DA68E7
:10060000502122F08002DA60D96062B60069036886
:10061000BDE810405B6818470446006903689B68A2
:10062000984794F82430002BD5D004F1080021F02D
:1006300087FD0023E06963601EF076F9206ABDE85B
:1006400010401EF071B900BF008003402DE9F04159
:100650008568002D31D0816D836F04464868D4F8D9
:10066000AC101B1A002BB8BF5B428B423ADBD4F8AC
:10067000B0108B422A4608DBE16F8B4265DB936842
:1006800023F002039360BDE8F081D4F888100029BC
:10069000F5D02B683B4A93421ED96A683A48B0FBB2
:1006A000F1F19B1A99420AD3CB1A002401200322AC
:1006B000AC60E8602B60AA602960BDE8F0816069E9
:1006C0000368002601240322AE601B68EC602960E9
:1006D000AA60BDE8F04118472B4BB3FBF1F129604C
:1006E000BDE8F081D4E92401D4F8A82002FB03F38B
:1006F000C61841F100073046394624F0B7FA07EE34
:10070000900AB1EEE70AB4EE400AF1EE10FA2ED1EB
:10071000FDEEC07A2A4617EE903A17EE901ADBB13A
:10072000002DB6D11949184D0E68B5FBF3F51EB171
:1007300002210120B047A26800200121032390601C
:10074000D16015609360BDE8F081CB1AD4F8A82081
:10075000D4E92601013BC9E7002D90D10B4B1B6862
:10076000002B8CD0022101209847A26887E73946E8
:10077000304624F07BFA00EE100A22F0ADFCA568AA
:10078000C6E700BF7FA9030000879303DC1BFF1FA0
:10079000F8B50446D0ED1F7A94ED1E7A806DF4EE24
:1007A000477AF1EE10FA436838D1FDEEC77A17EEBA
:1007B000905A94F890300BB1002D76D08368AB42FC
:1007C0002BD0002D0368B4BF4FF0FF3201229A42B4
:1007D00015D004F12801012608E013685B42012BC3
:1007E00013600BBF126B536B13601E6051F8042F24
:1007F000002AF2D1636FC3EB03139B003FD185EA5C
:10080000E572A2EBE572A368FAB9002B7AD09A6878
:1008100022F002029A608560F8BDF8BDD4ED236A2B
:10082000F5EEC06A77EEA67AF1EE10FAB4EEE77A4A
:100830002FDDF1EE10FAD8BFF0EE477ABDEEE77A81
:10084000C4ED1F7A17EE105AB3E7002B47D0196892
:10085000314EB14223D95E68304FB7FBF2F2891BAB
:100860008A4232D26069002601689E600127032611
:10087000DF6009681A609E608847A06DCBE7013B86
:10088000FDD185EAE572A2EBE572A368002ABCD02F
:10089000DBE7F1EE10FA58BFF0EE477ACEE71F49DA
:1008A000B1FBF2F21A608560F8BD04F10C0021F092
:1008B00047FC206AA5601EF037F8606A1EF034F825
:1008C000A36D9D6084F89050F8BD511A0027012651
:1008D00003249F60DE6019609C601A609BE71049EA
:1008E0000E4E0F68B6FBF2F627B101200221B84781
:1008F000A368A06D0024012103229C60D9601E60C2
:100900009A6088E7064B1B68002B80D001200221EB
:100910009847A368A06D7AE77FA903000087930337
:10092000DC1BFF1F70B5044608460D4625F048FC49
:1009300023680246294620465B68BDE87040184798
:1009400038B5044608460D4625F03AFC23680246B1
:1009500029465B68204698470546204621F082FCE0
:10096000284438BD38B5054621F0CCFC044628465D
:1009700021F078FC204438BD38B5054621F0C2FC92
:100980000446284621F06EFC204438BD38B50A22C2
:100990000023054621F076FC0446284621F062FC3F
:1009A000204438BD38B5C9B2054621F0B5FC04462F
:1009B000284621F057FC204438BD00BF10B509215E
:1009C0002C4820F0BFFF2C4821F04CFCFE212B4886
:1009D0001BF07AFD00282FD10A2128481BF074FD56
:1009E00098B9182125481BF06FFD00283AD10F2136
:1009F00022481BF069FD50BB09212048204C1BF008
:100A000063FD002832D1206009E01D4C1D480A23F7
:100A10001946236020F096FF174821F023FC0C2193
:100A2000194820F08FFF2168134821F06BFC124811
:100A3000BDE8104021F016BC114C144801230921D7
:100A4000236020F07FFF0C4821F00CFCE7E70C4C02
:100A50000F480F230A21236020F074FF064821F07D
:100A600001FCDCE7064C0B481823F3E70A4809238E
:100A7000CEE700BF888802002408FF1F6019FF1F0F
:100A80006C17FF1FA0880200D08802009488020023
:100A9000B8880200AC880200C488020070B50D4618
:100AA00084B00A2106464148144620F04BFF2946EF
:100AB0003F4821F027FC3E4821F0D4FBBCB13D4B20
:100AC000D3F8A420A2F10102B2FA82F252093A4C00
:100AD00023680193019923680093009B5B1A092BFB
:100AE000F9D9032E2FD8DFE806F0241A0F04224686
:100AF000EDE7002D51D12AB92E4B042093F8741044
:100B00001EF026FC04B070BD002D3DD1002AF9D1A5
:100B1000284B112093F877101EF01AFCF2E755BB12
:100B2000002AEFD1234B162093F876101EF010FC0C
:100B3000E8E7BDB9002AE5D11E4B0E2093F87510E9
:100B40001EF006FCDEE7002DDCD022681B4B039272
:100B500003991A6823680293029B5B1A9A42F9D898
:100B600004B070BD134B93F875100E2081F0010195
:100B70001EF0EEFBE9E70F4B93F87610162081F09C
:100B800001011EF0E5FBE0E70A4B93F87710112016
:100B900081F001011EF0DCFBD7E7064B93F87410DF
:100BA000042081F001011EF0D3FBCEE7E0880200B3
:100BB0002408FF1FE815FF1F141CFF1F5807FF1F05
:100BC000F0B52DED028B85B0044601AE0DF10F0797
:100BD0000FE0FF2D66D001A8357025F0F1FA01462F
:100BE00001A820F0AFFE334821F03CFB0136BE42A5
:100BF00029D0236820465B6998470021C5B22E485A
:100C000020F0A0FE2B4821F02DFB33212B4820F0B3
:100C100099FE284620F01AFF0221294820F092FE72
:100C20002946244821F06EFB224821F01BFB042DAD
:100C3000CFD11921234820F085FE01361D4821F02F
:100C400011FBBE42D5D101A824F018FA04211E4898
:100C5000B0EE408AF0EE608A20F074FE01A825F024
:100C6000AFFA014601A820F06DFE124821F0FAFA11
:100C70000721164820F066FEB0EE480AF0EE680A3A
:100C800004210C4821F048FB0A4821F0EBFAB0EEB1
:100C9000480AF0EE680A05B0BDEC028BF0BD23688F
:100CA0005B699847236820461B69984700282046BF
:100CB000F5DC9BE72408FF1FB0A20200EC880200CD
:100CC000FCB50200208902003C8902004489020030
:100CD00003280FD8DFE800F00B0805020A48FFF7E9
:100CE0006FBF0A48FFF76CBF0948FFF769BF0948A3
:100CF000FFF766BF9FED020B704700BFAFF30080A8
:100D0000000000000000F0BF0408FF1FF407FF1FF1
:100D1000E407FF1F2408FF1F012828D0022813D052
:100D200010B19FED140A7047134A1169D368D2EDD0
:100D3000056A03FB01F307EE103A60EE267AB8EE7F
:100D4000477A87EE870A70470B4B5A6B012AE8D81F
:100D5000D96B9A6BD3ED116A02FB01F207EE102AF0
:100D600060EE267AB8EE477A87EE870A7047FFF77B
:100D7000EFBB00BF00000000E815FF1F38B5434D72
:100D80004348EA6BAB6B95ED107AD5ED127A414C86
:100D900003FB02F32DED048B08EE103AB8EE488AFF
:100DA000DFED3D8A28EE078A0D2167EEA88AF0EE76
:100DB000409A20F0C7FD18EE100A23F0EBFA41EC40
:100DC000100B0221204621F0A7FA204621F04AFA12
:100DD0001121324820F0B6FD286C23F0DBFA41ECFB
:100DE000100B0221204621F097FA204621F03AFA12
:100DF0000F212B4820F0A6FD89EEA89A18EE900A44
:100E000023F0C8FA41EC100B0221204621F084FAAD
:100E1000204621F027FA1021224820F093FD19EEF8
:100E2000900A23F0B7FA41EC100B0221204621F082
:100E300073FA204621F016FA07211B4820F082FDA4
:100E400019EE100A23F0A6FA41EC100B02212046FD
:100E500021F062FA28EE098A204621F003FA0821DF
:100E6000124820F06FFD18EE100A23F093FA41ECBF
:100E7000100B0221204621F04FFA204621F0F2F912
:100E8000B0EE480ABDEC048B38BD00BFE815FF1F6B
:100E90007C8902002408FF1FDB0FC9408C890200F7
:100EA000A0890200B0890200C4890200CC89020036
:100EB000144A1548D2ED117AD16B936B80EE270A54
:100EC00010B503FB01F31921104C2DED028B08EE38
:100ED000103AB8EE488A28EE008A20F033FD18EE6A
:100EE000100A23F057FA41EC100B0221204621F0A2
:100EF00013FA204621F0B6F9B0EE480ABDEC028B99
:100F000010BD00BFE815FF1FD88902002408FF1F8D
:100F10000128F0EE407A1CD0022813D010B19FEDCA
:100F2000160A7047154AD2ED056A1169D36887EE33
:100F3000A67A03FB01F300EE103AB8EE400A20EE69
:100F4000070A70470D4B5B6B9BB1012BE7D1FFF795
:100F5000AFBF0A4AD2F8903023B9D2ED0A6A516A7B
:100F6000136AE4E7D2ED276AD2F89810D2F89430E9
:100F7000DDE7FFF703BF00BF00000000E815FF1F1B
:100F800038B52F4D2F4C95ED007AD4ED007AB5EEA3
:100F9000C07AF1EE10FA48BFB1EE477AF5EEC07AAA
:100FA00048BF85ED007AF1EE10FA44BFF1EE677AA2
:100FB000C4ED007A67EEA77A2DED048BE7EE077A91
:100FC00008EE100A17EE900A08EE901A23F0E2F9E4
:100FD00041EC100B21F0C0FF51EC100B23F026FD6B
:100FE00094ED006AD5ED006A07EE900A87EE867AE6
:100FF00087EEA69AF8EEE88AB8EEC88A67EE287AF5
:1010000017EE900A23F0C6F941EC100B21F004FF13
:1010100051EC100B23F00AFD68EE097A206017EE00
:10102000900A23F0B7F941EC100B21F0F5FE51ECDA
:10103000100B23F0FBFCBDEC048B286038BD00BF17
:101040007014FF1F6814FF1FBA4AF8B592E80A002F
:1010500003FB01F307EE903A92ED027AB64CF8EEFC
:10106000677A2DED028BB0EE408AF0EE608A67EE73
:10107000877A17EE900A23F08DF941EC100B21F0DE
:10108000CBFE51EC100B23F089FC09210546AB483F
:1010900020F058FC2168AA4821F034F9A84821F032
:1010A000E1F8B0EE480AF0EE680A0221A44821F007
:1010B00033F9A34821F0D6F82368013B042B00F252
:1010C000D180DFE803F045688BAD03009D4C2368B9
:1010D000022B84ED048B284600F0C78023F048F9EA
:1010E00053EC182B23F0D4FA23F058FCA0601621FF
:1010F000954820F027FC2946914821F003F910215A
:10110000924820F01FFCB0EE480AF0EE680A022177
:101110008B4821F001F903218D4820F013FC0621B2
:101120008C4820F00FFC06218B4820F00BFCA168B6
:10113000834821F0E7F8824821F094F8874B8148F2
:101140001968BDEC028B1822BDE8F8401DF060BFA5
:10115000834C2368022B84ED048B284600F0D58055
:1011600023F006F953EC182B23F092FA23F016FC27
:10117000A06006217B4820F0E5FB0621764820F0A0
:10118000E1FBA1686E4821F0BDF86D4821F06AF8D6
:10119000754B7348D4E7754C2368022B84ED048BA0
:1011A000284600F09E8023F0E3F853EC182B23F040
:1011B0006FFA23F0F3FBA06006216D4820F0C2FB1C
:1011C0000621654820F0BEFBA1685D4821F09AF831
:1011D0005B4821F047F8674B6448B1E7664C2368E9
:1011E000022B84ED048B284667D023F0C1F853EC22
:1011F000182B23F04DFA23F0D1FBA06006215F48A5
:1012000020F0A0FB0621544820F09CFBA1684C482C
:1012100021F078F84A4821F025F8594B56488FE7D5
:10122000584C2368022B84ED048B284631D023F0E0
:101230009FF853EC182B23F02BFA23F0AFFBA060A0
:101240000621514820F07EFB0621434820F07AFB1E
:10125000A1683B4821F056F8394821F003F84B4B80
:1012600048486DE7BDEC028BF8BD23F081F8002201
:1012700006460F46464B51EC180B23F009FA02467E
:101280000B463046394623F0D9F823F087FBA0609F
:101290002DE723F06DF8002206460F463C4B51EC3B
:1012A000180B23F0F5F902460B463046394623F079
:1012B000C5F823F073FBA060C2E723F059F80022C1
:1012C00006460F46324B51EC180B23F0E1F902466B
:1012D0000B463046394623F0B1F823F05FFBA0609F
:1012E0008CE723F045F8002206460F46284B51ECC8
:1012F000180B23F0CDF902460B463046394623F051
:101300009DF823F04BFBA06056E723F031F8002254
:1013100006460F461E4B51EC180B23F0B9F9024656
:101320000B463046394623F089F823F037FBA0609E
:101330001FE700BFE815FF1F7015FF1FF4890200AB
:101340002408FF1F5017FF1F288A0200408A02004E
:1013500098B50200548A0200088A02005C07FF1F49
:10136000F016FF1F008A02005007FF1F0817FF1F1B
:10137000108A02005407FF1F2017FF1F188A02005F
:101380006807FF1F3817FF1F208A02007807FF1F1A
:1013900000807640F8B51D212DED028B914D924CC9
:1013A000924E08EE100A924820F0CCFA914820F0B4
:1013B00059FF95E8090003FB00F307EE903A95ED1D
:1013C000027AD4ED036A8C4A8C49F8EE677AB8EE5B
:1013D000C88A67EE877A002387EEA67A0B601360CF
:1013E000C7EE087A17EE900A22F0D4FF41EC100BFA
:1013F00021F012FD51EC100B23F0D0FA2768306079
:10140000012F00F0B98065D3022F41D07C4F7D4879
:10141000152120F097FA3168764820F073FF75485F
:1014200020F020FF2421784820F08CFAE06822F098
:10143000B1FF41EC100B02216E4820F06DFF6D48AA
:1014400020F010FF2921714820F07CFAA06922F0D9
:10145000A1FF41EC100B0221664820F05DFF6548BA
:1014600020F000FF14216A4820F06CFA39686148C6
:1014700020F048FF5F4820F0F5FE1421654820F079
:1014800061FABDEC028B5B48BDE8F84020F0EABE93
:101490002B21614894ED068A20F054FAA06922F0CD
:1014A00079FF41EC100B3946524820F035FF514886
:1014B00020F0D8FE6B6B002B00F08980012BA5D1AA
:1014C000B0EE480AFFF7F4FC4D4FBDEEC00A87EDC1
:1014D000000A9CE794ED067AD5ED057A484F87EE31
:1014E000278AD5ED047A95ED037AF8EE677AB8EE9F
:1014F000477A67EE887A67EE877A17EE900A22F0CD
:1015000049FF41EC100B21F087FC51EC100B23F04C
:1015100045FA18213860414820F014FAA06922F0F9
:1015200039FF41EC100B0221324820F0F5FE314822
:1015300020F098FE24213A4820F004FA686922F04D
:1015400029FF41EC100B02212A4820F0E5FE294832
:1015500020F088FE1121334820F0F4F918EE100A2B
:1015600022F018FF41EC100B0221224820F0D4FE9B
:10157000204820F077FE4AE7D5F89030D4ED065A9F
:10158000F3B195ED276A95ED267AD5ED257A1C4FB6
:10159000C5EE866AB8EE477AF8EE677A26EE877A65
:1015A00067EE277A17EE900A22F0F4FE41EC100B5A
:1015B00021F032FC51EC100B23F0F0F9386026E7F3
:1015C00095ED0A6A95ED097AD5ED087ADFE7B0EE78
:1015D000480AFFF7D3FB0A4FBDEEC00A87ED000AA9
:1015E00015E700BFE815FF1F0814FF1F8015FF1F38
:1015F0005C8A02002408FF1FB412FF1F6418FF1F3B
:101600001C13FF1F008B0200188B0200408B02008E
:101610006C8B0200848B0200D48A02007C8A020058
:10162000988A0200C08A02000C4B1B68032B13D857
:10163000DFE803F00E0A06020146094820F0ECBD7F
:101640000146084820F0E8BD0146074820F0E4BD07
:101650000146064820F0E0BD704700BF4807FF1F65
:101660000408FF1FF407FF1FE407FF1F2408FF1FE4
:10167000F0B585B06C496D4C6D4E6E4F684620F0EC
:10168000BFFF00216846FFF7CFFF684620F078FFD4
:101690006949684620F0B4FF00216846FFF7C4FF9F
:1016A000684620F06DFF6549684620F0A9FF0021DB
:1016B0006846FFF7B9FF684620F062FF5E4968465A
:1016C00020F09EFF00216846FFF7AEFF684620F03D
:1016D00057FF5B49684620F093FF00216846FFF7FB
:1016E000A3FF684620F04CFF5349684620F088FF6E
:1016F00000216846FFF798FF684620F041FF5149F6
:10170000684620F07DFF00216846FFF78DFF6846A0
:1017100020F036FF4849684620F072FF00216846F5
:10172000FFF782FF684620F02BFF4749256891EDBF
:10173000027ADFED466A3668454A91E8090003FB04
:1017400000F307EE903A06EE105AF8EE677AB8EE1C
:10175000C66A67EE877A012E86EE277A67EE267ACA
:10176000C2ED007A50D033D3022E0FD1D7ED007ADC
:101770003046B8EEE70AFFF7CFFA364B3046012283
:10178000002183ED000AFFF789F92568324A334BBF
:1017900015600821002532481D6020F0D3F821682B
:1017A000304820F0AFFD2F4820F05CFD05212E4889
:1017B00020F0C8F839682B4820F0A4FD294820F013
:1017C00051FD294601220320FFF768F905B0F0BD5D
:1017D000D7ED007A0A69CB6891ED057A1D4DF8EED8
:1017E000E77A03FB02F327EE877A07EE903AF8EEEA
:1017F000677A0021C7EE276A08460122C5ED006A14
:10180000FFF74CF92568C1E7D7ED007AB8EEE70A93
:10181000FEF79EFE0F4B32463046002183ED000A54
:10182000FFF73CF92568B1E79C8B02006418FF1FA5
:101830000814FF1FB412FF1FB08B0200B48B02000C
:10184000C88B0200DC8B0200E815FF1F0000B443C8
:101850009016FF1FBC13FF1F6C15FF1FF812FF1F10
:101860006CA802002408FF1F5CA4020010B5F0EE73
:10187000407A0021F2EE046ABDEEE77AB8EEC77A4C
:10188000B4EE677AF1EE10FA04D00131062967EE62
:10189000A67AF1D11E4B1B68032B37D8DFE803F083
:1018A000291C0F0210EE100ACCB222F073FD41EC9D
:1018B000100B21461748BDE8104020F02DBD10EE5A
:1018C000100ACCB222F066FD41EC100B2146124802
:1018D000BDE8104020F020BD10EE100ACCB222F07E
:1018E00059FD41EC100B21460C48BDE8104020F09A
:1018F00013BD10EE100ACCB222F04CFD41EC100BDF
:1019000021460748BDE8104020F006BD10BD00BFCD
:101910004807FF1F0408FF1FF407FF1FE407FF1F0E
:101920002408FF1F084B1B68032B0BD8DFE803F0CC
:10193000080604021EF080BF1EF004BC1EF098B81A
:1019400020F084B8704700BF4807FF1F2DE9F04121
:10195000DFF85080104F114E114D044601464046AD
:1019600020F05AFC404620F07DFC2146384620F00D
:1019700053FC384620F076FC2146304620F04CFCE3
:10198000304620F06FFC2146284620F045FC2846D2
:10199000BDE8F04120F066BCE407FF1FF407FF1F1D
:1019A0000408FF1F2408FF1F2DE9F04FB24CA3B01D
:1019B00001210D201DF0E0FC23680893089A23689C
:1019C0000793079BAC4D9B1A0E2BF8D9AB4BAC4938
:1019D0001E681EA820F014FE00211EA8FFF724FE9A
:1019E0001EA820F0CDFD0A2231461EA820F03AFEA6
:1019F0001EA8FFF7ABFF1EA820F0C2FD40F2871023
:101A00001DF01AFE0C219F481EF03CF803219E4851
:101A10001EF038F82B680693069A23680593059BF9
:101A2000954D9B1A312BF8D90C2196481EF02AF8B7
:101A3000032195481EF026F82B680493049A236826
:101A40000393039B8C4D9B1A312BF8D907218F48A8
:101A50001EF018F803218C481EF014F82B6802932E
:101A6000029A23680193019B9B1A312BF9D91EF02E
:101A70008BF80028864D0CDD01230C2185482B6056
:101A80001FF060FF2968844820F03CFC824820F069
:101A9000E9FB40F287101EF07FF90C2179481EF017
:101AA000A9FB032178481EF0A5FB23680E930E9A2C
:101AB00023680D930D9B704E9B1A312BF8D90C2186
:101AC00070481EF097FB03216F481EF093FB3368AC
:101AD0000C930C9A23680B930B9B674E9B1A312B2C
:101AE000F8D9072169481EF085FB032166481EF0DE
:101AF00081FB33680A930A9A23680993099B9B1A0E
:101B0000312BF9D91EF0F8FB00280CDD02230C2143
:101B100062482B601FF016FF29685F4820F0F2FB37
:101B20005D4820F09FFB82201EF040FD0C215548AF
:101B30001EF08CFE032154481EF088FE2368149387
:101B4000149A23681393139B4B4E9B1A312BF8D98D
:101B50000C214C481EF07AFE03214B481EF076FE05
:101B600033681293129A23681193119B424E9B1A69
:101B7000312BF8D9072145481EF068FE0321424861
:101B80001EF064FE33681093109A23680F930F9B26
:101B90009B1A312BF9D91EF08DFE00280CDD032392
:101BA0000C213F482B601FF0CDFE29683A4820F0F9
:101BB000A9FB394820F056FB0A213A483A4E1FF05B
:101BC000C1FE2968344820F09DFB334820F04AFBD1
:101BD000364B1B683746C6EB03083D46A83608EB74
:101BE00005001DF0CDF905F8010BB542F7D1304BDA
:101BF000304E1B68B346C6EB03085D46343608EB2F
:101C000005001DF0BDF905F8010BB542F7D12A4BCF
:101C10002A4E1B683246C6EB03081546403608EBD1
:101C200005001DF0ADF905F8010BAE42F7D1244BCC
:101C3000244E1B68B246C6EB03085546343608EB03
:101C400005001DF09DF905F8010BB542F7D11E4BBB
:101C50001E4D1E68A946761BC846103506EB0800C7
:101C60001DF08EF908F8010BA845F7D1184B194D56
:101C70001E68A84630E000BF141CFF1F7420FF1F21
:101C8000F08B0200F88B0200B08B0200088C02007F
:101C90004807FF1F108C02002408FF1F208C020041
:101CA000308C0200408C0200E815FF1F7C14FF1FDF
:101CB0009007FF1F2819FF1F3C07FF1F1418FF1F65
:101CC0008407FF1FC013FF1F8C07FF1F7015FF1F26
:101CD0005007FF1FF016FF1F761B183506EB080094
:101CE0001DF04EF908F8010B4545F7D1C54BC64D1F
:101CF0001E68A846761B183506EB08001DF040F953
:101D000008F8010BA845F7D1C04BC14D1E68A84685
:101D1000761B183506EB08001DF032F908F8010BA8
:101D2000A845F7D1BB4BBC4D1E682B46761B984689
:101D3000403506EB08001DF023F908F8010B454576
:101D4000F7D1B64BB64D1E682B46761B98465C35D0
:101D500006EB08001DF014F908F8010BA845F7D1AF
:101D6000B04BB14D1E682B46761B9846543506EB9A
:101D700008001DF005F908F8010B4545F7D1AB4BFC
:101D8000AB4D1E682B46761B9846603506EB080067
:101D90001DF0F6F808F8010BA845F7D11321A54866
:101DA0001FF0D0FDDBF83010A34820F0ABFAA248BA
:101DB00020F058FA1221A1481FF0C4FDDAF83010C3
:101DC0009D4820F09FFA9C4820F04CFA1A219C482C
:101DD0001FF0B8FDD9F80010974820F093FA964804
:101DE00020F040FA132197481FF0ACFD8A4B92482F
:101DF00019680A22002320F045FA8F4820F032FAB1
:101E0000132191481FF09EFD904B8B4819680A22C0
:101E1000002320F037FA884820F024FA12218C4859
:101E20001FF090FD804B8448996C0A22002320F01B
:101E300029FA814820F016FA172186481FF082FD02
:101E40007B4B7D4819680A22002320F01BFA7A4850
:101E500020F008FA132180481FF074FD704B76487B
:101E6000996B0A22002320F00DFA734820F0FAF94A
:101E7000012104201DF080FA01210E201DF07CFAC2
:101E8000012116201DF078FA012111201DF074FAAD
:101E9000012200210320FEF701FE00210846012255
:101EA000FEF7FCFD012210460021FEF7F7FD01229E
:101EB00000210220FEF7F2FD0221387E1DF05CFABF
:101EC0000221387F1DF058FA23681A931A9A236862
:101ED0001993199B614D9B1A092BF8D90121387E62
:101EE0001DF036FA0121387F1DF032FA022197F8F1
:101EF0002C001DF041FA022197F830001DF03CFA49
:101F00002B681893189A23681793179B534D9B1AA5
:101F1000092BF8D9012197F82C001DF019FA01219D
:101F200097F830001DF014FA022197F84C001DF0CC
:101F300023FA022197F850001DF01EFA012197F8AC
:101F40004C001DF005FA97F8500001211DF000FA31
:101F50002B681693169A23681593159B9B1A092BC9
:101F6000F9D9012118201DF007FA012118201DF0D0
:101F7000EFF901210F201DF0FFF901210F201DF0C5
:101F8000E7F901210A201DF0F7F901210A201DF0CF
:101F9000DFF9012109201DF0EFF9012109201DF0D1
:101FA000D7F9FEF70BFD012200210320FEF776FD95
:101FB0002A4E032501210D201DF0CAF923681E9326
:101FC0001E9A23681D931D9B9B1A312BF9D9002162
:101FD0000D201DF0BDF933681C931C9A23681B93D8
:101FE0001B9B9B1AB3F5967FF8D3013DE2D10E21DE
:101FF0001B481FF0A7FC104820F034F923B0BDE8BF
:10200000F08F00BF5407FF1F0817FF1F6807FF1F4F
:102010002017FF1F6C07FF1FA815FF1F3407FF1FA6
:102020002013FF1F3807FF1F8014FF1F4C07FF1FDF
:102030000814FF1F4C8C02002408FF1F608C020054
:10204000748C0200908C0200A48C02001418FF1FF4
:10205000B88C0200CC8C0200E48C0200141CFF1F20
:10206000F88C020003280BD8DFE800F00806040211
:102070001EF030BC1EF050B91DF096BD1FF0FCBB29
:102080000020704708B51DF07FFD002801DD01200C
:1020900008BD1EF031F9002801DD022008BD1EF048
:1020A00009FC0028D4BF0020032008BD38B50D4C22
:1020B0002068FFF7D7FFC5B202E02068FFF7D2FF24
:1020C000FFF7E0FF0028F8DC042107481FF03AFC86
:1020D0002946064820F016F9044820F0C3F828469F
:1020E00038BD00BF4807FF1F088D02002408FF1FEE
:1020F00008B5FFF7C7FF002808DB154B1868FFF786
:10210000B1FF144BC0B25328187001D0002008BD95
:10211000012200210320FEF7C1FC0F4B1B68012B9D
:1021200009D003D3022B0BD0012008BD0122104699
:102130000021FEF7B3FC012210460021FEF7AEFCA1
:10214000012200210220FEF7A9FC012008BD00BFEA
:102150004807FF1FF413FF1F0814FF1FF0B51C21D1
:1021600083B02748274C284D284E294F1FF0EAFB03
:10217000284820F077F80E2127481FF0E3FB21685C
:10218000244820F0BFF8234820F06CF80023019386
:1021900009E0019B306818441CF00CFF019B0133DF
:1021A000142B019314DC2868FFF75CFFC0B2FF28F2
:1021B0002368014619D0032BEBD1019B3A680146F5
:1021C000D0181CF0F7FE019B0133142B0193EADDBC
:1021D0002368032B0CBF114B114B042219680DEB24
:1021E00002001CF015FF03B0F0BD032B0CBF084A22
:1021F000064A019B1068002118441CF0DBFEE7E74B
:10220000108D02008007FF1F4807FF1F7C07FF1F7C
:102210004407FF1F2408FF1F308D02008807FF1F9F
:102220006007FF1F2DE9F04F95B0074604A81AF08C
:1022300007F988201FF0D6FF0823102280E80C0041
:10224000C61800F18808354634462046002110346F
:1022500020F0D6F9A045F8D11721BF481FF072FB36
:10226000BE481FF0FFFF0CA80123BD4ABD491AF06C
:10227000D7F90E9A9DF83C309DF8341006928DF8EF
:102280001C308DF814100FAA0DF11D030DF12A005A
:1022900012F8011F03F8011B8342F9D1139B0B9322
:1022A0000CA81AF0DBF804A81AF006F9002800F0D0
:1022B000AF8104A81AF0EEF80A210446AA481FF0DC
:1022C00041FB214600230A22A4481FF0DBFFA3485C
:1022D0001FF0C8FF002F4AD017F1060900F1B780A0
:1022E0000024A24610E0013C0CA81AF0E5F8804654
:1022F000002842D00CA81AF0D1F801340CA81AF02A
:10230000ADF84C4500F3A380012204A90CA81AF0F3
:10231000FBF90CA81AF0A4F8804623F051FF0146FF
:1023200040461FF00FFB8D481FF09CFF0CA81AF0D1
:1023300099F80028D7D10CA81AF092F801468B48DA
:1023400023F062FD0A2100285CD189481FF0FAFAC7
:102350000CA81AF085F8804623F032FF014640466B
:102360001FF0F0FA7D48013C1FF07CFFC2E7814B73
:1023700064221A604FF00609B2E70F217E48DFF8A9
:10238000F4B11FF0DFFA214674481FF0BBFF0321B0
:102390007A481FF0D7FADBF8001070481FF0B2FF40
:1023A00004F1080303217548CBF800301FF0CAFA86
:1023B000DBF8001069481FF0A5FF68481FF052FFC6
:1023C00068466F4920F01CF941466846FFF72CF932
:1023D000684620F0D5F82220FFF7A4FA631E00EE2D
:1023E000103A4046B8EEC00AFFF740FA6846654921
:1023F00020F006F968464146FFF716F9684620F0D6
:10240000BFF877E760481FF09DFA214653481FF058
:1024100079FF032159481FF095FA0CA81AF020F80B
:10242000804623F0CDFE014640461FF08BFA032183
:1024300052481FF087FAA74240F3F48006EB0A11D6
:1024400046481FF0E9FE45481FF00CFF4CE7012607
:10245000741E03214D481FF075FA21463F481FF0B6
:1024600051FF032145481FF06DFA29463B481FF0F4
:10247000D3FEB41E39481FF0F5FE052C04D8DFE862
:1024800004F068666462359541490CA820F0B8F8FC
:1024900000210CA8FFF7C8F80CA820F071F83D49FE
:1024A0000CA820F0ADF800210CA8FFF7BDF80CA88F
:1024B00020F066F829460CA820F0B6F800210CA8F8
:1024C000FFF7B2F80CA820F05BF82E490CA820F01A
:1024D00097F800210CA8FFF7A7F80CA820F050F8F7
:1024E000072E00F08F8010350136B1E72A490CA87D
:1024F00020F086F800210CA8FFF796F80CA820F031
:102500003FF824490CA820F07BF800210CA8FFF725
:102510008BF80CA820F034F829460CA820F084F899
:1025200000210CA8FFF780F80CA820F029F8154925
:102530000CA820F065F80CA80021FFF775F80CA88E
:1025400020F01EF8CFE71549D1E71549CFE7154927
:10255000CDE71549CBE700BF408D02002408FF1FDF
:10256000588D02006019FF1F5C8D0200788D0200FB
:10257000848D02007007FF1FA08D02009C8D020059
:10258000B08D0200C48D0200908D0200CC8D02003F
:10259000D08D0200E88D02004C8E0200348E0200C5
:1025A0001C8E0200048E0200EC8D020023490CA850
:1025B00020F026F800210CA8FFF736F80CA81FF031
:1025C000DFFF1F490CA820F01BF800210CA8FFF723
:1025D0002BF80CA81FF0D4FF29460CA820F024F8F3
:1025E00000210CA8FFF720F80CA81FF0C9FF15491F
:1025F0000CA820F005F80CA80021FFF715F80CA88E
:102600001FF0BEFF04A819F029FF15B0BDE8F08F38
:102610000E210D481FF096F904A819F01FFF15B000
:10262000BDE8F08F0CA819F01BFF06EB0A18014655
:10263000404620F06DF80AF1010AFFE6648E0200C0
:10264000E88D0200C48D0200688D020008B5084BB9
:10265000DFED080AD3ED007A27EE800A20F0DCFCDB
:1026600020F032FC044BD3ED007A20EE270A08BD9F
:102670006C14FF1FDB0FC9409415FF1F08B52C4ACF
:102680002C4B92ED010A93ED007ADFED2B6A2B4B78
:10269000B8EEC77A9B6BC6EE877A012BB8EEC00AFC
:1026A0002DED028B27EE800A3BD034D3022B2CD0A9
:1026B0009FED238AFFF7CAFF224A234B92ED007A4F
:1026C000002283F8902072B6DFED207A93ED206A25
:1026D000D3ED1F6A30EE480AB8EEC77AC0EE275A2B
:1026E000C5EE877A67EE867AF4EEE67AC3ED1E7A57
:1026F000D3ED227AF1EE10FAD8BFF1EE677AC3ED8E
:10270000237A62B6BDEC028B08BD114B93ED018AB2
:10271000B8EEC88ACEE70F4B93ED018AB8EEC88AAF
:10272000C8E70D4B93ED018AB8EEC88AC2E700BF37
:10273000B812FF1F5C19FF1FDB0FC9402013FF1FDA
:10274000000000006817FF1FD814FF1FCDCCCC3C41
:102750009416FF1FD417FF1F7017FF1F2DE9F04FAE
:102760001621ADB00446B1481FF0ECF8B0481FF098
:1027700079FD601E092800F27B84DFE810F09400E8
:10278000CD01A9026B0179042603F901D303D30318
:102790000A00A84B1D680DF15008C8EB050544461A
:1027A0002BAE28191CF0ECFB04F8010BA642F8D163
:1027B000A14907A81FF024FF002107A8FEF734FF56
:1027C00007A81FF0DDFE2220FFF7ACF8DDED147A3C
:1027D0000020B8EEE70AFFF749F8984907A81FF06C
:1027E0000FFF002107A8FEF71FFF07A81FF0C8FE74
:1027F000934907A81FF004FF002107A8FEF714FF64
:1028000007A81FF0BDFE2220FFF78CF8DDED187A37
:102810000020B8EE670AFFF729F8884907A81FF0DB
:10282000EFFE07A80021FEF7FFFE07A81FF0A8FE95
:10283000229B012B00F0EC86C0F0B886022B40F002
:102840009582804907A81FF0DBFE002107A8FEF74C
:10285000EBFE07A81FF094FE2220FFF763F8DDEDE2
:10286000177A0020B8EE670AFFF700F8734907A847
:102870001FF0C6FE002107A8FEF7D6FE07A81FF02E
:102880007FFE714907A81FF0BBFE002107A8FEF7D5
:10289000CBFE07A81FF074FE2220FFF743F80020AC
:1028A000DDED1B7A1AE3694B1D6807AC2E1B0DF199
:1028B000500830191CF064FB04F8010BA045F8D156
:1028C000C8EB050521AE444628191CF059FB04F855
:1028D000010BA642F8D1584903A81FF091FE002130
:1028E00003A8FEF7A1FE03A81FF04AFE584903A85B
:1028F0001FF086FE002103A8FEF796FE03A81FF036
:102900003FFEDDED087A0020B8EEE70AFEF7AEFFE5
:102910004A4903A81FF074FE002103A8FEF784FEB5
:1029200003A81FF02DFE464903A81FF069FE0021F1
:1029300003A8FEF779FE03A81FF022FE444903A86E
:102940001FF05EFE002103A8FEF76EFE03A81FF035
:1029500017FEDDED107A0020B8EEE70AFEF786FFDD
:10296000364903A81FF04CFE03A80021FEF75CFEC9
:1029700003A81FF005FE139C012C00F03B85022CE0
:1029800000F0D184002C40F0F1812E4903A81FF003
:1029900037FE214603A8FEF747FE03A81FF0F0FD0F
:1029A0002B4903A81FF02CFE214603A8FEF73CFE8E
:1029B00003A81FF0E5FDDDED097A2046B8EEE70A31
:1029C000FEF754FF1D4903A81FF01AFE214603A875
:1029D000FEF72AFE03A81FF0D3FD1B4903A81FF032
:1029E0000FFE214603A8FEF71FFE03A81FF0C8FD37
:1029F000174903A81FF004FE214603A8FEF714FEA2
:102A000003A81FF0BDFDDDED117A2046B8EEE70A00
:102A1000FEF72CFF094903A81FF0F2FD03A8214689
:102A2000FEF702FE03A81FF0ABFD9FE17C8E0200C3
:102A30002408FF1F3407FF1F948E0200C48D02007C
:102A4000A88E0200BC8E0200D08E02009007FF1FED
:102A5000E88D0200924B1D680DF15008C8EB05058A
:102A6000444624AE28191CF08BFA04F8010BA64248
:102A7000F8D1149A052A00F279810123934013F0CA
:102A8000240440F0E98313F0120540F03A8613F075
:102A9000090F00F06B8107A882491FF0B1FD29469C
:102AA00007A8FEF7C1FD07A81FF06AFD2220FEF768
:102AB00039FFDDED157A2846B8EEE70AFEF7D6FEB7
:102AC00007A879491FF09CFD294607A8FEF7ACFD31
:102AD00007A81FF055FD07A874491FF091FD29466E
:102AE00007A8FEF7A1FD07A81FF04AFD2220FEF768
:102AF00019FFDDED167A2846B8EE670AFEF7B6FE36
:102B000007A869491FF07CFD07A82946FEF78CFD40
:102B100007A81FF035FD29E1654B1D680DF1500830
:102B2000C8EB0505444621AE28191CF029FA04F823
:102B3000010BA642F8D11E9B5E4801930B21DDF8E4
:102B400054B0DDF874A0DDF85890179F1F9E189DB3
:102B5000149C1EF0F7FE58481FF084FB209B032BAB
:102B600000F20481DFE813F03003FC02C8028702A0
:102B7000524B1D680DF15008C8EB0505444629AEBF
:102B800028191CF0FDF904F8010BA642F8D14C49B4
:102B900007A81FF035FD002107A8FEF745FD07A88F
:102BA0001FF0EEFC2220FEF7BDFEDDED147A0020C2
:102BB000B8EEE70AFEF75AFE3B4907A81FF020FDD2
:102BC000002107A8FEF730FD07A81FF0D9FC3D49FA
:102BD00007A81FF015FD002107A8FEF725FD07A88F
:102BE0001FF0CEFC2220FEF79DFEDDED1C7A0020BA
:102BF000B8EE670AFEF73AFE2B4907A81FF000FD62
:102C0000002107A8FEF710FD07A81FF0B9FC072157
:102C10002D481EF097FE269C2748214600230A22B5
:102C20001FF030FB24481FF01DFB012C00F04883EF
:102C3000C0F01484022C40F099801A4907A81FF0B4
:102C4000DFFC002107A8FEF7EFFC07A81FF098FCA7
:102C50002220FEF767FE1D4B93ED030A0020B8EE1D
:102C6000C00AFEF703FE104907A81FF0C9FC0021A7
:102C700007A8FEF7D9FC07A81FF082FC0B4907A89C
:102C80001FF0BEFC002107A8FEF7CEFC07A81FF02E
:102C900077FC2220FEF746FE0020DDED1F7A1DE1C5
:102CA0006C07FF1FBC8E0200C48D0200D08E020094
:102CB0008407FF1F408F02002408FF1F3807FF1FF3
:102CC000948E0200A88E0200388F02008014FF1F2D
:102CD0008A4B1D6807AC2D1B0BAE28191CF050F950
:102CE00004F8010BA642F8D10DF150088449404682
:102CF0001FF086FC00214046FEF796FC40461FF080
:102D00003FFC2220FEF70EFEDDED087A0020B8EE33
:102D1000E70AFEF7ABFD7B4940461FF071FC00213E
:102D20004046FEF781FC40461FF02AFC76494046AB
:102D30001FF066FC00214046FEF776FC40461FF07F
:102D40001FFC2220FEF7EEFDDDED0A7A0020B8EE32
:102D5000670AFEF78BFD6B4940461FF051FC404669
:102D60000021FEF761FC40461FF00AFC674940461F
:102D70001FF046FC00214046FEF756FC40461FF07F
:102D8000FFFB634940461FF03BFC00214046FEF735
:102D90004BFC40461FF0F4FB5E4940461FF030FC00
:102DA00000214046FEF740FC40461FF0E9FB584931
:102DB00040461FF025FC00214046FEF735FC40460A
:102DC0001FF0DEFB2DB0BDE8F08F534B1D680DF1F9
:102DD0005008C8EB0505444624AE28191CF0D0F86D
:102DE00004F8010BA642F8D1454907A81FF008FCDA
:102DF000002107A8FEF718FC07A81FF0C1FB22203E
:102E0000FEF790FDDDED157A0020B8EEE70AFEF73B
:102E10002DFD3C4907A81FF0F3FB002107A8FEF792
:102E200003FC07A81FF0ACFB374907A81FF0E8FB1D
:102E3000002107A8FEF7F8FB07A81FF0A1FB22203E
:102E4000FEF770FDDDED167A0020B8EE670AFEF79A
:102E50000DFD2C4907A81FF0D3FB07A80021FEF7A2
:102E6000E3FB07A81FF08CFB149B012B00F02883C9
:102E7000C0F06A83022B7FF479AF284907A81FF0BE
:102E8000BFFB002107A8FEF7CFFB07A81FF078FBC8
:102E90002220FEF747FDDDED1B7A0020B8EEE70AA1
:102EA000FEF7E4FC174907A81FF0AAFB002107A8BA
:102EB000FEF7BAFB07A81FF063FB194907A81FF02C
:102EC0009FFB002107A8FEF7AFFB07A81FF058FBE8
:102ED0002220FEF727FDDDED1C7A0020B8EE670A00
:102EE000FEF7C4FC074907A81FF08AFB07A80021CA
:102EF000FEF79AFB07A81FF043FB37E78C07FF1F7D
:102F0000948E0200C48D0200A88E0200748F02000D
:102F1000B08B02008C8F02003C07FF1FBC8E0200AA
:102F2000D08E0200C24B1D680DF15008C8EB05059C
:102F300044462CAE28191CF023F804F8010BA642D5
:102F4000F8D1BC49BC4C07A81FF05AFB002107A8C8
:102F5000FEF76AFB07A81FF013FB2220FEF7E2FC36
:102F6000DDED207A0020B8EEE70AFEF77FFCB349DA
:102F700007A81FF045FB002107A8FEF755FB07A88F
:102F80001FF0FEFAAE4907A81FF03AFB002107A880
:102F9000FEF74AFB07A81FF0F3FA2220FEF7C2FC57
:102FA000289D07EE905A0020B8EE670AFEF75EFCF7
:102FB000A24907A81FF024FB002107A8FEF734FB55
:102FC00007A81FF0DDFA0F219E481EF0BBFC00236E
:102FD0000A22216D9C481FF055F99B481FF042F9C9
:102FE00016219A481EF0AEFC002329460A22964874
:102FF0001FF048F994481FF035F92368012B00F0C1
:103000004D83C0F01983022B7FF4B0AE904907A81E
:103010001FF0F6FA002107A8FEF706FB07A81FF02D
:10302000AFFA2220FEF77EFCDDED237A0020B8EE19
:10303000E70AFEF71BFC814907A81FF0E1FA00210F
:1030400007A8FEF7F1FA07A81FF09AFA814907A826
:103050001FF0D6FA002107A8FEF7E6FA07A81FF02E
:103060008FFA2220FEF75EFC0020DDED2B7A35E79B
:103070000DF150087AE66F4907A81FF0C1FA002148
:1030800007A8FEF7D1FA07A81FF07AFA2220FEF768
:1030900049FC07EE90BA0020B8EEE70AFEF7E6FB1F
:1030A000664907A81FF0ACFA002107A8FEF7BCFA92
:1030B00007A81FF065FA624907A81FF0A1FA0021CE
:1030C00007A8FEF7B1FA07A81FF05AFA2220FEF768
:1030D00029FC07EE90AAB8EEE70A0020FEF7C6FB2F
:1030E00007A856491FF08CFA07A80021FEF79CFAA2
:1030F00007A81FF045FA39E6554907A81FF080FADE
:10310000002107A8FEF790FA07A81FF039FA22203D
:10311000FEF708FC07EE905A0020B8EEE70AFEF72B
:10312000A5FB464907A81FF06BFA002107A8FEF788
:103130007BFA07A81FF024FA464907A81FF060FA97
:10314000002107A8FEF770FA07A81FF019FA22203D
:10315000FEF7E8FB07EE904A0020B8EEE70ABDE76D
:103160003B4907A81FF04CFA002107A8FEF75CFABC
:1031700007A81FF005FA2220FEF7D4FB07EE907A8D
:103180000020B8EEE70AFEF771FB2C4907A81FF0F4
:1031900037FA002107A8FEF747FA07A81FF0F0F951
:1031A0002C4907A81FF02CFA002107A8FEF73CFACB
:1031B00007A81FF0E5F92220FEF7B4FB07EE906A9E
:1031C0000020B8EEE70A89E7214907A81FF018FA9E
:1031D000002107A8FEF728FA07A81FF0D1F922203E
:1031E000FEF7A0FB07EE909A0020B8EEE70AFEF784
:1031F0003DFB124907A81FF003FA002107A8FEF7BC
:1032000013FA07A81FF0BCF9124907A81FF0F8F934
:10321000002107A8FEF708FA07A81FF0B1F922203D
:10322000FEF780FBDDED017A0020B8EEE70A55E7F6
:103230004C07FF1F948E02000814FF1FC48D02006C
:10324000A88E02004C8F02002408FF1F5C8F020032
:10325000BC8E0200D08E0200B24907A81FF0D0F940
:10326000002107A8FEF7E0F907A81FF089F922203E
:10327000FEF758FBDDED1B7A0020B8EEE70AFEF7FB
:10328000F5FAA94907A81FF0BBF9002107A8FEF726
:10329000CBF907A81FF074F9A44907A81FF0B0F9EB
:1032A000002107A8FEF7C0F907A81FF069F922203E
:1032B000FEF738FBDDED1C7A0020B8EE670A0DE75B
:1032C000984907A81FF09CF9002107A8FEF7ACF960
:1032D00007A81FF055F92220FEF724FB944B93ED2D
:1032E000020A0020B8EEC00AFEF7C0FA8E4907A80D
:1032F0001FF086F9002107A8FEF796F907A81FF02E
:103300003FF98A4907A81FF07BF9002107A8FEF7BB
:103310008BF907A81FF034F92220FEF703FB0020E9
:10332000DDED1E7ADAE5182182481EF00BFB824B98
:10333000824819681EF0E6FF80481EF093FF1921AD
:103340007F481EF0FFFA14997C481EF0DBFF7B4893
:103350001EF088FF18217B481EF0F4FA079C77487E
:1033600021461EF0CFFF75481EF07CFF6D4903A873
:103370001FF046F9002103A8FEF756F903A81FF035
:10338000FFF82220FEF7CEFADDED0B7A0020B8EE32
:10339000E70AFEF76BFA644903A81FF031F9002130
:1033A00003A8FEF741F903A81FF0EAF864201BF018
:1033B000E9FF5E4903A81FF023F9002103A8FEF7E7
:1033C00033F903A81FF0DCF82220FEF7ABFA07EE72
:1033D000904AB8EEE70A0020FEF748FA524903A8DF
:1033E0001FF00EF903A80021FEF71EF903A81FF035
:1033F000C7F8BBE44B4903A81FF002F9002103A85A
:10340000FEF712F903A81FF0BBF82220FEF78AFA94
:10341000DDED0A7A0020B8EEE70AFEF727FA424906
:1034200003A81FF0EDF8002103A8FEF7FDF803A89C
:103430001FF0A6F83D4903A81FF0E2F8002103A8F9
:10344000FEF7F2F803A81FF09BF82220FEF76AFAB5
:10345000DDED127A0020B8EEE70ABDE7314907A892
:103460001FF0CEF8002107A8FEF7DEF807A81FF02E
:1034700087F82220FEF756FADDED157A0020B8EE27
:10348000E70AFEF7F3F9284907A81FF0B9F8002169
:1034900007A8FEF7C9F807A81FF072F8234907A884
:1034A0001FF0AEF8002107A8FEF7BEF807A81FF02E
:1034B00067F82220FEF736FA0020DDED1D7A0DE5D3
:1034C000184907A81FF09CF8002107A8FEF7ACF8E0
:1034D00007A81FF055F82220FEF724FADDED197A2F
:1034E000B8EEE70A0020FEF7C1F90F4907A81FF060
:1034F00087F8002107A8FEF797F807A81FF040F803
:103500000A4907A81FF07CF8002107A8FEF78CF8ED
:1035100007A81FF035F82220FEF704FA0020DDEDA1
:103520001A7ADBE4BC8E0200C48D0200D08E020049
:103530008014FF1FE48E02002819FF1F2408FF1FBC
:10354000008F02001C8F02008F4907A81FF058F857
:10355000002107A8FEF768F807A81FF011F822203D
:10356000FEF7E0F9DDED177A0020B8EEE70AFEF786
:103570007DF9864907A81FF043F8002107A8FEF748
:1035800053F807A81EF0FCFF814907A81FF038F880
:10359000002107A8FEF748F807A81EF0F1FF222037
:1035A000FEF7C0F90020DDED187A97E4764907A808
:1035B0001FF026F8002107A8FEF736F807A81EF02E
:1035C000DFFF2220FEF7AEF9DDED157A0020B8EE20
:1035D000E70AFEF74BF96D4907A81FF011F8002123
:1035E00007A8FEF721F807A81EF0CAFF684907A838
:1035F0001FF006F8002107A8FEF716F807A81EF02E
:10360000BFFF2220FEF78EF90020DDED197A65E478
:103610005D4907A81EF0F4FF002107A8FEF704F893
:1036200007A81EF0ADFF2220FEF77CF9DDED167A2B
:103630000020B8EE670A56E7534907A81EF0E0FFDE
:10364000002107A8FDF7F0FF07A81EF099FF222030
:10365000FEF768F9DDED217A0020B8EEE70AFEF703
:1036600005F94A4907A81EF0CBFF002107A8FDF77E
:10367000DBFF07A81EF084FF454907A81EF0C0FF26
:10368000002107A8FDF7D0FF07A81EF079FF222030
:10369000FEF748F90020DDED297A1FE43A4907A832
:1036A0001EF0AEFF002107A8FDF7BEFF07A81EF021
:1036B00067FF2220FEF736F9DDED227A0020B8EE12
:1036C000E70AFEF7D3F8314907A81EF099FF002159
:1036D00007A8FDF7A9FF07A81EF052FF2C4907A86D
:1036E0001EF08EFF002107A8FDF79EFF07A81EF021
:1036F00047FF2220FEF716F90020DDED2A7AFFF7BA
:10370000EDBB07A820491EF07BFF214607A8FDF767
:103710008BFF07A81EF034FF2220FEF703F9DDED32
:10372000187A2046B8EEE70AFEF7A0F807A817496E
:103730001EF066FF214607A8FDF776FF07A81EF0DA
:103740001FFF07A812491EF05BFF214607A8FDF7DF
:103750006BFF07A81EF014FF2220FEF7E3F8DDED53
:10376000197A2046B8EE670AFEF780F807A80749DD
:103770001EF046FF07A82146FDF756FF07A81EF0DA
:10378000FFFEFFF7F3BA00BFBC8E0200C48D02003B
:10379000D08E020070B5E84BAEB01D6804AC2D1B96
:1037A0002EAE28191BF0ECFB04F8010BB442F8D143
:1037B000E249E34DE34C68461EF022FF00216846D3
:1037C000FDF732FF68461EF0DBFE2220FEF7AAF866
:1037D000DDED047A0020B8EE670AFEF747F8DA4913
:1037E00068461EF00DFF00216846FDF71DFF684684
:1037F0001EF0C6FED54968461EF002FF002168464D
:10380000FDF712FF68461EF0BBFE2220FEF78AF885
:10381000DDED057A0020B8EE670AFEF727F8CA4901
:1038200068461EF0EDFE00216846FDF7FDFE684685
:103830001EF0A6FEC64968461EF0E2FE002168465C
:10384000FDF7F2FE68461EF09BFE2220FEF76AF8A6
:103850009DED060A0420FEF709F8BB4968461EF0F4
:10386000CFFE00216846FDF7DFFE68461EF088FEA9
:10387000B84968461EF0C4FE00216846FDF7D4FE34
:1038800068461EF07DFE2220FEF74CF89DF884105D
:103890006846002914BF294621461EF0B1FE0021CA
:1038A0006846FDF7C1FE68461EF06AFEA6496846F6
:1038B0001EF0A6FE00216846FDF7B6FE68461EF023
:1038C0005FFEA54968461EF09BFE00216846FDF795
:1038D000ABFE68461EF054FE2220FEF723F8DDED15
:1038E000257A0020B8EE670AFDF7C0FF96496846C2
:1038F0001EF086FE00216846FDF796FE68461EF023
:103900003FFE964968461EF07BFE00216846FDF7A3
:103910008BFE68461EF034FE2220FEF703F8DDED34
:10392000267A0020B8EE670AFDF7A0FF86496846B0
:103930001EF066FE00216846FDF776FE68461EF022
:103940001FFE874968461EF05BFE00216846FDF7B2
:103950006BFE68461EF014FE2220FDF7E3FFDDED4E
:10396000077A0020B8EE670AFDF780FF76496846BF
:103970001EF046FE00216846FDF756FE68461EF022
:10398000FFFD784968461EF03BFE00216846FDF7C2
:103990004BFE68461EF0F4FD2220FDF7C3FFDDED6F
:1039A000087A0020B8EE670AFDF760FF66496846AE
:1039B0001EF026FE00216846FDF736FE68461EF022
:1039C000DFFD694968461EF01BFE00216846FDF7D1
:1039D0002BFE68461EF0D4FD2220FDF7A3FF9DEDCF
:1039E000090A0420FDF742FF574968461EF008FE09
:1039F00000216846FDF718FE68461EF0C1FD5B49D0
:103A000068461EF0FDFD00216846FDF70DFE684684
:103A10001EF0B6FD2220FDF785FF9DF88510684653
:103A2000002914BF294621461EF0EAFD0021684600
:103A3000FDF7FAFD68461EF0A3FD434968461EF0F7
:103A4000DFFD00216846FDF7EFFD68461EF098FD9A
:103A5000474968461EF0D4FD00216846FDF7E4FDA5
:103A600068461EF08DFD2220FDF75CFFDDED0C7A2F
:103A70000020B8EE670AFDF7F9FE334968461EF0EC
:103A8000BFFD00216846FDF7CFFD68461EF078FDBA
:103A9000384968461EF0B4FD00216846FDF7C4FDB4
:103AA00068461EF06DFD2220FDF73CFFDDED0D7A2E
:103AB0000020B8EE670AFDF7D9FE234968461EF0DC
:103AC0009FFD00216846FDF7AFFD68461EF058FDDA
:103AD000294968461EF094FD00216846FDF7A4FDC3
:103AE00068461EF04DFD2220FDF71CFF9DED0E0ADD
:103AF0000520FDF7BBFE144968461EF081FD00213C
:103B00006846FDF791FD68461EF03AFD1B49684680
:103B10001EF076FD00216846FDF786FD68461EF022
:103B20002FFD2220FDF7FEFE9DF886106846002935
:103B300014BF2946214623E07C14FF1FB08F0200EA
:103B4000A48F0200A88F0200C48D0200C88F02005B
:103B5000E08F0200F88F0200109002002490020013
:103B60003C9002004C9002005C9002006C900200BD
:103B70007C9002008C9002009C900200AC900200AD
:103B80001EF03EFD00216846FDF74EFD68461EF022
:103B9000F7FCE84968461EF033FD00216846FDF752
:103BA00043FD68461EF0ECFCE34968461EF028FD24
:103BB00000216846FDF738FD68461EF0E1FC222032
:103BC000FDF7B0FEDDED297A0020B8EE670AFDF7BB
:103BD0004DFED84968461EF013FD00216846FDF7EA
:103BE00023FD68461EF0CCFCD44968461EF008FD53
:103BF00000216846FDF718FD68461EF0C1FC222032
:103C0000FDF790FEDDED2A7A0020B8EE670AFDF799
:103C10002DFEC84968461EF0F3FC00216846FDF7FA
:103C200003FD68461EF0ACFCC54968461EF0E8FC82
:103C300000216846FDF7F8FC68461EF0A1FC222032
:103C4000FDF770FE9DED2B0A0520FDF70FFEB9492B
:103C500068461EF0D5FC00216846FDF7E5FC684685
:103C60001EF08EFCB74968461EF0CAFC002168466B
:103C7000FDF7DAFC68461EF083FC2220FDF752FEB9
:103C80009DF8B0106846002914BF294621461EF051
:103C9000B7FC00216846FDF7C7FC68461EF070FCC3
:103CA000A44968461EF0ACFC68460021FDF7BCFC48
:103CB00068461EF065FC289B012B00F0E581A249B7
:103CC00068461EF09DFC00216846FDF7ADFC684685
:103CD0001EF056FC9D4968461EF092FC0021684685
:103CE000FDF7A2FC68461EF04BFC994968461EF0A1
:103CF00087FC00216846FDF797FC68461EF040FCF3
:103D0000924968461EF07CFC00216846FDF78CFC59
:103D100068461EF035FC8F4968461EF071FC002194
:103D20006846FDF781FC68461EF02AFC8749684614
:103D30001EF066FC00216846FDF776FC68461EF022
:103D40001FFC854968461EF05BFC00216846FDF7B4
:103D50006BFC68461EF014FC7C4968461EF050FC63
:103D600000216846FDF760FC68461EF009FC7B49AF
:103D700068461EF045FC00216846FDF755FC684684
:103D80001EF0FEFB2220FDF7CDFDDDED127A0020B6
:103D9000B8EE670AFDF76AFD664968461EF030FC1A
:103DA00000216846FDF740FC68461EF0E9FB6C49BF
:103DB00068461EF025FC00216846FDF735FC684684
:103DC0001EF0DEFB2220FDF7ADFDDDED137A0020B5
:103DD000B8EE670AFDF74AFD564968461EF010FC2A
:103DE00000216846FDF720FC68461EF0C9FB5D49CE
:103DF00068461EF005FC00216846FDF715FC684684
:103E00001EF0BEFB2220FDF78DFD9DED140A04205F
:103E1000FDF72CFD474968461EF0F2FB002168467D
:103E2000FDF702FC68461EF0ABFB4F4968461EF0EA
:103E3000E7FB00216846FDF7F7FB68461EF0A0FB94
:103E40002220FDF76FFD494A494B9DF887106846CF
:103E5000002914BF114619461EF0D2FB0021684606
:103E6000FDF7E2FB68461EF08BFB324968461EF008
:103E7000C7FB00216846FDF7D7FB68461EF080FBB4
:103E8000119C002C00F0BC803A4968461EF0B8FB3B
:103E900000216846FDF7C8FB68461EF071FB2B4900
:103EA00068461EF0ADFB00216846FDF7BDFB684685
:103EB0001EF066FB304968461EF0A2FB00216846F2
:103EC000FDF7B2FB68461EF05BFB204968461EF01A
:103ED00097FB68460021FDF7A7FB68461EF050FBE4
:103EE000264968461EF08CFB00216846FDF79CFBC6
:103EF00068461EF045FB2220FDF714FD9DED150AD6
:103F00000420FDF7B3FC0B4968461EF079FB002145
:103F10006846FDF789FB68461EF032FB2D9C002C9D
:103F200000F09B80164968461EF06AFB0021684637
:103F300028E000BFC48D0200BC900200D4900200B3
:103F4000EC900200049102006C910200B08B020020
:103F50007C9102008C910200A4910200BC910200AD
:103F6000CC910200DC910200EC910200A48F0200CF
:103F7000A88F0200FC9102000C9202003C92020009
:103F800060920200FDF750FB68461EF0F9FA6049A6
:103F900068461EF035FB68460021FDF745FB684684
:103FA0001EF0EEFA5B4968461EF02AFB00216846C7
:103FB000FDF73AFB68461EF0E3FA554968461EF0E5
:103FC0001FFB00216846FDF72FFB68461EF0D8FA5C
:103FD000514968461EF014FB00216846FDF724FB9A
:103FE00068461EF0CDFA4A4968461EF009FB0021DA
:103FF0006846FDF719FB68461EF0C2FA2EB070BD88
:10400000464968461EF0FCFA21466846FDF70CFB5F
:1040100068461EF0B5FA3E4968461EF0F1FA2146A0
:104020006846FDF701FB68461EF0AAFA3C4968465F
:104030001EF0E6FA21466846FDF7F6FA68461EF0DD
:104040009FFA334968461EF0DBFA68462146FDF7C1
:10405000EBFA68461EF094FA42E7324968461EF0D1
:10406000CFFA21466846FDF7DFFA68461EF088FA67
:10407000274968461EF0C4FA68462146FDF7D4FA7F
:1040800068461EF07DFA8DE7274968461EF0B8FAAB
:1040900000216846FDF7C8FA68461EF071FA1C490F
:1040A00068461EF0ADFA00216846FDF7BDFA684685
:1040B0001EF066FA1D4968461EF0A2FA0021684605
:1040C000FDF7B2FA68461EF05BFA114968461EF029
:1040D00097FA00216846FDF7A7FA68461EF050FAE5
:1040E000134968461EF08CFA00216846FDF79CFAD9
:1040F00068461EF045FA064968461EF081FA00211E
:104100006846FDF791FA68461EF03AFA094919E641
:10411000B08B0200749202008C9202001C9202008A
:104120002C9202004C9202001C9102002C91020081
:104130003C9102005491020070B5C84BAEB01D68AE
:1041400004AC2D1B2EAE28191AF01AFF04F8010B2F
:10415000A642F8D1C249C34C68461EF051FA00216C
:104160006846FDF761FA68461EF00AFA2220FDF75C
:10417000D9FBD4ED067A0020B8EE670AFDF776FB8E
:10418000B94968461EF03CFA00216846FDF74CFA32
:1041900068461EF0F5F9B54968461EF031FA00216F
:1041A0006846FDF741FA68461EF0EAF92220FDF75D
:1041B000B9FBD4ED077A0020B8EE670AFDF756FB8D
:1041C000A94968461EF01CFA00216846FDF72CFA42
:1041D00068461EF0D5F9A64968461EF011FA00217E
:1041E0006846FDF721FA68461EF0CAF92220FDF75D
:1041F00099FBD4ED1E7A0020B8EE670AFDF736FB76
:10420000994968461EF0FCF900216846FDF70CFA52
:1042100068461EF0B5F9974968461EF0F1F900218D
:104220006846FDF701FA68461EF0AAF92220FDF75C
:1042300079FBD4ED0B7A0020B8EE670AFDF716FB88
:10424000894968461EF0DCF900216846FDF7ECF963
:1042500068461EF095F9884968461EF0D1F900219C
:104260006846FDF7E1F968461EF08AF92220FDF75D
:1042700059FBD4ED0C7A0020B8EE670AFDF7F6FA88
:10428000794968461EF0BCF900216846FDF7CCF973
:1042900068461EF075F9794968461EF0B1F90021AB
:1042A0006846FDF7C1F968461EF06AF92220FDF75D
:1042B00039FBD4ED1F7A0020B8EE670AFDF7D6FA75
:1042C000694968461EF09CF900216846FDF7ACF983
:1042D00068461EF055F96A4968461EF091F90021BA
:1042E0006846FDF7A1F968461EF04AF92220FDF75D
:1042F00019FBD4ED137A0020B8EE670AFDF7B6FA81
:10430000594968461EF07CF900216846FDF78CF992
:1043100068461EF035F95B4968461EF071F90021C8
:104320006846FDF781F968461EF02AF92220FDF75C
:10433000F9FAD4ED147A0020B8EE670AFDF796FA80
:10434000494968461EF05CF900216846FDF76CF9A2
:1043500068461EF015F94C4968461EF051F90021D7
:104360006846FDF761F968461EF00AF92220FDF75C
:10437000D9FAD4ED207A0020B8EE670AFDF776FA74
:10438000394968461EF03CF900216846FDF74CF9B2
:1043900068461EF0F5F80D213C481DF0D3FAD4F81C
:1043A0008C103B4800230A221DF06CFF38481DF09A
:1043B00059FFD4F88C40002C43D1364968461EF092
:1043C0001FF968462146FDF72FF968461EF0D8F818
:1043D000314968461EF014F900216846FDF724F9BA
:1043E00068461EF0CDF82D4968461EF009F90021F7
:1043F0006846FDF719F968461EF0C2F82649684676
:104400001EF0FEF800216846FDF70EF968461EF022
:10441000B7F8234968461EF0F3F800216846FDF717
:1044200003F968461EF0ACF81B4968461EF0E8F830
:1044300000216846FDF7F8F868461EF0A1F82EB096
:1044400070BD184968461EF0DBF868460021FDF78C
:10445000EBF868461EF094F8BAE700BF7C14FF1F23
:10446000A0920200E815FF1FC48D0200B492020062
:10447000C8920200DC920200F09202000493020053
:10448000189302002C930200409302005493020000
:104490002408FF1F78930200B08B02008C93020067
:1044A000A89302006493020070B59D4BAEB01D68E6
:1044B00004AC2D1B2EAE28191AF062FD04F8010B76
:1044C000B442F8D1684697491EF09AF80021684630
:1044D000FDF7AAF868461EF053F82220FDF722FAED
:1044E000DDED197A0020B8EEE70AFDF7BFF968465E
:1044F0008D491EF085F868460021FDF795F868465D
:104500001EF03EF8684689491EF07AF80021684698
:10451000FDF78AF868461EF033F82220FDF702FA0C
:10452000DDED1A7A0020B8EE670AFDF79FF96846BC
:104530007D491EF065F868460021FDF775F868466C
:104540001EF01EF868467A491EF05AF800216846A7
:10455000FDF76AF868461EF013F82220FDF7E2F92D
:10456000DDED1B7A0020B8EEE70AFDF77FF968461B
:104570006D491EF045F868460021FDF755F868467C
:104580001DF0FEFF68466B491EF03AF800216846B0
:10459000FDF74AF868461DF0F3FF2220FDF7C2F947
:1045A000DDED1C7A0020B8EE670AFDF75FF968467A
:1045B0005D491EF025F868460021FDF735F868468C
:1045C0001DF0DEFF68465C491EF01AF800216846BF
:1045D000FDF72AF868461DF0D3FF2220FDF7A2F967
:1045E000DDED1D7A0020B8EEE70AFDF73FF96846D9
:1045F0004D491EF005F868460021FDF715F868469C
:104600001DF0BEFF68464D491DF0FAFF00216846C7
:10461000FDF70AF868461DF0B3FF2220FDF782F986
:10462000DDED1E7A0020B8EE670AFDF71FF9684637
:104630003D491DF0E5FF68460021FCF7F5FF68469F
:104640001DF09EFF68463E491DF0DAFF00216846D6
:10465000FCF7EAFF68461DF093FF2220FDF762F9A0
:10466000DDED1F7A0020B8EEE70AFDF7FFF8684697
:104670002D491DF0C5FF68460021FCF7D5FF6846AF
:104680001DF07EFF68462F491DF0BAFF00216846E5
:10469000FCF7CAFF68461DF073FF2220FDF742F9C0
:1046A000DDED207A0020B8EE670AFDF7DFF86846F6
:1046B0001D491DF0A5FF68460021FCF7B5FF6846BF
:1046C0001DF05EFF684620491DF09AFF68460021F4
:1046D000FCF7AAFF68461DF053FF68461B491DF012
:1046E0008FFF68460021FCF79FFF68461DF048FFDA
:1046F000684617491DF084FF68460021FCF794FFC7
:1047000068461DF03DFF684610491DF079FF684678
:104710000021FCF789FF68461DF032FF2EB070BD06
:104720007C14FF1FC0930200C48D0200D4930200CA
:10473000E8930200FC93020010940200249402000B
:10474000389402004C94020064940200B08B020082
:104750008094020070B5DA4B1B68013B84B0092BD2
:1047600000F2AC81DFE813F0580348045304C1049D
:10477000AA01E8042A064A070A00D001D149D24D0D
:1047800068461DF03DFF00216846FCF74DFF684676
:104790001DF0F6FE2220FDF7C5F8D5ED0C7A0020BD
:1047A000B8EEE70AFDF762F8C84968461DF028FF31
:1047B00000216846FCF738FF68461DF0E1FEC44959
:1047C00068461DF01DFF00216846FCF72DFF684676
:1047D0001DF0D6FE2220FDF7A5F8D5ED147A0020B5
:1047E000B8EE670AFDF742F8B84968461DF008FFC1
:1047F00000216846FCF718FF68461DF0C1FEB54968
:1048000068461DF0FDFE00216846FCF70DFF684676
:104810001DF0B6FE2220FDF785F8D5ED107A0020B8
:10482000B8EEE70AFDF722F8A84968461DF0E8FE51
:1048300000216846FCF7F8FE68461DF0A1FEA64977
:1048400068461DF0DDFE00216846FCF7EDFE684677
:104850001DF096FE2220FDF765F8D5ED077A0020C1
:10486000B8EEE70AFDF702F8984968461DF0C8FE61
:1048700000216846FCF7D8FE68461DF081FE974986
:1048800068461DF0BDFE00216846FCF7CDFE684677
:104890001DF076FE2220FDF745F895ED080A002070
:1048A000FCF7E4FF894968461DF0AAFE002168462E
:1048B000FCF7BAFE68461DF063FE894968461DF0A4
:1048C0009FFE00216846FCF7AFFE68461DF058FECB
:1048D0002220FDF727F895ED0B0A0020FCF7C6FF14
:1048E0007A4968461DF08CFE68460021FCF79CFE64
:1048F00068461DF045FEAE6A6C46002E02F0BB8095
:10490000012E23D1774968461DF07AFE00216846C2
:10491000FCF78AFE68461DF033FE2220FDF702F800
:10492000714968461DF06CFE00216846FCF77CFE6C
:1049300068461DF025FE654968461DF061FE684623
:104940000021FCF771FE68461DF01AFE6B6A022B0F
:1049500002F08080032B23D1644920461DF050FED5
:1049600000212046FCF760FE20461DF009FE2220B3
:10497000FCF7D8FF5E4920461DF042FE002120468C
:10498000FCF752FE20461DF0FBFD504920461DF06D
:1049900037FE20460021FCF747FE20461DF0F0FDC3
:1049A0002B68494D012B00F0B387C0F01C87022B08
:1049B00040F084804F4920461DF022FE0021204611
:1049C000FCF732FE20461DF0DBFD2220FCF7AAFF9B
:1049D000494920461DF014FE00212046FCF724FE24
:1049E00020461DF0CDFD394920461DF009FE00216D
:1049F0002046FCF719FE20461DF0C2FD3F49204627
:104A00001DF0FEFD00212046FCF70EFE20461DF0A5
:104A1000B7FD2220FCF786FFD5ED0F7A0020B8EE17
:104A2000E70AFCF723FF294920461DF0E9FD002194
:104A30002046FCF7F9FD20461DF0A2FD3049204636
:104A40001DF0DEFD00212046FCF7EEFD20461DF0A6
:104A500097FD2220FCF766FFD5ED177A0020B8EE0F
:104A6000670AFCF703FF194920461DF0C9FD002124
:104A70002046FCF7D9FD20461DF082FD2149204645
:104A80001DF0BEFD00212046FCF7CEFD20461DF0A6
:104A900077FD2220FCF746FF95ED130A0020B8EEC3
:104AA000C00AFCF7E3FE094920461DF0A9FD204697
:104AB0000021FCF7B9FD20461DF062FD04B070BD79
:104AC0008007FF1F989402000814FF1FC48D020086
:104AD000AC940200C09402002495020038950200B4
:104AE00084950200B49502005C970200989502003C
:104AF000EC950200D4940200CC9B0200E8940200E2
:104B0000FC94020010950200B549B64C68461DF0B1
:104B100077FD00216846FCF787FD68461DF030FDF3
:104B20002220FCF7FFFED4ED007A0020B8EEE70A61
:104B3000FCF79CFEAC4968461DF062FD002168460A
:104B4000FCF772FD68461DF01BFDA84968461DF084
:104B500057FD00216846FCF767FD68461DF010FD13
:104B60002220FCF7DFFED4ED047A0020B8EE670ABD
:104B7000FCF77CFE9C4968461DF042FD002168461A
:104B8000FCF752FD68461DF0FBFC994968461DF094
:104B900037FD00216846FCF747FD68461DF0F0FC34
:104BA0002220FCF7BFFED4ED087A0020B8EEE70A19
:104BB000FCF75CFE8C4968461DF022FD002168462A
:104BC000FCF732FD68461DF0DBFC8A4968461DF0A3
:104BD00017FD00216846FCF727FD68461DF0D0FC54
:104BE0002220FCF79FFED4ED0C7A0020B8EEE70AF5
:104BF000FCF73CFE7C4968461DF002FD002168463A
:104C0000FCF712FD68461DF0BBFC7B4968461DF0B1
:104C1000F7FC00216846FCF707FD68461DF0B0FC74
:104C20002220FCF77FFED4ED0D7A0020B8EEE70AD3
:104C3000FCF71CFE6C4968461DF0E2FC002168464A
:104C4000FCF7F2FC68461DF09BFC6C4968461DF0C1
:104C5000D7FC00216846FCF7E7FC68461DF090FC95
:104C60002220FCF75FFE94ED160A0020FCF7FEFD03
:104C70005D4968461DF0C4FC68460021FCF7D4FC81
:104C800068461DF07DFCA36B012B02F00283C2F08D
:104C90006982022B7FF412AF594968461DF0B0FCBF
:104CA00000216846FCF7C0FC68461DF069FC222024
:104CB000FCF738FE534968461DF0A2FC0021684607
:104CC000FCF7B2FC68461DF05BFC474968461DF0E6
:104CD00097FC00216846FCF7A7FC68461DF050FCD5
:104CE000494968461DF08CFC00216846FCF79CFC95
:104CF00068461DF045FC2220FCF714FED4ED037A33
:104D00000020B8EE670AFCF7B1FD374968461DF090
:104D100077FC00216846FCF787FC68461DF030FCF4
:104D20003A4968461DF06CFC00216846FCF77CFCA3
:104D300068461DF025FC2220FCF7F4FDD4ED077A2F
:104D40000020B8EE670AFCF791FD274968461DF080
:104D500057FC00216846FCF767FC68461DF010FC14
:104D60002B4968461DF04CFC00216846FCF75CFCB2
:104D700068461DF005FC2220FCF7D4FDD4ED0B7A2B
:104D80000020B8EEE70AFCF771FD174968461DF0F0
:104D900037FC00216846FCF747FC68461DF0F0FB35
:104DA0001C4968461DF02CFC00216846FCF73CFCC1
:104DB00068461DF0E5FB2220FCF7B4FD94ED150AD2
:104DC0000020FCF753FD084968461DF019FC00213E
:104DD0006846FCF729FC68461DF0D2FB04B070BDA4
:104DE000989402002013FF1FC48D0200AC940200AF
:104DF000C0940200249502003895020084950200B8
:104E0000D4940200CC9B0200E8940200FC940200BF
:104E100010950200B4950200BA49BB4C68461DF0DB
:104E2000EFFB00216846FCF7FFFB68461DF0A8FB7E
:104E30002220FCF777FDD4ED017A0020B8EEE70AD6
:104E4000FCF714FDB14968461DF0DAFB0021684605
:104E5000FCF7EAFB68461DF093FBAD4968461DF080
:104E6000CFFB00216846FCF7DFFB68461DF088FB9E
:104E70002220FCF757FDD4ED097A0020B8EEE70AAE
:104E8000FCF7F4FCA14968461DF0BAFB0021684616
:104E9000FCF7CAFB68461DF073FB9E4968461DF08F
:104EA000AFFB00216846FCF7BFFB68461DF068FBBE
:104EB0002220FCF737FDD4ED057A0020B8EEE70A92
:104EC000FCF7D4FC914968461DF09AFB6846002126
:104ED000FCF7AAFB68461DF053FB256B012D01F082
:104EE0005086022D01F0C686002D7FF4E7AD8A4979
:104EF00068461DF085FB29466846FCF795FB684629
:104F00001DF03EFB2220FCF70DFD844968461DF094
:104F100077FB29466846FCF787FB68461DF030FBA7
:104F20007A4968461DF06CFB29466846FCF77CFB15
:104F300068461DF025FB7A4968461DF061FB29464D
:104F40006846FCF771FB68461DF01AFB2220FCF74F
:104F5000E9FCD4ED027A2846B8EEE70AFCF786FCB5
:104F60006A4968461DF04CFB29466846FCF75CFB25
:104F700068461DF005FB6B4968461DF041FB29465C
:104F80006846FCF751FB68461DF0FAFA2220FCF750
:104F9000C9FCD4ED0A7A2846B8EEE70AFCF766FCAD
:104FA0005A4968461DF02CFB29466846FCF73CFB35
:104FB00068461DF0E5FA5C4968461DF021FB29466C
:104FC0006846FCF731FB68461DF0DAFA2220FCF750
:104FD000A9FC94ED060A2846B8EEC00AFCF746FC88
:104FE0004A4968461DF00CFB68462946FCF71CFB45
:104FF00068461DF0C5FA61E54C4C236B032B3FF668
:105000005DADDFE813F00B07960621067C053D49F0
:10501000474D68461DF0F4FA00216846FCF704FB92
:1050200068461DF0ADFA2220FCF77CFCD5ED017A34
:105030000020B8EEE70AFCF719FC344968461DF079
:10504000DFFA00216846FCF7EFFA68461DF098FA8F
:105050002F4968461DF0D4FA00216846FCF7E4FAAF
:1050600068461DF08DFA2220FCF75CFCD5ED037A32
:105070000020B8EE670AFCF7F9FB244968461DF0EA
:10508000BFFA00216846FCF7CFFA68461DF078FAAF
:10509000204968461DF0B4FA00216846FCF7C4FABE
:1050A00068461DF06DFA2220FCF73CFCD5ED027A33
:1050B0000020B8EEE70AFCF7D9FB144968461DF05A
:1050C0009FFA68460021FCF7AFFA68461DF058FACF
:1050D0002B68013B6C46042B3FF6F0ACDFE813F085
:1050E000CD071307BC07AB079A07124C2368052BA3
:1050F0003FF6E4ACDFE813F08E081E0B740ADD09FE
:105100004609F807989402002819FF1FC48D020071
:10511000AC940200C0940200D4940200049B0200EC
:10512000E8940200FC94020010950200C013FF1FD7
:105130007015FF1FA815FF1F9449954D68461DF077
:105140005FFA00216846FCF76FFA68461DF018FA0E
:105150002220FCF7E7FBD5ED017A0020B8EEE70A44
:10516000FCF784FB8B4968461DF04AFA002168462B
:10517000FCF75AFA68461DF003FA874968461DF0A5
:105180003FFA00216846FCF74FFA68461DF0F8F92F
:105190002220FCF7C7FBD5ED027A0020B8EE670AA3
:1051A000FCF764FB7B4968461DF02AFA002168463B
:1051B000FCF73AFA68461DF0E3F9784968461DF0B5
:1051C0001FFA00216846FCF72FFA68461DF0D8F94F
:1051D0002220FCF7A7FBD5ED097A0020B8EEE70AFC
:1051E000FCF744FB6B4968461DF00AFA684600214B
:1051F000FCF71AFA68461DF0C3F96B6B012B6C467D
:1052000000F04C87C1F01584302B01F01284312B53
:1052100000F0448762495E4E20461DF0F1F90021FE
:105220002046FCF701FA20461DF0AAF92220FCF7DF
:1052300079FB95ED0F0A0020FCF718FB5549204635
:105240001DF0DEF900212046FCF7EEF920461DF0A6
:1052500097F9544920461DF0D3F900212046FCF768
:10526000E3F920461DF08CF92220FCF75BFB95ED5D
:105270000E0A0020FCF7FAFA464920461DF0C0F954
:1052800000212046FCF7D0F920461DF079F92B6863
:10529000012B01F0E386C1F06B86022B7FF40EAC8C
:1052A000414920461DF0ACF900212046FCF7BCF92D
:1052B00020461DF065F92220FCF734FB3B492046CF
:1052C0001DF09EF900212046FCF7AEF920461DF0A6
:1052D00057F9304920461DF093F900212046FCF78C
:1052E000A3F920461DF04CF9314920461DF088F9FC
:1052F00000212046FCF798F920461DF041F92220B4
:10530000FCF710FBD6ED077A0020B8EEE70AFCF7B1
:10531000ADFA204920461DF073F900212046FCF724
:1053200083F920461DF02CF9224920461DF068F92A
:1053300000212046FCF778F920461DF021F92220B3
:10534000FCF7F0FAD6ED087A0020B8EE670AFCF711
:105350008DFA104920461DF053F900212046FCF734
:1053600063F920461DF00CF9134920461DF048F959
:1053700000212046FCF758F920461DF001F92220B3
:10538000FCF7D0FA96ED0C0AFFF788BB9894020060
:105390001418FF1FC48D0200AC940200C0940200D8
:1053A0003895020084950200D4940200CC9B020040
:1053B000E8940200FC940200109502008449854D97
:1053C00068461DF01DF900216846FCF72DF9684676
:1053D0001DF0D6F82220FCF7A5FAD5ED007A0020C2
:1053E000B8EEE70AFCF742FA7B4968461DF008F977
:1053F00000216846FCF718F968461DF0C1F87749A6
:1054000068461DF0FDF800216846FCF70DF9684676
:105410001DF0B6F82220FCF785FAD5ED087A0020B9
:10542000B8EE670AFCF722FA6B4968461DF0E8F807
:1054300000216846FCF7F8F868461DF0A1F86849B5
:1054400068461DF0DDF800216846FCF7EDF8684677
:105450001DF096F82220FCF765FAD5ED047A0020BD
:10546000B8EEE70AFCF702FA5B4968461DF0C8F897
:1054700000216846FCF7D8F868461DF081F85949C4
:1054800068461DF0BDF800216846FCF7CDF8684677
:105490001DF076F82220FCF745FAD5ED147A0020AD
:1054A000B8EE670AFCF7E2F94B4968461DF0A8F828
:1054B00068460021FCF7B8F868461DF061F8EE6C0C
:1054C0006C46002E01F03382012E00F09782AB6C07
:1054D000404D012B01F0D684C1F04584022B7FF4AE
:1054E000EDAA414920461DF08BF800212046FCF72B
:1054F0009BF820461DF044F82220FCF713FA3B49A4
:1055000020461DF07DF800212046FCF78DF820464E
:105510001DF036F8304920461DF072F80021204673
:10552000FCF782F820461DF02BF8314920461DF08B
:1055300067F800212046FCF777F820461DF020F898
:105540002220FCF7EFF9D5ED037A0020B8EEE70A48
:10555000FCF78CF9204920461DF052F80021204626
:10556000FCF762F820461DF00BF8224920461DF09A
:1055700047F800212046FCF757F820461DF000F8B8
:105580002220FCF7CFF9D5ED0B7A0020B8EE670AA0
:10559000FCF76CF9104920461DF032F80021204636
:1055A000FCF742F820461CF0EBFF134920461DF0A3
:1055B00027F800212046FCF737F820461CF0E0FFD2
:1055C0002220FCF7AFF995ED070AFFF767BA00BF95
:1055D000989402008014FF1FC48D0200AC94020056
:1055E000C094020098950200D4940200CC9B020063
:1055F000E8940200FC94020010950200B549B64DF3
:1056000068461CF0FDFF00216846FCF70DF868466F
:105610001CF0B6FF2220FCF785F9D5ED0C7A0020AE
:10562000B8EEE70AFCF722F9AC4968461CF0E8FF3F
:1056300000216846FBF7F8FF68461CF0A1FFA84967
:1056400068461CF0DDFF00216846FBF7EDFF684669
:105650001CF096FF2220FCF765F9D5ED147A0020A6
:10566000B8EE670AFCF702F99C4968461CF0C8FFCF
:1056700000216846FBF7D8FF68461CF081FF994976
:1056800068461CF0BDFF00216846FBF7CDFF684669
:105690001CF076FF2220FCF745F9D5ED107A0020AA
:1056A000B8EEE70AFCF7E2F88C4968461CF0A8FF60
:1056B00000216846FBF7B8FF68461CF061FF8A4985
:1056C00068461CF09DFF00216846FBF7ADFF684669
:1056D0001CF056FF2220FCF725F9D5ED047A0020B6
:1056E000B8EEE70AFCF7C2F87C4968461CF088FF70
:1056F00000216846FBF798FF68461CF041FF7B4994
:1057000068461CF07DFF00216846FBF78DFF684668
:105710001CF036FF2220FCF705F995ED030A002066
:10572000FCF7A4F86D4968461CF06AFF0021684642
:10573000FBF77AFF68461CF023FF6D4968461CF0B2
:105740005FFF00216846FBF76FFF68461CF018FFFB
:105750002220FCF7E7F895ED060A0020FCF786F812
:105760005E4968461CF04CFF68460021FBF75CFF71
:1057700068461CF005FF6E696C46002E01F0CA8178
:10578000012E23D15B4968461CF03AFF0021684690
:10579000FBF74AFF68461CF0F3FE2220FCF7C2F834
:1057A000554968461CF02CFF00216846FBF73CFF7A
:1057B00068461CF0E5FE494968461CF021FF684632
:1057C0000021FBF731FF68461CF0DAFEAB68023BB4
:1057D000052B3FF6E5A8DFE813F0440888087708B2
:1057E000660855089908454920461CF009FF002124
:1057F0002046FBF719FF20461CF0C2FE2220FCF7D2
:1058000091F83F4920461CF0FBFE00212046FBF7A3
:105810000BFF20461CF0B4FE304920461CF0F0FE81
:1058200000212046FBF700FF20461CF0A9FE354969
:1058300020461CF0E5FE00212046FBF7F5FE204641
:105840001CF09EFE2220FCF76DF8D5ED0D7A0020AD
:10585000B8EEE70AFCF70AF8204920461CF0D0FE13
:1058600000212046FBF7E0FE20461CF089FE264979
:1058700020461CF0C5FE00212046FBF7D5FE204641
:105880001CF07EFE2220FCF74DF8D5ED157A0020A5
:10589000B8EE670AFBF7EAFF104920461CF0B0FE9D
:1058A00000212046FBF7C0FE20461CF069FE174988
:1058B00020461CF0A5FE00212046FBF7B5FE204641
:1058C0001CF05EFE2220FCF72DF895ED110AFFF783
:1058D000E5B800BF989402000814FF1FC48D0200B1
:1058E000AC940200C0940200249502003895020096
:1058F00084950200B49502005C970200D4940200E3
:10590000049B0200E8940200FC940200109502003F
:10591000BE4920461CF074FE00212046FBF784FEA1
:1059200020461CF02DFE2220FBF7FCFFB849204644
:105930001CF066FE00212046FBF776FE20461CF098
:105940001FFEB44920461CF05BFE00212046FBF7F9
:105950006BFE20461CF014FEAF4920461CF050FEA2
:1059600000212046FBF760FE20461CF009FE2220A5
:10597000FBF7D8FFD5ED0E7A0020B8EEE70AFBF76B
:1059800075FFA44920461CF03BFE00212046FBF792
:105990004BFE20461CF0F4FDA04920461CF030FED2
:1059A00000212046FBF740FE20461CF0E9FD2220A6
:1059B000FBF7B8FFD5ED167A0020B8EE670AFBF7C3
:1059C00055FF944920461CF01BFE00212046FBF7A2
:1059D0002BFE20461CF0D4FD914920461CF010FE01
:1059E00000212046FBF720FE20461CF0C9FD2220A6
:1059F000FBF798FF95ED120AFFF750B88949684602
:105A00001CF0FEFD00216846FBF70EFE68461CF008
:105A1000B7FD2220FBF786FF834968461CF0F0FDA6
:105A200000216846FBF700FE68461CF0A9FD794995
:105A300068461CF0E5FD00216846FBF7F5FD684669
:105A40001CF09EFD794968461CF0DAFD002168468D
:105A5000FBF7EAFD68461CF093FD2220FBF762FF8E
:105A6000D5ED0C7A0020B8EEE70AFBF7FFFE694996
:105A700068461CF0C5FD00216846FBF7D5FD684669
:105A80001CF07EFD6A4968461CF0BAFD002168469C
:105A9000FBF7CAFD68461CF073FD2220FBF742FFAE
:105AA00095ED0F0A0020FBF7E1FE5A4968461CF00D
:105AB000A7FD00216846FBF7B7FD68461CF060FDB6
:105AC0005C4968461CF09CFD00216846FBF7ACFD74
:105AD00068461CF055FD2220FBF724FF95ED0E0AC9
:105AE0000020FBF7C3FE4B4968461CF089FD684661
:105AF0000021FBF799FD68461CF042FDE7E44349AD
:105B000068461CF07DFD00216846FBF78DFD684668
:105B10001CF036FD2220FBF705FF474968461CF0C4
:105B20006FFD00216846FBF77FFD68461CF028FDED
:105B3000384968461CF064FD00216846FBF774FD97
:105B400068461CF01DFD3D4968461CF059FD0021CA
:105B50006846FBF769FD68461CF012FD2220FBF742
:105B6000E1FED4ED017A0020B8EEE70AFBF77EFEF5
:105B7000284968461CF044FD00216846FBF754FDA7
:105B800068461CF0FDFC2E4968461CF039FD0021DA
:105B90006846FBF749FD68461CF0F2FC2220FBF743
:105BA000C1FED4ED097A0020B8EEE70AFBF75EFEED
:105BB000184968461CF024FD00216846FBF734FDB7
:105BC00068461CF0DDFC1F4968461CF019FD0021E9
:105BD0006846FBF729FD68461CF0D2FC2220FBF743
:105BE000A1FE94ED050AB8EEC00A0020FBF73EFEC8
:105BF000684608491CF004FD68460021FBF714FDC7
:105C000068461CF0BDFC04B070BD00BFD494020017
:105C100078C60200C48D0200E8940200FC940200E1
:105C200010950200249502005C970200389502004E
:105C300084950200B4950200989A0200989402009C
:105C4000AC940200C0940200E54968461CF0D8FC00
:105C500000216846FBF7E8FC68461CF091FC222016
:105C6000FBF760FEDF4968461CF0CAFC002168466D
:105C7000FBF7DAFC68461CF083FCDB4968461CF045
:105C8000BFFC00216846FBF7CFFC68461CF078FC9F
:105C9000D64968461CF0B4FC00216846FBF7C4FCFA
:105CA00068461CF06DFC2220FBF73CFED4ED047A24
:105CB0000020B8EEE70AFBF7D9FDCB4968461CF097
:105CC0009FFC00216846FBF7AFFC68461CF058FCBF
:105CD000C74968461CF094FC00216846FBF7A4FC09
:105CE00068461CF04DFC2220FBF71CFED4ED007A28
:105CF0000020B8EEE70AFBF7B9FDBB4968461CF087
:105D00007FFC00216846FBF78FFC68461CF038FCDE
:105D1000B84968461CF074FC00216846FBF784FC17
:105D200068461CF02DFC2220FBF7FCFD94ED080AD0
:105D300059E7AB4968461CF063FC00216846FBF755
:105D400073FC68461CF01CFC2220FBF7EBFDAA4903
:105D500068461CF055FC00216846FBF765FC684668
:105D60001CF00EFCA04968461CF04AFC0021684665
:105D7000FBF75AFC68461CF003FC9C4968461CF083
:105D80003FFC00216846FBF74FFC68461CF0F8FB1F
:105D90002220FBF7C7FDD4ED037A0020B8EEE70A16
:105DA000FBF764FD904968461CF02AFC0021684618
:105DB000FBF73AFC68461CF0E3FB8D4968461CF093
:105DC0001FFC00216846FBF72FFC68461CF0D8FB3F
:105DD0002220FBF7A7FDD4ED0B7A0020B8EEE70AEE
:105DE000FBF744FD804968461CF00AFC0021684628
:105DF000FBF71AFC68461CF0C3FB7E4968461CF0A2
:105E0000FFFB00216846FBF70FFC68461CF0B8FB5F
:105E10002220FBF787FD94ED070AE4E67049684607
:105E20001CF0EEFB00216846FBF7FEFB68461CF009
:105E3000A7FB2220FBF776FD704968461CF0E0FBCB
:105E400000216846FBF7F0FB68461CF099FB6649A9
:105E500068461CF0D5FB00216846FBF7E5FB684669
:105E60001CF08EFB614968461CF0CAFB00216846A5
:105E7000FBF7DAFB68461CF083FB2220FBF752FDA0
:105E8000D4ED027A0020B8EEE70AFBF7EFFC5649A2
:105E900068461CF0B5FB00216846FBF7C5FB684669
:105EA0001CF06EFB524968461CF0AAFB00216846B4
:105EB000FBF7BAFB68461CF063FB2220FBF732FDC0
:105EC000D4ED0A7A0020B8EEE70AFBF7CFFC46498A
:105ED00068461CF095FB00216846FBF7A5FB684669
:105EE0001CF04EFB434968461CF08AFB00216846C3
:105EF000FBF79AFB68461CF043FB2220FBF712FDE0
:105F000094ED060A6FE636493D4D68461CF078FB75
:105F100000216846FBF788FB68461CF031FB222015
:105F2000FBF700FD374920461CF06AFB00212046A4
:105F3000FBF77AFB20461CF023FB2B4920461CF084
:105F40005FFB00212046FBF76FFB20461CF018FB8F
:105F50002D4920461CF054FB00212046FBF764FB32
:105F600020461CF00DFB2220FBF7DCFCD5E90401E8
:105F70001EF05CFD00EE100A0020FBF777FC1A49CA
:105F800020461CF03DFB00212046FBF74DFB204640
:105F90001CF0F6FA6B68012B07D0C0F0E185302BBE
:105FA00000F0DE85312B7EF489AD184920461CF0C7
:105FB00027FB00212046FBF737FB20461CF0E0FAC8
:105FC0002220FBF7AFFC124920461CF019FB2046AB
:105FD0000021FBF729FB20461CF0D2FAFEF763BD37
:105FE000D4940200CC9B0200C48D0200E89402000D
:105FF000FC9402001095020078C60200049B020087
:106000000817FF1F6C9902002495020038950200C2
:1060100054950200CA49CB4D68461CF0F1FA0021A4
:106020006846FBF701FB68461CF0AAFA2220FBF742
:1060300079FCC54977E7C249C44D68461CF0E0FACF
:1060400000216846FBF7F0FA68461CF099FA222016
:10605000FBF768FCBE4966E7B949BE4D68461CF0CF
:10606000CFFA00216846FBF7DFFA68461CF088FA91
:106070002220FBF757FCB84955E7B149B74D6846B0
:106080001CF0BEFA00216846FBF7CEFA68461CF009
:1060900077FA2220FBF746FCB14944E7B149204694
:1060A0001CF0AEFA00212046FBF7BEFA20461CF099
:1060B00067FA2220FBF736FCAB4920461CF0A0FA19
:1060C00000212046FBF7B0FA20461CF059FAA749F8
:1060D00020461CF095FA20460021FBF7A5FA204641
:1060E0001CF04EFAFFF796B8954968461CF088FAFE
:1060F00000216846FBF798FA68461CF041FA222016
:10610000FBF710FC9A4968461CF07AFA00216846B1
:10611000FBF78AFA68461CF033FA944968461CF08B
:106120006FFA00216846FBF77FFA68461CF028FAF0
:10613000904968461CF064FA00216846FBF774FA3F
:1061400068461CF01DFA2220FBF7ECFBD4ED077A21
:106150000020B8EEE70AFBF789FB844968461CF08B
:106160004FFA00216846FBF75FFA68461CF008FA10
:10617000814968461CF044FA00216846FBF754FA4E
:1061800068461CF0FDF92220FBF7CCFBD4ED087A21
:106190000020B8EE670AFBF769FB744968461CF0FB
:1061A0002FFA00216846FBF73FFA68461CF0E8F931
:1061B000724968461CF024FA00216846FBF734FA5D
:1061C00068461CF0DDF92220FBF7ACFBD4ED097A20
:1061D0000020B8EEE70AFBF749FB644968461CF06B
:1061E0000FFA00216846FBF71FFA68461CF0C8F951
:1061F0005C4968461CF004FA00216846FBF714FA73
:1062000068461CF0BDF92220FBF78CFB002094EDC2
:106210000F0AEBE44A4968461CF0F2F9002168468F
:10622000FBF702FA68461CF0ABF92220FBF77AFB79
:10623000534968461CF0E4F900216846FBF7F4F97D
:1062400068461CF09DF9494968461CF0D9F90021BF
:106250006846FBF7E9F968461CF092F9454968463B
:106260001CF0CEF900216846FBF7DEF968461CF009
:1062700087F92220FBF756FBD4ED017A0020B8EE17
:10628000E70AFBF7F3FA394968461CF0B9F900212F
:106290006846FBF7C9F968461CF072F9364968464A
:1062A0001CF0AEF900216846FBF7BEF968461CF009
:1062B00067F92220FBF736FBD4ED027A0020B8EE16
:1062C000670AFBF7D3FA294968461CF099F90021BF
:1062D0006846FBF7A9F968461CF052F92749684659
:1062E0001CF08EF900216846FBF79EF968461CF009
:1062F00047F92220FBF716FBD4ED037A0020B8EE15
:10630000E70AFBF7B3FA194968461CF079F900214E
:106310006846FBF789F968461CF032F9114968466E
:106320001CF06EF900216846FBF77EF968461CF008
:1063300027F92220FBF7F6FA002094ED0A0A55E42B
:10634000D49402005017FF1F449A02003817FF1F11
:106350007C9402002017FF1FE4990200F016FF1F33
:10636000E0BC0200249502007C950200C48D02006E
:1063700070950200E8940200FC940200109502005F
:106380005C950200E24968461CF03AF90021684633
:10639000FBF74AF968461CF0F3F82220FBF7C2FA33
:1063A000DC4968461CF02CF900216846FBF73CF9F3
:1063B00068461CF0E5F8D84968461CF021F9002130
:1063C0006846FBF731F968461CF0DAF8D3496846AD
:1063D0001CF016F900216846FBF726F968461CF008
:1063E000CFF82220FBF79EFAD4ED047A0020B8EE15
:1063F000E70AFBF73BFAC84968461CF001F900219F
:106400006846FBF711F968461CF0BAF8C4496846BB
:106410001CF0F6F800216846FBF706F968461CF008
:10642000AFF82220FBF77EFAD4ED057A0020B8EE13
:10643000670AFBF71BFAB84968461CF0E1F800212F
:106440006846FBF7F1F868461CF09AF8B5496846CB
:106450001CF0D6F800216846FBF7E6F868461CF009
:106460008FF82220FBF75EFAD4ED067A0020B8EE12
:10647000E70AFBF7FBF9A84968461CF0C1F80021C0
:106480006846FBF7D1F868461CF07AF8A6496846DA
:106490001CF0B6F800216846FBF7C6F868461CF009
:1064A0006FF82220FBF73EFA002094ED0E0AFFF76A
:1064B0009DBB974968461CF0A3F800216846FBF78E
:1064C000B3F868461CF05CF82220FBF72BFA9749DA
:1064D00068461CF095F800216846FBF7A5F8684669
:1064E0001CF04EF88C4968461CF08AF8002168467A
:1064F000FBF79AF868461CF043F8884968461CF098
:106500007FF800216846FBF78FF868461CF038F8E2
:106510002220FBF707FAD4ED017A0020B8EEE70A53
:10652000FBF7A4F97C4968461CF06AF8002168462C
:10653000FBF77AF868461CF023F8794968461CF0A6
:106540005FF800216846FBF76FF868461CF018F802
:106550002220FBF7E7F9D4ED027A0020B8EE670AB3
:10656000FBF784F96C4968461CF04AF8002168463C
:10657000FBF75AF868461CF003F86A4968461CF0B5
:106580003FF800216846FBF74FF868461BF0F8FF1C
:106590002220FBF7C7F9D4ED037A0020B8EEE70A12
:1065A000FBF764F95C4968461CF02AF8002168464C
:1065B000FBF73AF868461BF0E3FF5B4968461CF0BE
:1065C0001FF800216846FBF72FF868461BF0D8FF3C
:1065D0002220FBF7A7F9002094ED0D0AFFF706BB78
:1065E0004B4968461CF00CF800216846FBF71CF884
:1065F00068461BF0C5FF2220FBF794F94C4968461A
:106600001BF0FEFF00216846FBF70EF868461BF002
:10661000B7FF414968461BF0F3FF00216846FBF7CE
:1066200003F868461BF0ACFF3C4968461BF0E8FFE6
:1066300000216846FAF7F8FF68461BF0A1FF222008
:10664000FBF770F9D4ED077A0020B8EEE70AFBF704
:106650000DF9314968461BF0D3FF00216846FAF76F
:10666000E3FF68461BF08CFF2D4968461BF0C8FF0E
:1066700000216846FAF7D8FF68461BF081FF222008
:10668000FBF750F9D4ED087A0020B8EE670AFBF763
:10669000EDF8214968461BF0B3FF00216846FAF780
:1066A000C3FF68461BF06CFF1E4968461BF0A8FF3D
:1066B00000216846FAF7B8FF68461BF061FF222008
:1066C000FBF730F9D4ED097A0020B8EEE70AFBF7C2
:1066D000CDF8114968461BF093FF00216846FAF790
:1066E000A3FF68461BF04CFF0F4968461BF088FF6C
:1066F00000216846FAF798FF68461BF041FF222008
:10670000FBF710F9002094ED0C0AFFF76FBA00BFF9
:10671000D494020068950200C48D0200E89402003F
:10672000FC9402001095020024950200609502007E
:106730006C950200E34968461BF062FF0021684641
:10674000FAF772FF68461BF01BFF2220FBF7EAF8FE
:10675000DD4968461BF054FF00216846FAF764FFE4
:1067600068461BF00DFFD94968461BF049FF002120
:106770006846FAF759FF68461BF002FFD44968469D
:106780001BF03EFF00216846FAF74EFF68461BF0FB
:10679000F7FE2220FBF7C6F8D4ED047A0020B8EE0D
:1067A000E70AFBF763F8C94968461BF029FF002197
:1067B0006846FAF739FF68461BF0E2FEC5496846AD
:1067C0001BF01EFF00216846FAF72EFF68461BF0FB
:1067D000D7FE2220FBF7A6F8D4ED057A0020B8EE0C
:1067E000670AFBF743F8B94968461BF009FF002127
:1067F0006846FAF719FF68461BF0C2FEB6496846BC
:106800001BF0FEFE00216846FAF70EFF68461BF0FB
:10681000B7FE2220FBF786F8D4ED067A0020B8EE0A
:10682000E70AFBF723F8A94968461BF0E9FE0021B7
:106830006846FAF7F9FE68461BF0A2FEA7496846CB
:106840001BF0DEFE00216846FAF7EEFE68461BF0FC
:1068500097FE2220FBF766F8002094ED0B0AFFF765
:10686000C5B99F4920461BF0CBFE00212046FAF710
:10687000DBFE20461BF084FE2220FBF753F89949EB
:10688000FEF779B8964920461BF0BAFE0021204653
:10689000FAF7CAFE20461BF073FE2220FBF742F8EF
:1068A0009149FEF768B88E4920461BF0A9FE0021E9
:1068B0002046FAF7B9FE20461BF062FE2220FBF7C5
:1068C00031F88A49FEF757B8854920461BF098FEF3
:1068D00000212046FAF7A8FE20461BF051FE222098
:1068E000FBF720F88249FEF746B87D4920461BF0A9
:1068F00087FE00212046FAF797FE20461BF040FE57
:106900002220FBF70FF87B49FEF735B87449204683
:106910001BF076FE00212046FAF786FE20461BF08B
:106920002FFE2220FAF7FEFF7349FEF724B86B49C9
:1069300068461BF065FE31466846FAF775FE684604
:106940001BF01EFE2220FAF7EDFF6C4968461BF093
:1069500057FE31466846FAF767FE68461BF010FEA0
:106960005A4968461BF04CFE31466846FAF75CFE11
:1069700068461BF005FE624968461BF041FE314641
:106980006846FAF751FE68461BF0FAFD2220FAF736
:10699000C9FFD5ED0D7A3046B8EEE70AFAF766FF83
:1069A0004A4968461BF02CFE31466846FAF73CFE21
:1069B00068461BF0E5FD534968461BF021FE314651
:1069C0006846FAF731FE68461BF0DAFD2220FAF736
:1069D000A9FF95ED110A3046FAF748FF3B49684692
:1069E0001BF00EFE31466846FAF71EFE68461BF0A5
:1069F000C7FD454968461BF003FE31466846FAF775
:106A000013FE68461BF0BCFD2220FAF78BFF95EDC4
:106A1000100A3046FAF72AFF2C4968461BF0F0FDB1
:106A200068463146FAF700FE68461BF0A9FDFEF7FE
:106A30004EBD2A4920461BF0E3FD00212046FAF70F
:106A4000F3FD20461BF09CFD2220FAF76BFF2F4937
:106A5000FFF733BB224920461BF0D2FD0021204620
:106A6000FAF7E2FD20461BF08BFD2220FAF75AFFD1
:106A70002749FDF780BF244968461BF0C1FD314618
:106A80006846FAF7D1FD68461BF07AFD2220FAF736
:106A900049FF1A4968461BF0B3FD31466846FAF7CC
:106AA000C3FD68461BF06CFD084968461BF0A8FD55
:106AB00068463146FAF7B8FD68461BF061FDFDF700
:106AC00045BF00BFD494020064950200C48D02004B
:106AD000E8940200FC940200109502002495020044
:106AE00098950200C8950200D8950200D49502003E
:106AF000D0950200CC950200DC950200AC95020016
:106B00003895020084950200B49502007495020045
:106B1000E0950200CF4968461BF072FD3146684699
:106B2000FAF782FD68461BF02BFD2220FAF7FAFEE9
:106B3000C94968461BF064FD31466846FAF774FDA2
:106B400068461BF01DFDC54968461BF059FD6846A7
:106B50003146FAF769FD68461BF012FDFEF736BEB6
:106B6000BF4920461BF04CFD00212046FAF75CFD92
:106B700020461BF005FD2220FAF7D4FEB949FFF7A5
:106B800023BAB94968461BF03BFD00216846FAF775
:106B90004BFD68461BF0F4FC2220FAF7C3FEB34914
:106BA00068461BF02DFD00216846FAF73DFD68465A
:106BB0001BF0E6FCA94968461BF022FD002168464F
:106BC000FAF732FD68461BF0DBFCA94968461BF06A
:106BD00017FD00216846FAF727FD68461BF0D0FC38
:106BE0002220FAF79FFED4ED037A0020B8EEE70AE0
:106BF000FAF73CFE994968461BF002FD0021684601
:106C0000FAF712FD68461BF0BBFC9A4968461BF078
:106C1000F7FC00216846FAF707FD68461BF0B0FC58
:106C20002220FAF77FFED4ED0B7A0020B8EEE70AB7
:106C3000FAF71CFE894968461BF0E2FC0021684611
:106C4000FAF7F2FC68461BF09BFC8B4968461BF088
:106C5000D7FC00216846FAF7E7FC68461BF090FC79
:106C60002220FAF75FFE94ED070A0020B8EEC00A72
:106C7000FEF7A7B87C4968461BF0C2FC00216846B5
:106C8000FAF7D2FC68461BF07BFC2220FAF74AFE9A
:106C90007A4968461BF0B4FC00216846FAF7C4FC48
:106CA00068461BF06DFC6D4968461BF0A9FC00218D
:106CB0006846FAF7B9FC68461BF062FC6C49684606
:106CC0001BF09EFC00216846FAF7AEFC68461BF0FC
:106CD00057FC2220FAF726FED4ED047A0020B8EE05
:106CE000E70AFAF7C3FD5D4968461BF089FC0021FD
:106CF0006846FAF799FC68461BF042FC5D49684615
:106D00001BF07EFC00216846FAF78EFC68461BF0FB
:106D100037FC2220FAF706FED4ED007A0020B8EE08
:106D2000E70AFAF7A3FD4D4968461BF069FC00210C
:106D30006846FAF779FC68461BF022FC4E49684623
:106D40001BF05EFC00216846FAF76EFC68461BF0FB
:106D500017FC2220FAF7E6FD94ED080A0020B8EEB1
:106D6000C00AFEF72EB8404920461BF049FC00211E
:106D70002046FAF759FC20461BF002FC2220FAF7C5
:106D8000D1FD3F4920461BF03BFC00212046FAF78D
:106D90004BFC20461BF0F4FB304920461BF030FC36
:106DA00000212046FAF740FC20461BF0E9FB304961
:106DB00020461BF025FC00212046FAF735FC204632
:106DC0001BF0DEFB2220FAF7ADFDD5ED017A0020A5
:106DD000B8EEE70AFAF74AFD204920461BF010FCFE
:106DE00000212046FAF720FC20461BF0C9FB214970
:106DF00020461BF005FC00212046FAF715FC204632
:106E00001BF0BEFB2220FAF78DFDD5ED097A00209C
:106E1000B8EE670AFAF72AFD104920461BF0F0FB8E
:106E200000212046FAF700FC20461BF0A9FB12497E
:106E300020461BF0E5FB00212046FAF7F5FB204633
:106E40001BF09EFB2220FAF76DFD95ED050AFDF77C
:106E500025BE00BFB4950200AC950200C48D0200AF
:106E6000389502004C950200D494020078C60200C6
:106E7000E8940200FC94020010950200CC9B0200F2
:106E8000049B0200B04920461BF0BAFB00212046BB
:106E9000FAF7CAFB20461BF073FB2220FAF742FDEB
:106EA000AA4920461BF0ACFB00212046FAF7BCFBA8
:106EB00020461BF065FBA64920461BF0A1FB0021E4
:106EC0002046FAF7B1FB20461BF05AFBA1492046A9
:106ED0001BF096FB00212046FAF7A6FB20461BF08C
:106EE0004FFB2220FAF71EFDD5ED027A0020B8EE06
:106EF000E70AFAF7BBFC964920461BF081FB00210C
:106F00002046FAF791FB20461BF03AFB92492046B7
:106F10001BF076FB00212046FAF786FB20461BF08B
:106F20002FFB2220FAF7FEFCD5ED0A7A0020B8EEFE
:106F3000670AFAF79BFC864920461BF061FB00219B
:106F40002046FAF771FB20461BF01AFB83492046C6
:106F50001BF056FB00212046FAF766FB20461BF08B
:106F60000FFB2220FAF7DEFC95ED060AFDF796BD31
:106F7000754920461BF044FB00212046FAF754FBDC
:106F800020461BF0FDFA2220FAF7CCFC744920467B
:106F90001BF036FB00212046FAF746FB20461BF08B
:106FA000EFFA6B4920461BF02BFB00212046FAF735
:106FB0003BFB20461BF0E4FA664920461BF020FB11
:106FC00000212046FAF730FB20461BF0D9FA222098
:106FD000FAF7A8FCD6ED037A0020B8EEE70AFAF734
:106FE00045FC5B4920461BF00BFB00212046FAF7CD
:106FF0001BFB20461BF0C4FA574920461BF000FB40
:1070000000212046FAF710FB20461BF0B9FA222097
:10701000FAF788FCD6ED047A0020B8EE670AFAF792
:1070200025FC4B4920461BF0EBFA00212046FAF7DD
:10703000FBFA20461BF0A4FA484920461BF0E0FA70
:1070400000212046FAF7F0FA20461BF099FA222098
:10705000FAF768FC96ED0A0AFDF720BD3A4920468A
:107060001BF0CEFA00212046FAF7DEFA20461BF08C
:1070700087FA2220FAF756FC344920461BF0C0FA62
:1070800000212046FAF7D0FA20461BF079FA304961
:1070900020461BF0B5FA00212046FAF7C5FA204633
:1070A0001BF06EFA2B4920461BF0AAFA002120465D
:1070B000FAF7BAFA20461BF063FA2220FAF732FCFC
:1070C000D6ED057A0020B8EEE70AFAF7CFFB2049A3
:1070D00020461BF095FA00212046FAF7A5FA204633
:1070E0001BF04EFA1C4920461BF08AFA002120466C
:1070F000FAF79AFA20461BF043FA2220FAF712FC1C
:10710000D6ED067A0020B8EE670AFAF7AFFB104911
:1071100020461BF075FA00212046FAF785FA204632
:107120001BF02EFA0D4920461BF06AFA002120467A
:10713000FAF77AFA20461BF023FA2220FAF7F2FB3C
:1071400096ED0B0AFDF7AABCD494020078C60200A3
:10715000C48D0200E8940200FC9402001095020025
:10716000049B0200964968461BF04AFA00216846D3
:10717000FAF75AFA68461BF003FA2220FAF7D2FB14
:10718000904968461BF03CFA00216846FAF74CFA31
:1071900068461BF0F5F98C4968461BF031FA00216E
:1071A0006846FAF741FA68461BF0EAF987496846EB
:1071B0001BF026FA00216846FAF736FA68461BF0FB
:1071C000DFF92220FAF7AEFBD4ED017A0020B8EE09
:1071D000E70AFAF74BFB7C4968461BF011FA0021DD
:1071E0006846FAF721FA68461BF0CAF978496846FA
:1071F0001BF006FA00216846FAF716FA68461BF0FB
:10720000BFF92220FAF78EFBD4ED057A0020B8EE04
:10721000670AFAF72BFB6C4968461BF0F1F900216D
:107220006846FAF701FA68461BF0AAF96949684608
:107230001BF0E6F900216846FAF7F6F968461BF0FC
:107240009FF92220FAF76EFBD4ED097A0020B8EE00
:10725000E70AFAF70BFB5C4968461BF0D1F90021FD
:107260006846FAF7E1F968461BF08AF95A49684618
:107270001BF0C6F900216846FAF7D6F968461BF0FC
:107280007FF92220FAF74EFB002094ED130AFDF758
:1072900098BD4B4968461BF0B3F900216846FAF7E0
:1072A000C3F968461BF06CF92220FAF73BFB4B4907
:1072B00068461BF0A5F900216846FAF7B5F968465B
:1072C0001BF05EF9404968461BF09AF900216846B8
:1072D000FAF7AAF968461BF053F93C4968461BF0D7
:1072E0008FF900216846FAF79FF968461BF048F9C4
:1072F0002220FAF717FBD4ED027A0020B8EE670AD5
:10730000FAF7B4FA304968461BF07AF9002168466A
:10731000FAF78AF968461BF033F92D4968461BF0E5
:107320006FF900216846FAF77FF968461BF028F9E3
:107330002220FAF7F7FAD4ED067A0020B8EE670AB1
:10734000FAF794FA204968461BF05AF9002168467A
:10735000FAF76AF968461BF013F91E4968461BF0F4
:107360004FF900216846FAF75FF968461BF008F903
:107370002220FAF7D7FAD4ED0A7A0020B8EEE70A0D
:10738000FAF774FA104968461BF03AF9002168468A
:10739000FAF74AF968461BF0F3F80F4968461BF004
:1073A0002FF900216846FAF73FF968461BF0E8F824
:1073B0002220FAF7B7FA002094ED140AFDF701BD78
:1073C000D4940200049B0200C48D0200E8940200E1
:1073D000FC94020010950200B495020078C60200E9
:1073E0002DE9F043C44DC54CD5F800E02468BEF14A
:1073F000010F2DED028B1F4604BFC14B1C68ADB0C1
:1074000006460D46904608A800230122214617F0A3
:10741000C5FA0FA815F050F8002840F0918118A87F
:107420009DF83A30B74908AA15F0FAF81A9A9DF86B
:107430006C309DF8641011928DF848308DF8401032
:107440001BAA0DF149030DF1560012F8011F03F8B4
:10745000011B8342F9D11F9B169318A814F0FEFF5D
:107460000FA815F029F88146002836D101230921FB
:10747000A5488DF83B301AF065FA20461EF0A0FEB4
:10748000014620461AF05EFA0F21A0489FEDA08A1F
:107490001AF058FA9F481AF0E5FE9F4918A81BF009
:1074A000AFF8494618A8FAF7BFF818A81BF068F813
:1074B0009A4918A81BF0A4F818A84946FAF7B4F896
:1074C00018A81BF05DF808A817F086FAB0EE480A75
:1074D0002DB0BDEC028BBDE8F0830024502218A92A
:1074E00008A88DF83B4017F0D5FA002800F0F1808D
:1074F000502300932A4618AB314608A817F03AFCEF
:10750000002800F0218118A81EF05AFE014618A894
:107510001AF018FA7F481AF0A5FE814904A81BF05A
:107520006FF804A82146FAF77FF804A81BF028F8A2
:10753000002F00F03D812220FAF7F4F918A904A8E1
:107540001BF05EF8214604A8FAF76EF804A81BF0B9
:1075500017F82220FAF7E6F9724904A81BF050F850
:10756000002104A8FAF760F804A81BF009F807EE58
:10757000908A0020B8EEE70AFAF778F9674904A87C
:107580001BF03EF8002104A8FAF74EF804A81AF000
:10759000F7FF30461EF014FE014630461AF0D2F9CD
:1075A0005C481AF05FFE28461EF00AFE0146284697
:1075B0001AF0C8F957481AF055FE052158481AF034
:1075C000C1F9002F00F0008122201AF03FFA18A81C
:1075D0001EF0F6FD014618A81AF0B4F922201AF0A0
:1075E00035FA01214F481AF0ADF9414649481AF0E1
:1075F00089FE48481AF036FE4B4904A81BF000F8F3
:10760000002104A8FAF710F804A81AF0B9FF222004
:10761000FAF788F9314604A81AF0F2FF002104A80D
:10762000FAF702F804A81AF0ABFF404904A81AF0D0
:10763000E7FF002104A8F9F7F7FF04A81AF0A0FF5C
:107640003B4904A81AF0DCFF002104A8F9F7ECFF7D
:1076500004A81AF095FF2220FAF764F9294604A835
:107660001AF0CEFF002104A8F9F7DEFF04A81AF0F3
:1076700087FF2E4904A81AF0C3FF002104A8F9F7D8
:10768000D3FF04A81AF07CFF2A4904A81AF0B8FF17
:10769000002104A8F9F7C8FF04A81AF071FF2220FE
:1076A000FAF740F918A904A81AF0AAFF002104A8C3
:1076B000F9F7BAFF04A81AF063FF1C4904A81AF0EE
:1076C0009FFF04A80021F9F7AFFF04A81AF058FFA4
:1076D0005AE0092118489FED0E8A1AF033F908A8DC
:1076E0001EF06EFD014608A81AF02CF90C21134873
:1076F0001AF028F9E7E600BFB017FF1F6407FF1F65
:107700007407FF1F6019FF1FF49502000096020026
:10771000000000002408FF1F10960200B08B02003A
:10772000389602004096020044960200C48D020082
:10773000589602006C9602001C96020028960200E1
:107740000FA814F0ABFE6AE6102123481AF0FAF8ED
:1077500022481AF087FD042121481AF0F3F8304638
:107760001EF02EFD014630461AF0ECF803211D48AC
:107770001AF0E8F828461EF023FD014628461AF0C4
:10778000E1F816481AF06EFD174A1368049304993D
:1077900013680393039B5B1A632BF9D918A81DF098
:1077A0006DFC51EC100B1DF041F908EE100A8AE651
:1077B00018A904A81AF024FF04A83946F9F734FFE1
:1077C00004A81AF0DDFEC7E618A81EF0F9FC014671
:1077D00018A81AF0B7F804E7888B02002408FF1FE6
:1077E0008096020088960200141CFF1F38B5684D71
:1077F0006849694C284600234FF43C72FFF7F0FDBE
:10780000BDEEC00A284600234FF44972634984ED57
:10781000000AFFF7E5FDBDEEC00A284600234FF43D
:107820004A725F4984ED0C0AFFF7DAFDBDEEC00A2B
:10783000284600233C225B4984ED140AFFF7D0FD63
:10784000BDEEC00A284600234FF45872564984ED15
:10785000100AFFF7C5FDBDEEC00A284600234FF40D
:107860005772524984ED0D0AFFF7BAFDBDEEC00A0A
:107870002846002340224E4984ED150AFFF7B0FD4B
:10788000BDEEC00A284600234FF45572494984EDE5
:10789000110AFFF7A5FDBDEEC00A284600234FF4EC
:1078A0005672454984ED0E0AFFF79AFDBDEEC00AF7
:1078B000284600234422414984ED160AFFF790FD33
:1078C000BDEEC00A284600234FF44C723C4984EDBB
:1078D000120AFFF785FDBDEEC00A284600234FF4CB
:1078E0004B72384984ED0F0AFFF77AFDBDEEC00AEE
:1078F000284600231C22344984ED170AFFF770FD47
:10790000BDEEC00A284600234FF4D8722F4984EDFB
:10791000130AFFF765FDBDEEC00A284600234FF4A9
:10792000FE722B4984ED050AFFF75AFDBDEEC00A31
:10793000284601234FF4BA72264984ED020AFFF764
:107940004FFDBDEEC00A2846B8EEC00A00234FF432
:10795000F872214984ED030AFFF742FDBDEEC00A2B
:10796000284601234FF41B721C4984ED040AFFF7DB
:1079700037FDBDEEC00A1A4BB8EEC00A20461968A2
:1079800084ED060A6022BDE8384017F041BB00BF15
:10799000949602008C9602000814FF1FA096020025
:1079A000B4960200C4960200DC960200E89602003B
:1079B000F096020004970200109702001897020048
:1079C0002C9702003897020040970200549702005B
:1079D000649702007097020080970200909702005F
:1079E0004C07FF1F38B5224D2249234C284600235F
:1079F0009C22FFF7F5FCBDEEC00A284601234FF498
:107A000096721E4984ED090AFFF7EAFCBDEEC00A32
:107A10002846B8EEC00A00234FF4DA72184984ED04
:107A20000B0AFFF7DDFCBDEEC00A284601234FF428
:107A30001F72144984ED0A0AFFF7D2FCBDEEC00A9A
:107A40002846B8EEC00A00234FF43D720E4984ED7B
:107A5000080AFFF7C5FC0D4BBDEEC00A20461968A9
:107A600084ED070A6022BDE8384017F0D1BA00BFA4
:107A7000B4970200A09702000814FF1F909702001D
:107A80005497020070970200809702004C07FF1F76
:107A900038B54A4D4A494B4C284600234FF4EC7206
:107AA000FFF79EFCBDEEC00A284600234FF461722A
:107AB000454984ED0C0AFFF793FCBDEEC00A284649
:107AC00000234FF46B72414984ED010AFFF788FCF3
:107AD000BDEEC00A2846002314223D4984ED090A60
:107AE000FFF77EFCBDEEC00A284600234FF4537218
:107AF000384984ED050AFFF773FCBDEEC00A28463D
:107B000000234FF45472344984ED020AFFF768FCF5
:107B1000BDEEC00A284600233822304984ED0A0A07
:107B2000FFF75EFCBDEEC00A284600234FF47672D4
:107B30002B4984ED060AFFF753FCBDEEC00A284628
:107B400000234FF45172274984ED030AFFF748FCE4
:107B5000BDEEC00A284600235422234984ED0B0AB7
:107B6000FFF73EFCBDEEC00A284600234FF45272D8
:107B70001E4984ED070AFFF733FCBDEEC00A284614
:107B800000234FF446721A4984ED040AFFF728FCDB
:107B9000BDEEC00A284600236C22164984ED000A77
:107BA000FFF71EFC144BBDEEC00A2046196884ED99
:107BB000080A3422BDE8384017F02ABABC97020000
:107BC0008C960200C013FF1FA0960200B49602001C
:107BD000C4960200DC960200E8960200F0960200CD
:107BE0000497020010970200189702002C970200D9
:107BF00038970200409702008407FF1F38B54A4DAE
:107C00004A494B4C284600234FF40E72FFF7E8FB1D
:107C1000BDEEC00A284600234FF45A72454984ED50
:107C20000C0AFFF7DDFBBDEEC00A284600234FF427
:107C30006472414984ED010AFFF7D2FB0023BDEED7
:107C4000C00A28461A463D4984ED090AFFF7C8FBD9
:107C5000BDEEC00A284600234FF46E72384984ED09
:107C6000050AFFF7BDFBBDEEC00A284600234FF40E
:107C70007372344984ED020AFFF7B2FBBDEEC00A0D
:107C8000284600231022304984ED0A0AFFF7A8FB9A
:107C9000BDEEC00A284600234FF478722B4984EDCC
:107CA000060AFFF79DFBBDEEC00A284600234FF4ED
:107CB0007B72274984ED030AFFF792FBBDEEC00AF1
:107CC000284600230822234984ED0B0AFFF788FB8E
:107CD000BDEEC00A284600234FF47E721E4984ED93
:107CE000070AFFF77DFBBDEEC00A284600234FF4CC
:107CF0007F721A4984ED040AFFF772FBBDEEC00AD9
:107D0000284600230C22164984ED000AFFF768FB81
:107D1000144BBDEEC00A2046196884ED080A3422CF
:107D2000BDE8384017F074B9C09702008C96020085
:107D30002819FF1FA0960200B4960200C496020004
:107D4000DC960200E8960200F0960200049702001A
:107D500010970200189702002C9702003897020033
:107D6000409702009007FF1F38B5594D59495A4CAA
:107D7000284600234FF41872FFF732FBBDEEC00A0D
:107D8000284600234FF4D272544984ED000AFFF7CD
:107D900027FBBDEEC00A284601234FF41972504953
:107DA00084ED0D0AFFF71CFB284601234FF41D72DA
:107DB0004C4984ED0F0AFFF713FB284600234FF4CC
:107DC0005D72494984ED0E0AFFF70AFBBDEEC00A59
:107DD000284600234FF46772444984ED010AFFF7F7
:107DE000FFFABDEEC00A284600234C22404984ED2C
:107DF000020AFFF7F5FABDEEC00A284600234FF449
:107E00006F723C4984ED090AFFF7EAFABDEEC00A39
:107E1000284600234FF47472374984ED030AFFF7B4
:107E2000DFFABDEEC00A284600234822334984ED1C
:107E3000040AFFF7D5FABDEEC00A284600234FF426
:107E400079722F4984ED0A0AFFF7CAFABDEEC00A1B
:107E5000284600234FF47C722A4984ED050AFFF777
:107E6000BFFABDEEC00A284600231822264984ED39
:107E7000060AFFF7B5FABDEEC00A284600234FF404
:107E80006872224984ED0B0AFFF7AAFABDEEC00A18
:107E9000284600234FF463721D4984ED070AFFF75B
:107EA0009FFABDEEC00A284600235022194984EDEE
:107EB000080AFFF795FA184BBDEEC00A204619686C
:107EC00084ED0C0A4022BDE8384017F0A1B800BF8D
:107ED000C89702008C9602001418FF1FD09702006A
:107EE000DC970200E8970200A0960200B496020018
:107EF000C4960200DC960200E8960200F0960200AA
:107F00000497020010970200189702002C970200B5
:107F100038970200409702003C07FF1F38B5724DAA
:107F20007249734C284600234FF4E872FFF758FA61
:107F3000BDEEC00A284600234FF40D726D4984ED52
:107F4000120AFFF74DFABDEEC00A284600234FF48F
:107F50000C72694984ED140AFFF742FABDEEC00ABB
:107F6000284600234FF46072644984ED130AFFF73A
:107F700037FABDEEC00A284600234FF46A72604902
:107F800084ED000AFFF72CFABDEEC00A2846002354
:107F900004225C4984ED080AFFF722FABDEEC00A0C
:107FA000284600234FF47172574984ED040AFFF705
:107FB00017FABDEEC00A284600234FF469725349F0
:107FC00084ED010AFFF70CFABDEEC00A2846002333
:107FD00058224F4984ED090AFFF702FABDEEC00AA4
:107FE000284600234FF470724A4984ED050AFFF7D2
:107FF000F7F9BDEEC00A284600234FF475724649D2
:1080000084ED020AFFF7ECF9BDEEC00A2846002312
:108010006022424984ED0A0AFFF7E2F9BDEEC00A88
:10802000284600234FF447723D4984ED060AFFF7C6
:10803000D7F9BDEEC00A284600234FF448723949EB
:1080400084ED030AFFF7CCF9BDEEC00A28460023F1
:108050003022354984ED0B0AFFF7C2F9BDEEC00AA4
:10806000284600234FF40B72304984ED070AFFF7CE
:10807000B7F9BDEEC00A284601234FF49A722C4985
:1080800084ED0D0AFFF7ACF928460123E8222949BF
:1080900084ED110AFFF7A4F9284600234FF4397242
:1080A000254984ED100AFFF79BF9BDEEC00A28466A
:1080B00001234FF43A72214984ED0C0AFFF790F93D
:1080C000284601234FF4A2721D4984ED0F0AFFF7E1
:1080D00087F91C4B84ED0E0A204619685422BDE82E
:1080E000384016F095BF00BFF49702008C9602004E
:1080F0008014FF1FFC97020054970200A096020014
:10810000B4960200C4960200DC960200E8960200D3
:10811000F0960200049702001097020018970200E0
:108120002C97020038970200409702000498020042
:10813000149802002C980200449802005098020003
:10814000689802003807FF1F38B5844D8449854C74
:1081500028460023A422FFF743F9BDEEC00A2846B3
:108160000023D022804984ED0E0AFFF739F9BDEED5
:10817000C00A28460023F0227C4984ED0C0AFFF750
:108180002FF9BDEEC00A284600234FF4E272784969
:1081900084ED0F0AFFF724F9BDEEC00A284601233B
:1081A0004FF42E72734984ED0D0AFFF719F9284632
:1081B00000234FF44F72704984ED160AFFF710F94F
:1081C000BDEEC00A284600234FF450726B4984ED7F
:1081D000000AFFF705F9BDEEC00A28460123642214
:1081E000674984ED040AFFF7FBF8BDEEC00A284694
:1081F00000234FF45C72634984ED080AFFF7F0F83E
:10820000BDEEC00A284600234FF46D725E4984ED2E
:10821000010AFFF7E5F8BDEEC00A28460023342224
:108220005A4984ED050AFFF7DBF8BDEEC00A28467F
:1082300001234FF48A72564984ED090AFFF7D0F8FA
:10824000BDEEC00A2846B8EEC00A01234FF4927270
:10825000504984ED130AFFF7C3F8BDEEC00A284663
:10826000B8EEC00A00234FF45B724B4984ED100A4C
:10827000FFF7B6F8BDEEC00A284600234FF4597246
:10828000464984ED020AFFF7ABF8BDEEC00A284666
:1082900000232C22424984ED060AFFF7A1F8BDEE27
:1082A000C00A284601234FF48E723E4984ED0A0A23
:1082B000FFF796F8BDEEC00A2846B8EEC00A0123C3
:1082C000E022394984ED140AFFF78AF8BDEEC00AAE
:1082D0002846B8EEC00A00234FF44E72334984EDAD
:1082E000110AFFF77DF8BDEEC00A284600234FF4BF
:1082F0004D722F4984ED030AFFF772F8BDEEC00AF4
:108300002846002320222B4984ED070AFFF768F84E
:10831000BDEEC00A284601234FF40272264984EDBF
:108320000B0AFFF75DF8BDEEC00A2846B8EEC00A9A
:1083300001234FF40472214984ED150AFFF750F828
:10834000BDEEC00A1E4BB8EEC00A2046196884ED87
:10835000120A5C22BDE8384016F05ABE7C98020032
:108360008C9602002013FF1F84980200549702008D
:108370008C98020094980200A0960200B496020025
:10838000C4960200DC960200E8960200F096020015
:10839000A8980200BC9802000497020010970200FF
:1083A00018970200D0980200E49802002C9702006F
:1083B0003897020040970200F89802000C990200DA
:1083C0003407FF1F2DE9F84FA54CA649A64FDFF84B
:1083D0000883DFF808B3A54DA54EDFF804A3DFF846
:1083E00004932DED028B204600234FF4B872FEF764
:1083F000F7FFBDEEC00A204600234FF462729D498C
:1084000087ED000AFEF7ECFFBDEEC00A2046002310
:108410004FF46C72984987ED010AFEF7E1FFBDEE5B
:10842000C00A204600236822944987ED030AFEF71C
:10843000D7FFBDEEC00A204641460023C02287ED8B
:10844000020AFEF7CDFFBDEEC00A204600234FF41E
:108450000F728B498BED000AFEF7C2FFBDEEC00A1A
:1084600001234FF4B072204686498BED010AFEF7D6
:10847000B7FF10EE100A1BF08DFF41EC100BCBE99B
:108480000401F8F7E1FD414620460023A022FEF753
:10849000A7FFBDEEC00A204600234FF431727A498F
:1084A00085ED000AFEF79CFFBDEEC00A01234FF4E4
:1084B000B4722046754985ED010AFEF791FF10EE72
:1084C000100A1BF067FF41EC180B41EC100BC5E9DB
:1084D0000401F8F7B9FD0C216D48DFF80C8219F0A2
:1084E00031FAB0EE480AF0EE680A0221304619F07F
:1084F00013FF304619F0B6FE1B21664819F022FA28
:10850000A968304619F0FEFE304619F0ABFE1B217B
:10851000614819F017FA95ED040B0221304619F065
:10852000FBFE304619F09EFE2046002398225B4950
:10853000FEF756FFBDEEC00A204600234FF414722A
:1085400057498AED000AFEF74BFFBDEEC00A012332
:108550004FF41172204653498AED010AFEF740FF9D
:1085600010EE100A1BF016FF41EC100BCAE90401D3
:10857000F8F76AFD204600234FF4D6724A49FEF709
:108580002FFFBDEEC00A204600234FF41372474967
:1085900089ED000AFEF724FFBDEEC00A01234FF467
:1085A00028722046424989ED010AFEF719FF10EEB4
:1085B000100A1BF0EFFE41EC100BC9E90401F8F7BB
:1085C00043FD204600234FF4DC723A49FEF708FFD2
:1085D000BDEEC00A204600234FF40672364988EDEE
:1085E000000AFEF7FDFEBDEEC00A01234FF42A7219
:1085F0002046324988ED010AFEF7F2FE10EE100A1D
:108600001BF0C8FE41EC100BC8E90401F8F71CFD93
:108610002B4B38461968102216F0FAFC294B5846A5
:108620001968182216F0F4FC274B284619681822FE
:1086300016F0EEFC254B50461968182216F0E8FC9F
:10864000234B48461968182216F0E2FCBDEC028B59
:10865000204B404619681822BDE8F84F16F0D8BCE8
:1086600028990200209902007015FF1F0817FF1FAC
:108670002408FF1FA0960200B4960200C4960200D0
:10868000489902005899020060990200709902000E
:108690007899020088990200A4990200C09902000A
:1086A000D8990200E8990200F0990200089A0200A5
:1086B000189A0200209A0200389A0200489A020092
:1086C0008C07FF1F5007FF1F5407FF1F6807FF1F7E
:1086D0007807FF1F5C07FF1F30990200F016FF1F8D
:1086E0002017FF1F3817FF1F5017FF1F38B5B42280
:1086F00000239A499A489B4C9A4DFEF771FE00233D
:10870000C82299499648FEF76BFE0023D422974968
:108710009348FEF765FEBDEEC00A0023F42294499B
:108720008F4884ED000AFEF75BFEBDEEC00A012310
:108730004FF486728F498A4884ED010AFEF750FE95
:108740000023F8228C49864884ED020AFEF748FE91
:10875000F7EE007AB4EEE70AF1EE10FAACBF0123AF
:10876000002384F87430D822012384497C48FEF722
:1087700037FEBCEEC00A0123DC228149784884ED33
:10878000210AFEF72DFEBCEEC00A00234FF4EA7268
:108790007C49734884ED220AFEF722FEBDEEC00A32
:1087A00000234FF4E67278496D4884ED040AFEF721
:1087B00017FEBDEEC00A01234FF4007273496848EA
:1087C00084ED030AFEF70CFE0023FC227049644886
:1087D00084ED050AFEF704FEF7EE007AB4EEE70A30
:1087E000F1EE10FAACBF0123002385F875304FF489
:1087F000F272002367495A485A4DFEF7F1FDBDEE6B
:10880000C00A00234FF4F0726349554884ED090A09
:10881000FEF7E6FDBDEEC00A01234FF4F4725F4996
:108820004F4884ED080AFEF7DBFD00234FF4807209
:108830005B494B4884ED0A0AFEF7D2FDF7EE007A59
:10884000B4EEE70AF1EE10FAACBF0123002385F87D
:108850007630CC22002353494148424DFEF7C0FDFB
:10886000BDEEC00A0023C4224F493D4884ED260ACC
:10887000FEF7B6FDBDEEC00A0123D8224B493848A9
:1088800084ED250AFEF7ACFD00234FF465724849DC
:10889000334884ED270AFEF7A3FDF7EE007AB4EE25
:1088A000E70AF1EE10FAACBF0123002385F8A030EF
:1088B0004FF4087200233F4929482A4DFEF790FDE6
:1088C000BDEEC00A00234FF407723B49244884EDF3
:1088D0000F0AFEF785FDBDEEC00A01234FF40972B1
:1088E00036491F4884ED0E0AFEF77AFD00234FF447
:1088F000827233491A4884ED100AFEF771FDF7EED3
:10890000007AB4EEE70AF1EE10FAACBF01230023BF
:1089100085F877304FF4CC7201232A491048FEF7CE
:108920005FFD0023942228490D4884ED110AFEF7CB
:1089300057FDBCEEC00A01234FF42C7223490848AE
:1089400084ED0D0AFEF74CFD214B84ED120A1968E7
:108950000448A822BDE8384016F05ABB509A0200DD
:108960005C9A0200E815FF1F649A0200789A0200E0
:108970008C9A0200A09A0200B49A0200C89A0200DF
:10898000DC9A0200F89A0200089B0200189B020081
:108990002C9B0200389B0200489B0200589B02005F
:1089A0006C9B0200789B02008C9B02009C9B020047
:1089B000B09B0200C09B0200D09B0200E09B020023
:1089C000EC9B0200F89B02000C9C02001C9C020025
:1089D0007C14FF1F38B53A4D3A493B4C28460023DA
:1089E0004FF4EE72FEF7FCFCBDEEC00A28460023F1
:1089F0004FF4C472354984ED130AFEF7F1FCBDEE65
:108A0000C00A28460023B022314984ED140AFEF73B
:108A1000E7FCBDEEC00A284600234FF4D4722D496E
:108A200084ED200AFEF7DCFCBDEEC00A28460023D8
:108A30004FF43072284984ED060AFEF7D1FCBDEEF2
:108A4000C00A284600238C22244984ED070AFEF739
:108A5000C7FCBDEEC00A284600234FF4157220491A
:108A600084ED1E0AFEF7BCFCBDEEC00A28460023BA
:108A70004FF410721B4984ED0B0AFEF7B1FCBDEEFA
:108A8000C00A28460023B022174984ED0C0AFEF7DD
:108A9000A7FCBDEEC00A28460023B822134984ED86
:108AA0001F0AFEF79DFC124BBDEEC00A2046196856
:108AB00084ED1F0AA822BDE8384016F0A9BA00BF0D
:108AC0002C9C0200249C0200E815FF1F349C02002D
:108AD0003C9C0200449C02004C9C0200549C0200FE
:108AE0005C9C0200649C02006C9C0200749C02006E
:108AF0007C14FF1F38B5314D3149324C28460023D4
:108B00004FF43E72FEF76CFCBDEEC00A284600230F
:108B10004FF43F722C4984ED150AFEF761FCBDEE5F
:108B2000C00A284600234FF44072284984ED160AF3
:108B3000FEF756FCBDEEC00A284600234FF44172F2
:108B4000234984ED170AFEF74BFCBDEEC00A284608
:108B500000234FF444721F4984ED180AFEF740FCCD
:108B6000BDEEC00A284600234FF445721A4984ED31
:108B7000190AFEF735FCBDEEC00A284600234FF463
:108B80004272164984ED1A0AFEF72AFCBDEEC00AAD
:108B9000284600234FF44372114984ED1B0AFEF767
:108BA0001FFC104BBDEEC00A2046196884ED1C0A5C
:108BB000A822BDE8384016F02BBA00BF809C020006
:108BC000A0960200E815FF1FB4960200889C0200E0
:108BD000989C0200A89C0200B89C0200C89C02005D
:108BE000D89C02007C14FF1F70B5574D5749584C54
:108BF000584E284600234FF4E472FEF7F1FBBDEE19
:108C0000C00A284600234FF47272534984ED000ACB
:108C1000FEF7E6FBBDEEC00A284600234FF477724C
:108C20004E4984ED010AFEF7DBFBBDEEC00A284683
:108C3000002328224A4984ED020AFEF7D1FBBDEE4B
:108C4000C00A28460123A822464984ED030AFEF7FC
:108C5000C7FB284601234FF4C672434984ED0A0A34
:108C6000FEF7BEFB284600234FF47A723F4984ED9D
:108C70000D0AFEF7B5FBBDEEC00A284600234FF4EF
:108C80007D723B4984ED040AFEF7AAFBBDEEC00AE3
:108C9000284600232422374984ED050AFEF7A0FB6D
:108CA000BDEEC00A284601234FF4AA72324984ED72
:108CB000060AFEF795FB284601234FF49E722F49C2
:108CC00084ED0B0AFEF78CFB284600234FF45E72FE
:108CD0002B4984ED0E0AFEF783FBBDEEC00A284641
:108CE00000234FF45F72274984ED070AFEF778FBF3
:108CF000BDEEC00A284600235C22234984ED080A01
:108D0000FEF76EFBBDEEC00A284601234FF4A672A3
:108D10001E4984ED090AFEF763FB2046316884EDA5
:108D20000C0A402216F074F928464FF4FA721849DA
:108D30000123FEF755FB316884ED0F0A20464022DF
:108D4000BDE8704016F064B9E89C02008C96020001
:108D5000A815FF1F6C07FF1FDC960200E8960200B3
:108D6000F0960200F09C0200FC9C020004970200B6
:108D70001097020018970200089D0200149D02003F
:108D80002C9702003897020040970200209D0200B5
:108D90002C9D0200464B474A1B68116810B5012BF9
:108DA00008BF454B9AB008BF19680AA800230122E2
:108DB00015F0F4FD11A813F07FFB002840F083812B
:108DC00002A89DF842303D490AAA13F029FC049AF2
:108DD0009DF814309DF80C1013928DF850308DF8DA
:108DE000481005AA0DF151030DF15E0012F8011FA4
:108DF00003F8011B8342F9D1099B189302A813F0D1
:108E00002DFB11A813F058FB0446002864D1012360
:108E100018212B488DF8433018F094FD294819F09B
:108E200021FA294902A819F0EBFB214602A8F8F71C
:108E3000FBFB02A819F0A4FB244902A819F0E0FBEF
:108E4000214602A8F8F7F0FB02A819F099FB204987
:108E500002A819F0D5FB214602A8F8F7E5FB02A805
:108E600019F08EFB194902A819F0CAFB214602A885
:108E7000F8F7DAFB02A819F083FB164902A819F0EB
:108E8000BFFB214602A8F8F7CFFB02A819F078FB38
:108E90000E4902A819F0B4FB214602A8F8F7C4FB5A
:108EA00002A819F06DFB0AA815F096FD1AB010BDC6
:108EB000B017FF1F6407FF1F7407FF1F6019FF1F14
:108EC000509D02002408FF1F6C9D0200B08B020021
:108ED000A0AD020010960200002314217C488DF8FA
:108EE000433018F02FFD7B4819F0BCF911A813F09E
:108EF000E3FA002840F0E380FFF7F8FBFFF7FAFD04
:108F0000FFF768FDFEF77AFEFEF7C2FDFFF75AFA9B
:108F1000FFF76AFEFEF728FFFFF700F8FEF766FC92
:108F2000FFF712F9FEF75EFD6B4902A819F068FB26
:108F3000002102A8F8F778FB02A819F021FB674985
:108F400002A819F05DFB002102A8F8F76DFB02A84A
:108F500019F016FB624A1368019301991368009394
:108F6000009B5B1A0E2BF9D95E4902A819F048FB49
:108F7000002102A8F8F758FB02A819F001FB574995
:108F800002A819F03DFB002102A8F8F74DFB02A84A
:108F900019F0F6FA544902A819F032FB002102A890
:108FA000F8F742FB02A819F0EBFA4C4902A819F0B5
:108FB00027FB002102A8F8F737FB02A819F0E0FA16
:108FC0004A4902A819F01CFB002102A8F8F72CFB63
:108FD00002A819F0D5FA414902A819F011FB0021A5
:108FE00002A8F8F721FB02A819F0CAFA404902A822
:108FF00019F006FB002102A8F8F716FB02A819F0E9
:10900000BFFA364902A819F0FBFA002102A8F8F7C6
:109010000BFB02A819F0B4FA364902A819F0F0FACD
:10902000002102A8F8F700FB02A819F0A9FA2B49C1
:1090300002A819F0E5FA002102A8F8F7F5FA02A84B
:1090400019F09EFA2C4902A819F0DAFA002102A8B8
:10905000F8F7EAFA02A819F093FA204902A819F0E1
:10906000CFFA002102A8F8F7DFFA02A819F088FA6F
:10907000224902A819F0C4FA002102A8F8F7D4FA8C
:1090800002A819F07DFA154902A819F0B9FA0021D1
:1090900002A8F8F7C9FA02A819F072FA184902A84A
:1090A00019F0AEFA002102A8F8F7BEFA02A819F0EA
:1090B00067FA0A4902A819F0A3FA0021EDE611A8FF
:1090C00013F0ECF918E711A813F0E8F978E600BFFF
:1090D000389D02002408FF1F6C9D0200B08B020027
:1090E000141CFF1FA0AD02007C9D0200889D0200A1
:1090F000949D0200A09D0200AC9D0200B89D02005C
:10910000C49D020090F8903010B504461BB906E0EB
:10911000012016F037F9A368002BF9D110BDF7F73D
:1091200033FAF8E78368E3B1816D826F4B68D21A36
:1091300030B482EAE273D0F8AC40A3EBE273A3420E
:1091400010DBD0F8B020934214DA1A190025C26758
:109150002346C0F8B05030BC4A68086800FB0323BF
:10916000CB60704700225C00C0F8B020C0F8AC2093
:10917000C467F0E7C26FD31AEDE700BF10B504462D
:10918000FFF7D0FFA3682BB1012016F0FBF8A3680E
:10919000002BF9D110BD00BF07EE901AF8EE676AF8
:1091A00007EE902A9FED1C7ADFED1C5A9FED1C6A9A
:1091B0004167F8EE677A66EE876A67EE877A66EE51
:1091C000A56A27EEA57AF6EE007AF0EE675AE6EE8B
:1091D000865AF0B4E7EE067A0346124F5861FDEE68
:1091E000E56AFDEEE77A104E026780250022012431
:1091F000076046600574C466C0ED066AC0ED077A74
:109200008260C26080F82820C265026680F864200F
:109210008266F0BC704700BFBD378635C0E1644C44
:109220000000003D8C8702008087020038B590F86E
:109230006430114A0260044600F10C0553B128461F
:1092400018F07EFF0023206AA36015F06DFB606AB2
:1092500015F06AFB094B6360284618F071FF002384
:10926000A360206A15F060FB606A15F05DFB28467C
:1092700018F066FF204638BD8C8702008087020008
:1092800010B5034B03600446FFF7D0FF204610BD26
:10929000C487020010B5054B03600446FFF7C6FF04
:1092A0002046B82118F0A0FF204610BDC487020058
:1092B00010B5034B03600446FFF7B8FF204610BD0E
:1092C000A887020010B5054B03600446FFF7AEFF08
:1092D0002046942118F088FF204610BDA887020080
:1092E00010B50446FFF7A2FF2046782118F07CFF56
:1092F000204610BD884231D02DE9F04700F1040826
:10930000414516468A46814617D0D9F80010D8F84C
:109310000000B04798B9D8F80050444601E02368EF
:1093200063602746284654F8041DB0470028F6D14C
:109330003D6008F10408C245E7D1BDE8F087C9EBFC
:1093400008029308D8F8004005D0C2F10400404458
:1093500049461CF0FBF9C9F80040EAE7704700BF36
:109360002DE9F8430B1A432B1CDD00F14008894618
:1093700041461746FFF7BEFFC14515D0D8F800504B
:10938000444601E0236863602646284654F8041DDD
:10939000B8470028F6D108F10408C1453560EDD181
:1093A000BDE8F883FFF7A6FFBDE8F8832DE9F04F8D
:1093B000561E06EBD67683B07610B14201928846EF
:1093C000054699460C9F5CDA8A4600E0DA460AF1C7
:1093D00001034FEA430B0BF18041013955F833008B
:1093E00055F8211005EBC304B84718B10BF1FF3B4A
:1093F00005EB8B04236845F82A30B345E6DB019B77
:10940000DA0707D4019BA3F1020A0AEBDA7ABBEB75
:109410006A0F06D0C34514DCC4F8009003B0BDE861
:10942000F08F0BF1010B4FEA4B0B0BF18043013B2B
:109430000BF1FF3B55F823302360C34505EB8B044C
:10944000EADD0BF1FF3606EBD6767610494655F885
:109450002600B847731E03EBD37305EB86045B103D
:1094600030B905EB8B04C4F8009003B0BDE8F08F71
:1094700055F8262045F82B20B045CDDAB3461E46D8
:10948000E4E7019BDB0700EB8104C5D48B46B9E719
:109490002DE9F04F0C1A432C85B040F38980054626
:1094A000894692461E46002A61D0031D0393E410AC
:1094B000686855F82410B0470AF1FF3A59F8041CBF
:1094C000002834D055F82400B047002837D02B6846
:1094D00055F824202A6045F8243068682968039FDD
:1094E000CB46B846B04780B9ABF104042168286880
:1094F000A346043CB0470028F8D15F4509D23A683A
:10950000DBF800103960CBF8002057F8040F296809
:10951000E7E749463346524638467C1BFFF7B8FF1B
:10952000432C45DDBAF1000F22D0B946BFE7686889
:10953000B04798B195E8030029606860CFE759F813
:10954000041C6868B0470028F4D02B6859F8042C34
:109550002A6049F8043C68682968C0E759F8041C87
:1095600055F82400B0472B680028B1D0EEE78846B4
:10957000A410A71E7F1005EB870900E0013F59F8F2
:1095800004390096224639462846FFF70FFF002F80
:10959000F4D158F8043D2A680096C5EB0804C8F8D1
:1095A00000200021A2102846FFF700FF072CF0DC66
:1095B00005B0BDE8F08F00BF836833B1614B1B6815
:1095C00013B101210220184770472DE9F04700F13F
:1095D0002C064FEA810906EB0905AE422DED028B00
:1095E00010EE107A8846044610D04FEAA902B2FA6B
:1095F00082F2C2F11F02520029463046524BFFF759
:1096000047FF514A29463046FFF7AAFEE16AA165A5
:109610008A69002A00F08E8082EAE273A3EBE2738B
:10962000B8F1010F4FF000020B618A6012DD09F101
:10963000280EA644304650F8042F936983EAE37C51
:10964000ACEBE37CC2F810C00B697045C3EB4C0374
:109650005361F0D1AE4271D04A6A04F1300306E0A2
:109660001968496A8A4203F1040328BF0A469D42E9
:10967000F6D108EE102A0023251D84F8903084F8D6
:109680002830284615F03CF92062284615F038F9B4
:10969000606215F009F904F10800616915F0BAF883
:1096A000A36DD4ED1C6A93ED067A9FED286A5B6882
:1096B000F8EE487AF8EE666AB8EEC77A67EEA67AF0
:1096C00084ED207A87EE867A0022E26784ED217AA3
:1096D00072B6D4F88430C4F8883062B672B694EDAD
:1096E000200AD4ED1F7A07EE107A27EE000AB4EEB6
:1096F000E70AD4ED227A84ED1E0AF1EE10FAD8BF03
:10970000F1EE677AC4ED237A62B6114A236AE06902
:1097100000211160DB00516803F1804303F56033E1
:1097200001440D2019611060DA68502122F0800296
:10973000DA60D960BDEC028BBDE8F087E36A93ED97
:10974000098A98E7DC1BFF1F7D0400000024744990
:10975000008003402DE9F04F2DED028BD3B041F294
:109760008832052181462DA8FFF716FDA748A84B92
:109770002D9300230360A74DA748DFF8B482036050
:109780002A6BA648D8F81C608DF84431012103608B
:10979000D8F818704891032A00F20484DFE812F028
:1097A000DE00C500AC000400D5ED057A9FED9C8A73
:1097B0006B68D5F824B00193F8EEE77A07EE109ABB
:1097C00067EE887AB8EEC78A022227EE888A0324D9
:1097D000F6B230460121FFB200920DF1740A15F085
:1097E000B7FD3846012115F0B3FD2146009A8D4C96
:1097F000504614F019FF00231E9323680693069920
:1098000023680593059A874B521A042AF8D90199BF
:109810000093504614F04AFF594614F03BFF82492A
:1098200014F068FF01221146286BF7F737F9479AC1
:1098300052AB02F10B0E03EB8E0E03EB82024FF0E4
:10984000000C42F868ACB7EE000A01212DA84EF8D2
:1098500090CCCDF81CC1FFF7AFFE009B1B680493B2
:10986000049A23680393039B9B1A042BF9D90023C2
:109870008DF8443172B6DDED4D7A9DED4C7A68EE8F
:10988000277AB4EEE77ACDED4B7ADDED4F7AF1EE43
:1098900010FA58BFF1EE677ACDED507A62B6DFF874
:1098A00094A1DFF894B1DFED5E8A2F9B002B00F0CE
:1098B000EC80F8F7E7FB002840F39080DAF800002E
:1098C000F8F7D0FBC0B253288BF8000000F05082AC
:1098D000662840F08380DAF80000F7F7F9F951ECD8
:1098E000100B1BF05BF82B6B032B59D8DFE813F040
:1098F000360328031A034B00D5ED087A9FED488AFA
:109900002B690193F8EEE77A07EE109A67EE887AF2
:10991000B8EEC78AD8F85060D8F84C70D5F800B0C7
:10992000172227EE888A102452E7D5ED077A9FED9B
:109930003C8AEB680193F8EEE77A07EE109A67EE3F
:10994000887AB8EEC78AD8F83060D8F82C70D5F885
:109950002CB0142227EE888A152439E7D5ED067A33
:109960009FED2F8AAB680193F8EEE77A07EE109A25
:1099700067EE887AB8EEC78AD5F828B0052227EEB8
:10998000888A062424E707EE900AB8EEE78A07EEF5
:10999000909A28EE288AF8EEE77A686128EE278AFE
:1099A000224B1C481968342215F032FB00238DF835
:1099B000443172B6DDED4D7A9DED4C7A68EE277A32
:1099C000F4EEC77ACDED4B7ADDED4F7AF1EE10FA79
:1099D000D8BFF1EE677ACDED507A62B6304615F019
:1099E000BDFC10B9B9F1010F2AD0384615F0B6FC0C
:1099F00010B9B9F1FF3F23D023680C930C9A236868
:109A00000B930B9B9B1A092BF9D94EE7F812FF1FFA
:109A1000A8870200C013FF1F6418FF1FB412FF1FA6
:109A20000AD7233C141CFF1FC09EF87F8407FF1F2A
:109A3000E815FF1F4807FF1FF413FF1F0000000079
:109A40008DF8440172B65FED036ADDED4D7A9DED50
:109A50004C7A67EEA67AF4EEC77AF1EE10FACDED05
:109A60004B7A00F38982DDED4F7AF1EE677ACDED26
:109A7000507A62B630A818F063FB002335982F9314
:109A800014F052FF369814F04FFF286B032800F0B3
:109A9000A3811E9BA24AA34F136007EE903A4FF09A
:109AA000000AB8EEE70AC7F800A0F7F735F919AED3
:109AB000DFF8B4929C4989ED000A304618F0A0FD09
:109AC00051463046F7F7B0FD304618F059FD2220D8
:109AD000F7F728FF99ED000A5046F7F7C7FE222056
:109AE000F7F720FFFF20F7F71DFFFF20F7F71AFF1A
:109AF000FF20F7F717FF2368189318992368179327
:109B0000179B8A4A5B1A042BF8D987490092304682
:109B100018F076FD00213046F7F786FD304618F044
:109B20002FFD2220F7F7FEFE99ED000A0020F7F73F
:109B30009DFE2220F7F7F6FEFF20F7F7F3FEFF2049
:109B4000F7F7F0FEFF20F7F7EDFE009A1368169383
:109B5000169923681593159B744A5B1A042BF8D940
:109B600073490092304618F04BFD00213046F7F75C
:109B70005BFD304618F004FD2220F7F7D3FE97ED89
:109B8000000A0020B8EEC00AF7F770FE2220F7F7AF
:109B9000C9FEFF20F7F7C6FEFF20F7F7C3FEFF2040
:109BA000F7F7C0FE009A13681493149A236813936E
:109BB000139B9B1A042BF9D901220021286BF6F77D
:109BC0006DFF2B6B032B4AD8DFE803F08D70530237
:109BD000D8F8A430012B00F0E3815649304618F044
:109BE0000FFD00213046F7F71FFD304618F0C8FC86
:109BF0005149304618F004FD00213046F7F714FDB6
:109C0000304618F0BDFC4D49304618F0F9FC0021F3
:109C10003046F7F709FD304618F0B2FC48493046A7
:109C200018F0EEFC00213046F7F7FEFC304618F045
:109C3000A7FC4449304618F0E3FC00213046F7F712
:109C4000F3FC304618F09CFC3F49304618F0D8FC35
:109C500030460021F7F7E8FC304618F091FC3B4B0A
:109C60002D932DA8FFF7E2FA53B0BDEC028BBDE8AF
:109C7000F08FD8F8A430012B00F08E8134493046A3
:109C800018F0BEFC00213046F7F7CEFC304618F045
:109C900077FC2949304618F0B3FC00213046F7F72D
:109CA000C3FC304618F06CFC2A49ADE7D8F8A43064
:109CB000012B00F064812849304618F0A1FC0021F6
:109CC0003046F7F7B1FC304618F05AFC1A493046D6
:109CD00018F096FC00213046F7F7A6FC304618F045
:109CE0004FFC1E4990E7D8F8A430012B00F05681B4
:109CF0001B49304618F084FC00213046F7F794FCED
:109D0000304618F03DFC0C49304618F079FC002133
:109D10003046F7F789FC304618F032FC114973E7FA
:109D2000B412FF1F6C15FF1FE09D0200141CFF1FE3
:109D3000D09D0200C49E0200B08B0200D89E02009B
:109D4000E88D02002C9E0200C48D0200A88702004C
:109D5000889E02009C9E02004C9E0200609E0200B3
:109D6000049E0200189E0200BC13FF1F00000000AA
:109D700000238DF8443172B65FED046ADDED4D7A53
:109D80009DED4C7A67EEA67AF4EEC77ACDED4B7A6C
:109D9000DDED4F7AF1EE10FAD8BFF1EE677ACDED36
:109DA000507A62B623680A930A9A23680993099B3A
:109DB000814E9B1A042BF8D92DA8FFF7A3F933681D
:109DC0000893089A23680793079B9B1A632BF9D97A
:109DD000286B03287FF45DAED8F80410D8F8003063
:109DE0001E9A98ED027ADFED756A7548754F02602C
:109DF00003FB01F307EE903A06EE102AF8EE677ABD
:109E0000B8EEC66A67EE877A6F4B70491A6086EEC5
:109E1000277A6F4B19AE4FF000093046C3F8009017
:109E200067EE267AC7ED007A18F0EAFB494630461D
:109E3000F7F7FAFB304618F0A3FB2220F7F772FD84
:109E400097ED000A4846F7F711FD2220F7F76AFD63
:109E5000FF20F7F767FDFF20F7F764FDFF20F7F716
:109E600061FD23681293129923681193119B524A42
:109E70005B1A042BF8D955490092304618F0C0FB04
:109E800000213046F7F7D0FB304618F079FB22204E
:109E9000F7F748FD97ED000A0020F7F7E7FC2220CE
:109EA000F7F740FDFF20F7F73DFDFF20F7F73AFDFC
:109EB000FF20F7F737FD009A13681093109A236874
:109EC0000F930F9B3C4F9B1A042BF8D94149304606
:109ED00018F096FB00213046F7F7A6FB304618F045
:109EE0004FFB2220F7F71EFD394B93ED000A0020AF
:109EF000B8EEC00AF7F7BAFC2220F7F713FDFF20EF
:109F0000F7F710FDFF20F7F70DFDFF20F7F70AFD2B
:109F10003B680E930E9A23680D930D9B9B1A042B9E
:109F2000F9D949E607EE900AB8EEE78A07EE909A6B
:109F300028EE288AF8EEE77A286228EE278A2FE5AD
:109F400007EE900AB8EEE78A07EE909A28EE288A84
:109F5000F8EEE77AE86128EE278A21E507EE900A15
:109F6000B8EEE78A07EE909A28EE288AF8EEE77AAC
:109F7000A86128EE278A13E5DDED4F7A77E51649CB
:109F8000304618F03DFB00213046F7F74DFB3046D8
:109F900018F0F6FA114958E61149F1E71149EFE7CF
:109FA0001149EDE74FF0000B9FED108ACDF804B09A
:109FB000052206240CE400BF141CFF1F0000B4435C
:109FC0006418FF1F9016FF1F6C15FF1FD09D020025
:109FD000B412FF1FE09D0200389E0200B08B020009
:109FE000749E0200F09D0200B09E0200000000007E
:109FF0002DE9F04F2DED048BADF54B7D144600900F
:10A00000029141F28832052180A8FFF7C5F84FF090
:10A01000000B754B8093012541F288320521A5A8DC
:10A020009B95724E8DF890B2FFF7B6F86E4BA593E4
:10A030000222032140A8C0958DF824B314F0F4FA4D
:10A0400010216B48D6F81C80D6F81890694F17F08D
:10A0500079FC2146684818F055F9674818F002F96C
:10A06000032C4FF005024FF0060150A8BABF5D4621
:10A0700001245C4614F0D8FA1422152160A814F0CB
:10A08000D3FA172270A8102114F0CEFA3A6B012AE5
:10A0900001F01E82022A01F0EE81002A00F0B8854C
:10A0A0009FED568ADFF87CA15FFA88F840460121CF
:10A0B0005FFA89F915F04CF90121484615F048F985
:10A0C00000224192DAF800207B690C9203930C99EC
:10A0D0007B68D7F824B00193DAF800300B930B9B20
:10A0E0005B1A042BF8D9019A029B03FB02F3194671
:10A0F00040A814F0DBFA594614F0CCFA404914F0A9
:10A10000F9FA08213F4817F01DFC0A213E4817F0D4
:10A1100019FC0199384818F0F5F8374818F0A2F8FA
:10A120000821384817F00EFC0721384817F00AFCC0
:10A130005946314818F0E6F82F4818F093F80821EE
:10A14000304817F0FFFB1121314817F0FBFB2C4979
:10A15000294818F0D7F8284818F084F8E4B1D7F85F
:10A1600030B0BBF1010F01F0D182BBF1020F01F061
:10A170007482BBF1000F01F014820521254817F00D
:10A18000E1FB0421244817F0DDFB01211A4818F0F7
:10A19000B9F8194818F066F8002D41F0CF80DFEDCE
:10A1A000178A9FED1E9A14B9002D00F06D87DAF81A
:10A1B00000301893189ADAF800301793179B9B1AFF
:10A1C000042BF8D9F7F75EFF0028C0F2AF80DFF864
:10A1D00058B0DBF80000F7F745FF1149C0B2A0F115
:10A1E0005303087022E000BFA8870200E815FF1F94
:10A1F000EC9E02002819FF1F2408FF1F000000002A
:10A20000C09EF87F009F02000C9F0200548F020046
:10A21000189F02002C9F0200349F02000AD7233CA3
:10A22000F413FF1F141CFF1F4807FF1F722B7DD85C
:10A23000DFE813F0FE037C007C007C007C007C00E7
:10A240007C008604B1037C007C007C007C007C00E8
:10A250007C007C002A037C007C007C007C007C006D
:10A260007C007C00D70272027C0042020B027C0060
:10A270007C007C007C007C007C007C007C007C00FE
:10A280007C007C007C007C007C007C007C007C00EE
:10A290007C007C007C007C007C007C007C007C00DE
:10A2A0007C007C007C007C007C007C007C007C00CE
:10A2B0007C007C007C007C007C007C007C007C00BE
:10A2C0007C007C007C007C007C007C007C007C00AE
:10A2D0007C007C007C007C00BE016A017C007C006C
:10A2E0007C007C0002018A007C007C007C007C00F9
:10A2F0007C007C007C007C007C007C007C007C007E
:10A300007C007C007C007C007C007C007C007C006D
:10A310007C007C007C007C007300F7F7C7FEA04B3C
:10A32000386319689F48342214F072FE002C6FD1F4
:10A33000DAF800303493349ADAF800303393339BF0
:10A340009B1A042BF8D92EE7A79B002BEED1D7ED53
:10A35000087A3969009370A8B8EEE78A14F0A6F974
:10A36000914914F0C7F9012211460220F6F796FB35
:10A37000BF9A009BBF93CAA901EB820470AA44F85C
:10A38000643CB7EE000A0121A5A844F8682CFFF749
:10A3900013F9009B8DF8243328EE098A72B6DDED9F
:10A3A000C57A9DEDC47A67EEA87AF4EEC77ACDED52
:10A3B000C37ADDEDC77AF1EE10FAD8BFF1EE677A15
:10A3C000CDEDC87A62B6DAF800302E932E9ADAF81C
:10A3D00000302D932D9B9B1A042BF8D900238DF868
:10A3E000243372B6DDEDC57A9DEDC47A68EE277A26
:10A3F000F4EEC77ACDEDC37ADDEDC77AF1EE10FA4F
:10A40000D8BFF1EE677ACDEDC87A62B6012300932A
:10A41000404614F0A3FF044618B9009B012B00F03E
:10A420002484484614F09AFF044618B9009B01336F
:10A4300000F0268501247BE7A79B002B7FF476AFF5
:10A440003969D7ED087A0093494270A8B8EEE78AD7
:10A4500014F02CF9554914F04DF90122114602204F
:10A46000F6F71CFBBF9A009BBF93CAA901EB8204BD
:10A4700070AA44F8643CB7EE000A0121A5A844F88C
:10A48000682CFFF799F8009B8DF8243328EE098A91
:10A4900072B6DDEDC57A9DEDC47A67EEA87AF4EE6A
:10A4A000C77ACDEDC37ADDEDC77AF1EE10FAD8BFE9
:10A4B000F1EE677ACDEDC87A62B6DAF800302C9307
:10A4C0002C9ADAF800302B932B9B9B1A042BF8D98B
:10A4D00000238DF8243372B6DDEDC57A9DEDC47A84
:10A4E00068EE277AF4EEC77ACDEDC37ADDEDC77A50
:10A4F000F1EE10FAD8BFF1EE677ACDEDC87A62B608
:10A500004FF0FF33009383E7A79B002B7FF40EAF40
:10A51000D7ED077AF968009360A8B8EEE78A14F0DF
:10A52000C5F8214914F0E6F8012211461046F6F765
:10A53000B5FABF9A009BBF93CAA901EB820460AA37
:10A5400044F8643CB7EE000A0121A5A844F8682C41
:10A55000FFF732F8009B8DF8243328EE098A72B693
:10A56000DDEDC57A9DEDC47A67EEA87AF4EEC77A80
:10A57000CDEDC37ADDEDC77AF1EE10FAD8BFF1EE7A
:10A58000677ACDEDC87A62B6DAF800302A932A9A53
:10A59000DAF800302993299B9B1A042BF8D91DE780
:10A5A0009007FF1F2819FF1FC09EF87F406107809A
:10A5B000A79B002B7FF4BAAEF968D7ED077A00931A
:10A5C000494260A8B8EEE78A14F070F8AA4914F07E
:10A5D00091F8012211461046F6F760FABF9A009BE7
:10A5E000BF93CAA901EB820460AA44F8643CB7EEA9
:10A5F000000A0121A5A844F8682CFEF7DDFF009BA6
:10A600008DF8243328EE098A72B6DDEDC57A9DED0A
:10A61000C47A67EEA87AF4EEC77ACDEDC37ADDEDA1
:10A62000C77AF1EE10FAD8BFF1EE677ACDEDC87AAD
:10A6300062B6DAF800302893289ADAF800302793C7
:10A64000279B9B1A042BF8D942E7DBF80000F6F7AA
:10A650003FFB51EC100B1AF0A1F93B6B874A012B21
:10A6600000F07F87022B00F0858733B907EE900A50
:10A67000B8EEE78A906128EE098A814B7F48196815
:10A68000342214F0C5FC00238DF8243372B6DDEDBE
:10A69000C57A9DEDC47A68EE277AF4EEC77ACDEDDF
:10A6A000C37ADDEDC77AF1EE10FAD8BFF1EE677A22
:10A6B000CDEDC87A62B639E6DBF80000F6F708FBA4
:10A6C00051EC100B1AF06AF96D4B834619686B4810
:10A6D000C7F814B0342214F09BFC00238DF890329C
:10A6E00072B607EE90BAB8EEE77ADDEDA07ADDED4E
:10A6F0009F6A27EE097A67EE277AF4EEE67ACDEDC7
:10A700009E7ADDEDA27AF1EE10FAD8BFF1EE677A0B
:10A71000CDEDA37A62B609E6DDF808B2BBF1000F11
:10A720007FF404AED7ED057A019BF8EEE77A594243
:10A7300040A867EE899A13F0B9FF524913F0DAFF87
:10A74000012211460320F6F7A9F99A9ACDF868B2CA
:10A7500080AB03EB8205184640ABB7EE000A01213F
:10A76000EB62C5F830B0FEF727FF8DF890B272B6F5
:10A77000DDEDA07A9DED9F7A67EEA87AF4EEC77AB8
:10A78000CDED9E7ADDEDA27AF1EE10FAD8BFF1EEB2
:10A79000677ACDEDA37A62B6DAF800302693269A6E
:10A7A000DAF800302593259B9B1A042BF8D9002357
:10A7B0008DF8903272B6DDEDA07A9DED9F7A69EE4C
:10A7C000A77AF4EEC77ACDED9E7ADDEDA27AF1EEAE
:10A7D00010FAD8BFF1EE677ACDEDA37A62B6012503
:10A7E000A4E5DDF808B2BBF1000F7FF49FADD7ED13
:10A7F000057A0199F8EEE77A40A867EE899A13F096
:10A8000055FF204913F076FF012211460320F6F789
:10A8100045F99A9ACDF868B280AB03EB82051846E9
:10A8200040ABB7EE000A0121EB62C5F830B0FEF78D
:10A83000C3FE8DF890B272B6DDEDA07A9DED9F7AE1
:10A8400067EEA87AF4EEC77ACDED9E7ADDEDA27AB6
:10A85000F1EE10FAD8BFF1EE677ACDEDA37A62B6C9
:10A86000DAF800302493249ADAF800302393239BFB
:10A870009B1A042BF8D99AE7406107802819FF1F1B
:10A880009007FF1FC09EF87F00238DF8243372B617
:10A89000DDEDC57A9DEDC47A67EEA87AF4EEC77A4D
:10A8A000CDEDC37ADDEDC77AF1EE10FAD8BFF1EE47
:10A8B000677ACDEDC87A62B6DAF800302093209A34
:10A8C000DAF800301F931F9B9B1A042BF8D9A5A818
:10A8D000FEF718FC396B012900F05C86022900F0B4
:10A8E000528619B901220846F6F7D8F8D6F8A430EE
:10A8F000012B00F02886B8493CA817F081FE002102
:10A900003CA8F6F791FE3CA817F03AFEB3493CA8E4
:10A9100017F076FE00213CA8F6F786FE3CA817F05B
:10A920002FFEAF493CA817F06BFE00213CA8F6F7BC
:10A930007BFE3CA817F024FEAA493CA817F060FE55
:10A9400000213CA8F6F770FE3CA817F019FEA649B6
:10A950003CA817F055FE00213CA8F6F765FE3CA880
:10A9600017F00EFEA1493CA817F04AFE00213CA8B2
:10A97000F6F75AFE3CA817F003FEDAF800302293EF
:10A98000229ADAF800302193219B9B1AB3F57A7F43
:10A99000F7D30024CCE4DDF89CB2BBF1000F7FF4C8
:10A9A000C5ACB968D7ED067A494250A8B8EEE78A37
:10A9B00013F07CFE8E4913F09DFE0122114658468D
:10A9C000F6F76CF8BF9ACDF8FCB2CAAB03EB820481
:10A9D00050ABB7EE000A0121A5A844F8683C44F842
:10A9E00064BCFEF7E9FD28EE098A8DF824B372B63F
:10A9F000DDEDC57A9DEDC47A67EEA87AF4EEC77AEC
:10AA0000CDEDC37ADDEDC77AF1EE10FAD8BFF1EEE5
:10AA1000677ACDEDC87A62B6DAF800301E931E9AD6
:10AA2000DAF800301D931D9B9B1A042BF8D94FE5D3
:10AA30000821704816F086FF06216F4816F082FF45
:10AA400000238DF8903272B6DDEDA07A9DED9F7AED
:10AA500067EEA87AF4EEC77ACDED9E7ADDEDA27AA4
:10AA6000F1EE10FAD8BFF1EE677ACDEDA37A62B6B7
:10AA7000DAF800301A931A9ADAF800301993199B11
:10AA80009B1A042BF8D980A8FEF73CFB08215948F3
:10AA900016F058FF0721594816F054FF584817F090
:10AAA000E1FB012200210320F5F7F8FFD6F8A430DE
:10AAB000012B00F03A8553493CA817F0A1FD002175
:10AAC0003CA8F6F7B1FD3CA817F05AFD43493CA855
:10AAD00017F096FD00213CA8F6F7A6FD3CA817F05C
:10AAE0004FFD49493CA817F08BFD00213CA8F6F723
:10AAF0009BFD3CA817F044FD3A493CA817F080FDA7
:10AB000000213CA8F6F790FD3CA817F039FD364926
:10AB10003CA817F075FD00213CA8F6F785FD3CA880
:10AB200017F02EFD31493CA817F06AFD00213CA822
:10AB3000F6F77AFD3CA817F023FD0025FFF7F6BBDA
:10AB4000DDF89CB2BBF1000F7FF4F0ABD7ED067AD5
:10AB5000B96850A8B8EEE78A13F0A8FD2B4913F0A6
:10AB6000C9FD012211465846F5F798FFBF9ACDF866
:10AB7000FCB2CAAB03EB820450ABB7EE000A012172
:10AB8000A5A844F8683C44F864BCFEF715FD28EE1F
:10AB9000098A8DF824B372B6DDEDC57A9DEDC47ACD
:10ABA00067EEA87AF4EEC77ACDEDC37ADDEDC77A09
:10ABB000F1EE10FAD8BFF1EE677ACDEDC87A62B641
:10ABC000DAF800301C931C9ADAF800301B931B9BB8
:10ABD0009B1A042BF8D901E49C9F0200B08B020061
:10ABE000B09F0200E88D02002C9E0200C48D02007E
:10ABF00040610780009F02003C9F0200449F0200CA
:10AC00002408FF1F609F0200749F0200C09EF87F0F
:10AC1000009BB968D7ED067AD7F828B0519201FBAE
:10AC200003F150A80192B8EEE78AD6F81C80D6F856
:10AC30001890DFF848A213F039FD594613F02AFDA9
:10AC4000019A114613F070FDDAF800200692069979
:10AC5000DAF800300593059B5B1A042BF8D97C4980
:10AC600050A813F061FDFFF71FBA1821794816F0BC
:10AC700069FE794817F0F6FA8DF8244372B6DDEDD7
:10AC8000C57A9DEDC47A67EEA87AF4EEC77AF1EE44
:10AC900010FACDEDC37A40F30D83DDEDC77ACDED2B
:10ACA000C87A62B6A8A817F04BFA0024AD98A7940A
:10ACB00013F03AFEAE9813F037FED6F88C30002B26
:10ACC00078D08DF8904272B6DDEDA07A9DED9F7A36
:10ACD00067EEA87AF4EEC77ACDED9E7ADDEDA27A22
:10ACE000F1EE10FAD8BFF1EE677ACDEDA37A62B635
:10ACF000DAF800303093309ADAF800302F932F9B37
:10AD00009B1A042BF8D983A817F01AFA0025889803
:10AD1000829513F009FE899813F006FE2946012258
:10AD20000320F5F7BBFED6F8A430012B00F0858395
:10AD30004A493CA817F064FC29463CA8F6F774FC85
:10AD40003CA817F01DFC46493CA817F059FC2946C1
:10AD50003CA8F6F769FC3CA817F012FC41493CA856
:10AD600017F04EFC29463CA8F6F75EFC3CA817F00D
:10AD700007FC3D493CA817F043FC29463CA8F6F7E0
:10AD800053FC3CA817F0FCFB38493CA817F038FCF2
:10AD900029463CA8F6F748FC3CA817F0F1FB3449DB
:10ADA0003CA817F02DFC3CA82946F6F73DFC3CA832
:10ADB00017F0E6FBD6F8A430012B00F080822D4975
:10ADC0003CA817F01DFC00213CA8F6F72DFC3CA880
:10ADD00017F0D6FB22493CA817F012FC00213CA832
:10ADE000F6F722FC3CA817F0CBFB23493CA817F050
:10ADF00007FC00213CA8F6F717FC3CA817F0C0FBA5
:10AE000019493CA817F0FCFB00213CA8F6F70CFC04
:10AE10003CA817F0B5FB15493CA817F0F1FB002141
:10AE20003CA8F6F701FC3CA817F0AAFB10493CA887
:10AE300017F0E6FB00213CA8F6F7F6FB3CA817F05C
:10AE40009FFB484614F08AFA0024FFF771BA00BF4E
:10AE5000C09EF87FC49F02002408FF1F609F02006D
:10AE6000B08B0200749F0200E88D02002C9E02004D
:10AE7000C48D02009C9F0200B09F0200141CFF1FA3
:10AE80001821774816F05EFD764817F0EBF98DF83B
:10AE9000244372B6DDEDC57A9DEDC47A67EEA87ADB
:10AEA000F4EEC77AF1EE10FACDEDC37A40F3FD81EE
:10AEB000DDEDC77ACDEDC87A62B6A8A817F040F9E3
:10AEC0000024AD98A79413F02FFDAE9813F02CFD3D
:10AED000D6F88C30002B78D08DF8904272B6DDED2C
:10AEE000A07A9DED9F7A67EEA87AF4EEC77ACDED51
:10AEF0009E7ADDEDA27AF1EE10FAD8BFF1EE677A14
:10AF0000CDEDA37A62B6DAF800303293329ADAF8ED
:10AF100000303193319B9B1A042BF8D983A817F08A
:10AF20000FF900258898829513F0FEFC899813F09C
:10AF3000FBFC294601220320F5F7B0FDD6F8A4302A
:10AF4000012B00F08B8248493CA817F059FB294699
:10AF50003CA8F6F769FB3CA817F012FB43493CA854
:10AF600017F04EFB29463CA8F6F75EFB3CA817F00D
:10AF700007FB3F493CA817F043FB29463CA8F6F7DE
:10AF800053FB3CA817F0FCFA3A493CA817F038FBF1
:10AF900029463CA8F6F748FB3CA817F0F1FA3649D9
:10AFA0003CA817F02DFB29463CA8F6F73DFB3CA832
:10AFB00017F0E6FA31493CA817F022FB3CA82946D5
:10AFC000F6F732FB3CA817F0DBFAD6F8A430012BD9
:10AFD00000F082812A493CA817F012FB00213CA80E
:10AFE000F6F722FB3CA817F0CBFA20493CA817F053
:10AFF00007FB00213CA8F6F717FB3CA817F0C0FAA6
:10B0000020493CA817F0FCFA00213CA8F6F70CFBFD
:10B010003CA817F0B5FA17493CA817F0F1FA00213F
:10B020003CA8F6F701FB3CA817F0AAFA12493CA885
:10B0300017F0E6FA00213CA8F6F7F6FA3CA817F05C
:10B040009FFA0E493CA817F0DBFA00213CA8F6F75E
:10B05000EBFA3CA817F094FA0024FFF769B900BF97
:10B06000E09F02002408FF1F609F0200B08B0200D7
:10B07000749F0200E88D02002C9E0200C48D020025
:10B080009C9F0200B09F020008219A489A4C16F03B
:10B0900059FC0521994816F055FC0721984816F0EF
:10B0A00051FC984817F0DEF83A6B012A00F0D28183
:10B0B000022A00F0BE8112B9519A2260519571683E
:10B0C0003268419896ED027ADFED8F6A8F4D02FB70
:10B0D00001F307EE903A06EE100AF8EE677AB8EE42
:10B0E000C66A67EE877A8A4A8A49106086EE277AAE
:10B0F0003CA867EE267AC5ED007A17F081FA0021A8
:10B100003CA8F6F791FA3CA817F03AFA2220F6F795
:10B1100009FC95ED000A0020F6F7A8FB2220F6F7BF
:10B1200001FCFF20F6F7FEFBFF20F6F7FBFBFF20FC
:10B13000F6F7F8FBDAF800203B923B99DAF800309A
:10B140003A933A9B744E5B1A042BF7D971493CA889
:10B1500017F056FA00213CA8F6F766FA3CA817F05B
:10B160000FFA2220F6F7DEFB95ED000A0020F6F735
:10B170007DFB2220F6F7D6FBFF20F6F7D3FBFF205E
:10B18000F6F7D0FBFF20F6F7CDFB326839923999FC
:10B19000DAF800303893389B5F4E5B1A042BF7D9EE
:10B1A00094ED000A386B5D4DB8EEC00AF5F7B4FDBA
:10B1B0005B4985ED000A3CA817F022FA00213CA863
:10B1C000F6F732FA3CA817F0DBF92220F6F7AAFBD3
:10B1D00095ED000A0020F6F749FB2220F6F7A2FBC6
:10B1E000FF20F6F79FFBFF20F6F79CFBFF20F6F70A
:10B1F00099FB326837923799DAF800303693369BEC
:10B20000454C5B1A042BF7D945493CA817F0F8F9CF
:10B2100000213CA8F6F708FA3CA817F0B1F9222063
:10B22000F6F780FB95ED000A0020F6F71FFB2220C1
:10B23000F6F778FBFF20F6F775FBFF20F6F772FBB9
:10B24000FF20F6F76FFB22683C923C99DAF8003059
:10B250003593359B5B1A042BF8D90024314B41946C
:10B260002146012203201C60F5F718FC21462046E8
:10B270000122F5F713FC012221461046F5F70EFCDA
:10B28000214601220220F5F709FC274BA593A5A82A
:10B29000FDF7CCFF244B809380A8FDF7C7FF0DF589
:10B2A0004B7DBDEC048BBDE8F08FDDEDC77AF1EE90
:10B2B000677AFFE5DDEDC77AF1EE677AEFE41B49C7
:10B2C0003CA817F09DF900213CA8F6F7ADF93CA881
:10B2D00017F056F91649AAE514493CA817F090F959
:10B2E00000213CA8F6F7A0F93CA817F049F910494D
:10B2F000A8E600BF009F0200B412FF1F2C9F0200AF
:10B30000449F02002408FF1F0000B4439016FF1F53
:10B310006C15FF1FD09D0200141CFF1FBC13FF1FE4
:10B32000E09D0200F812FF1FA8870200889F02001C
:10B33000B08B0200000000000AD7233C0122114616
:10B340000320F5F7ABFBDAF8002016921699DAF82D
:10B3500000301593159B5B1A042BF8D99A9A80AB91
:10B3600002F10B0E03EB8E0E03EB82024FF0000B8B
:10B3700040ABD362B7EE000A012180A8CEF804B03A
:10B38000CDF868B2FEF718F98DF890B272B65FED9D
:10B39000176ADDEDA07A9DED9F7A67EEA67AF4EE4E
:10B3A000C77ACDED9E7ADDEDA27AF1EE10FAD8BF24
:10B3B000F1EE677ACDEDA37A62B6DAF80020149246
:10B3C0001499DAF800301393139B5B1A092BF8D900
:10B3D00000228DF8902272B69DED037A5FED2A7AF5
:10B3E0009DEDA06ADDED9F6AB8EEC77A67EE277A19
:10B3F00067EE867AF4EEE67ACDED9E7ADDEDA27AFE
:10B40000F1EE10FAD8BFF1EE677ACDEDA37A62B60D
:10B410000821B44816F096FA0421B34816F092FABF
:10B420000121B24816F06EFFB04816F01BFFFEF780
:10B43000B6BE719A2260719541E6AD493CA817F0FD
:10B44000DFF829463CA8F6F7EFF83CA817F098F883
:10B45000A849A5E4619A2260619530E6A4493CA818
:10B4600017F0CEF829463CA8F6F7DEF83CA817F00E
:10B4700087F8A0499FE5009B3969D7ED087A3A68BB
:10B48000019201FB03F170A8B8EEE78ACDF8C4B1D0
:10B49000D6F85080D6F84C90DFF864A213F006F985
:10B4A000019A114613F0F6F8594613F03DF9DAF80F
:10B4B00000200A920A99DAF800300993099B5B1A76
:10B4C000042BF8D98C4970A813F02EF9FEF7ECBDC7
:10B4D000009BF968D7ED077AFA6A019201FB03F144
:10B4E00060A8B8EEE78ACDF884B1D6F83080D6F8F7
:10B4F0002C90DFF80CA213F0D9F8019A114613F042
:10B50000C9F8594613F010F9DAF8002008920899A2
:10B51000DAF800300793079B5B1A042BF8D97649B9
:10B5200060A813F001F9FEF7BFBD71493CA817F000
:10B5300067F800213CA8F6F777F83CA817F020F848
:10B540006C49FFF7F0BA6D493CA817F059F8002193
:10B550003CA8F6F769F83CA817F012F86549FFF720
:10B5600002BA07EE900AB8EEE78AD06128EE098A9F
:10B57000FFF783B807EE900AB8EEE78A106228EE6C
:10B58000098AFFF77AB8084601220021F5F786FA02
:10B59000FFF7ACB90A4608460021F5F77FFAFFF736
:10B5A000A5B9012211465846F5F778FABF9ACDF8A9
:10B5B000FCB2CAAB03EB820E50ABB7EE000A01211E
:10B5C000A5A84EF8683C4EF864BCFDF7F5FF8DF871
:10B5D00024B372B6DFED4B6ADDEDC57A9DEDC47A1A
:10B5E00067EEA67AF4EEC77ACDEDC37ADDEDC77AC1
:10B5F000F1EE10FAD8BFF1EE677ACDEDC87A62B6F7
:10B60000DAF800200E920E99DAF800300D930D9BB7
:10B610005B1A092BF8D99FED3C7AD7ED067AF8EE44
:10B62000E77A002267EE877A8DF8242372B6DDED83
:10B63000C56A9DEDC47A67EEA67AF4EEC77ACDEDC1
:10B64000C37ADDEDC77AF1EE10FAD8BFF1EE677A72
:10B65000CDEDC87A62B6FEF790BD0122584611467C
:10B66000F5F71CFABF9ACAAB02F10B0E03EB8E0E74
:10B6700003EB82024FF0000B70AB42F8683CB7EE70
:10B68000000A0121A5A84EF890BCCDF8FCB2FDF748
:10B6900093FF8DF824B372B6DFED1A6ADDEDC57A3B
:10B6A0009DEDC47A67EEA67AF4EEC77ACDEDC37A43
:10B6B000DDEDC77AF1EE10FAD8BFF1EE677ACDED85
:10B6C000C87A62B6DAF8002012921299DAF80030DD
:10B6D0001193119B5B1A092BF8D99FED0B7AD7EDCB
:10B6E000087A9CE7009F0200349F02002408FF1F95
:10B6F0004C9F0200B08B0200C09EF87F889F020022
:10B70000141CFF1F000000000AD7233C5A4659466C
:10B710005846F5F7C3F900228DF8242372B65FED81
:10B72000076ADDEDC57A9DEDC47A67EEA67AF4EE80
:10B73000C77ACDEDC37ADDEDC77AF1EE10FAD8BF46
:10B74000F1EE677ACDEDC87A62B6BF9ACAAB02F164
:10B750000B0103EB810103EB820260A8002342F896
:10B76000680CB7EE000A41F8903CA5A80121BF93F0
:10B77000FDF722FFDAF8002010921099DAF8003075
:10B780000F930F9B5B1A092BF8D91FED217AD7ED88
:10B79000077A44E72DE9F04F8B002DED028B00F185
:10B7A0002C0808EB0305A84585B004460F46B0EE0B
:10B7B000408A00F006819A10B2FA82F2C2F11F02AA
:10B7C0005200B64B29464046FDF762FEB34A294671
:10B7D0004046FDF7C5FDE66AA665012F40F30B81E3
:10B7E0003069C64601225EF8041F0B690132C0EBC6
:10B7F000430397424B61F6DCA84500F02681D4F85C
:10B800002C8004F13002D8F8183011460DE00F6892
:10B81000BF6983EAE37E87EAE77CAEEBE37EACEBCD
:10B82000E77C0431F445B8BF3B468D42EFD1002B95
:10B83000B8BF5B4207EE903AF8EEE77AD8F82430CA
:10B84000D6F81C80366A67EE887AFCEEE77A17EE47
:10B85000907A06E01168496A8B4202F1040228BF1F
:10B860000B469542F6D11D4600B127B905B0BDEC97
:10B87000028BBDE8F08F4FF0000304F1040984F857
:10B880002830484613F03CF82062484613F038F858
:10B89000606213F009F8616904F1080012F0BAFF60
:10B8A000A36D5A68DB68A267C2EB0309B9F1000F08
:10B8B000B8BFC9F1000908FB08F306FB06F09B4678
:10B8C00007FB07F2CDF804904FF0000C00219146E1
:10B8D000019BE367B0EB0B0261EB0C03C4E92601AB
:10B8E0006D00104619465A4663464FF0000AC4E9F7
:10B8F0002423C4F88870C4F884602A460023C4F85E
:10B90000A850C4F88080C4E9289ACDE902BC19F097
:10B91000EBF9019A801841EBE271CB0FC01841F1AD
:10B9200000014F104FEA3006002E43DBB24241DBEC
:10B93000DDE902BCB9EB0B096AEB0C0A2A460023CD
:10B940004846514619F0D0F9864240F38780C0EB53
:10B950004606C4F8B060C4F8AC00A368B8F1000FA4
:10B9600076D0002B7FD01A684D498A4245D84D4A7F
:10B97000B2FBF8F21A60226A4B49E4690020032501
:10B980000126DE60AA4098609D60086002F1804355
:10B990004A6803F5603322440D201A610860DA68B2
:10B9A000502122F08002DA60D96005B0BDEC028B34
:10B9B000BDE8F08F192013F0E5FC192013F0E2FC2C
:10B9C000F8E7C66A866501293FF70AAF3069324653
:10B9D000B369756AD2F81C80166A002BB8BF5B4247
:10B9E00007EE903AB8EEE77A67EE087AFCEEE77A6F
:10B9F00017EE907A38E7306901E758682949B1FBBA
:10BA0000F8F1121A914209D38A1A0026012503205F
:10BA10009E60DD601A6098601960ACE7606902683A
:10BA20000027012503269F601268DD6019609E6073
:10BA30009047A368002B9ED11C4A1268002A9AD016
:10BA4000284602219047A36895E73246E66ABFE799
:10BA5000DBB19A6822F002029A608CE7C4F8B06009
:10BA6000C4F8AC6079E7114A0E4D1268B5FBF8F5E1
:10BA70001AB1022101209047A3680020012103226E
:10BA80009860D9601D609A6075E7084B1B687BB1B0
:10BA9000022101209847A368DBE700BF6D04000086
:10BAA0007FA903000087930300800340DC1BFF1F76
:10BAB0004346CEE72DE9F04F2DED028BEDB08046E9
:10BAC00041F288320E463EA80521FDF765FB184B72
:10BAD0003E930522002306210EA8599312F0A4FDDF
:10BAE000142215211EA812F09FFD124F17221021BB
:10BAF0002EA812F099FD35210F48FC69BD6915F09B
:10BB000021FF0E4816F0AEFB41460C4816F0FAFB3A
:10BB10000A4816F0A7FBB8F1050F00F23C87DFE8F2
:10BB200018F003023D039F05B70429060F0000BF6C
:10BB3000C4870200E815FF1F0CA002002408FF1FA5
:10BB40000122114602203C6DD7F84CB0C54DF4F7E8
:10BB5000A5FF7B6B95ED0F0A002B41F05080F5F7A8
:10BB60000DF910EE100A18F015FCCDE900016A6A13
:10BB7000EB699FEDBD7A03FB02F308EE103AF8EE95
:10BB8000C87A4FF0000927EE878A2EA8FDEEC87A02
:10BB9000CDF8BC9017EE901A12F088FD296A12F0C9
:10BBA00079FD8246304618F0E3FBDDE9002318F00A
:10BBB00045FC18F0F3FE0146504612F0B5FD0D218C
:10BBC000AA4815F0BFFE786C18F0E4FB41EC100BAE
:10BBD0000221A74816F0A0FBA54816F043FB0A2156
:10BBE000A44815F0AFFE4B460A22F96BA04816F0A8
:10BBF00049FB9F4816F036FB0B219F4815F0A2FE2B
:10BC00004B460A22B96B9A4816F03CFB984816F04E
:10BC100029FB0921994815F095FEE86B18F0BAFB4D
:10BC200041EC100B0421924816F076FB904816F078
:10BC300019FB0621924815F085FE9DED000B0221AF
:10BC40008B4816F069FB8A4816F00CFB0A218D48D8
:10BC500015F078FEE969864816F054FB844816F022
:10BC600001FB0E21884815F06DFE696A804816F0C8
:10BC700049FB7F4816F0F6FA0B21844815F062FE66
:10BC800018EE100A18F086FB41EC100B02217848E0
:10BC900016F042FB764816F0E5FA06217C4815F0CE
:10BCA00051FE296A72484B460A2216F0EBFA704898
:10BCB00016F0D8FA589BCDF860916CA903F10B02ED
:10BCC00001EB820201EB83032EAD43F88C5CB7EEEF
:10BCD000000A01213EA842F8B49CFFF75BFDE4B2E4
:10BCE0005FFA8BF52046012113F032FB2846012133
:10BCF00013F02EFB409BDFF8B8A1DFF8B891DFF816
:10BD0000B8B143B3204613F029FB10B9002E00F35D
:10BD10001886284613F022FB10B9002EC0F229869F
:10BD2000F6F7B0F9002809DBDAF80000F6F79AF91F
:10BD3000C0B2532889F8000000F0FB85554A13680B
:10BD40000593059913680493049B5B1A012BF9D999
:10BD5000409B002BD6D150490AA816F051FC002177
:10BD60000AA8F5F761FC0AA816F00AFC4B490AA8D4
:10BD700016F046FC00210AA8F5F756FC0AA816F0B2
:10BD8000FFFB47490AA816F03BFC00210AA8F5F77B
:10BD90004BFC0AA816F0F4FB40490AA816F030FC48
:10BDA00000210AA8F5F740FC0AA816F0E9FB3D4976
:10BDB0000AA816F025FC00210AA8F5F735FC0AA808
:10BDC00016F0DEFB35490AA816F01AFC00210AA875
:10BDD000F5F72AFC0AA816F0D3FB33490AA816F097
:10BDE0000FFC00210AA8F5F71FFC0AA816F0C8FBF3
:10BDF0002A490AA816F004FC0AA80021F5F714FC49
:10BE00000AA816F0BDFBB8F1050F0ED8012404FAFC
:10BE100008F818F0240540F0C18518F0120940F028
:10BE2000D48518F0090F40F04186D7F8A430012BD3
:10BE300000F0A3851D490AA816F0E2FB00210AA81C
:10BE4000F5F7F2FB0AA816F09BFB14490AA816F0B6
:10BE5000D7FB00210AA8F5F7E7FB0AA816F090FB2C
:10BE60002CE000BFA815FF1F0AD7233C84A00200C6
:10BE70002408FF1F94A00200A0A00200ACA00200B2
:10BE800068A40200B8A00200DCBA0200C4A002004C
:10BE9000FCA30200141CFF1FF4A00200B08B0200E0
:10BEA00008A102001CA1020030A1020078A102003A
:10BEB0004807FF1FF413FF1FE816FF1FA1490AA838
:10BEC00016F09EFB00210AA8F5F7AEFB0AA816F0B3
:10BED00057FB9D490AA816F093FB00210AA8F5F725
:10BEE000A3FB0AA816F04CFB98490AA816F088FB99
:10BEF00000210AA8F5F798FB0AA816F041FB94491F
:10BF00000AA816F07DFB00210AA8F5F78DFB0AA808
:10BF100016F036FB8F4B3E933EA8FDF787F96DB0C8
:10BF2000BDEC028BBDE8F08F12218B48FC69D7F87D
:10BF300018B08A4D15F006FD0F99894816F0E2F900
:10BF4000874816F08FF9012211460020F4F7A6FD6C
:10BF50001121844815F0F6FC0F99814816F0D2F9AA
:10BF60007F4816F07FF92B680393039A2B6802939E
:10BF7000029B9B1A052BF9D97B4DD7ED057AD5EDA0
:10BF80000A6A3A69FB6886EEA77A03FB02F307EEBA
:10BF9000903AF8EE677A67EE877A17EE900A18F013
:10BFA000F9F9EA686B689FED717A03FB02F308EE1A
:10BFB000103AF8EEC87A814627EE878A8A46FDEE67
:10BFC000C87A0EA817EE901A12F070FBA9680EA896
:10BFD00012F060FB304618F0CBF94A46534618F091
:10BFE0002DFA18F0DBFC01460EA812F09DFB17217C
:10BFF0005F4815F0A7FC0F99594816F083F9584887
:10C0000016F030F935215B4815F09CFC544816F0C9
:10C0100029F90021524816F075F9514816F022F915
:10C020000D21554815F08EFC786918F0B3F941ECF4
:10C03000100B02214A4816F06FF9494816F012F920
:10C040000A214E4815F07EFC00230A223969444833
:10C0500016F018F9424816F005F90B21484815F07A
:10C0600071FC00230A22F9683D4816F00BF93C48A0
:10C0700016F0F8F80921434815F064FCA86A18F096
:10C0800089F941EC100B0221354816F045F9344886
:10C0900016F0E8F806213C4815F054FC4AEC109BD9
:10C0A00002212F4816F038F92D4816F0DBF80A2146
:10C0B000364815F047FC6968294816F023F92848E6
:10C0C00016F0D0F80E21324815F03CFCE9682448FF
:10C0D00016F018F9224816F0C5F80B212D4815F076
:10C0E00031FC18EE100A18F055F941EC100B022142
:10C0F0001B4816F011F91A4816F0B4F80621264824
:10C1000015F020FCA968164800230A2216F0BAF898
:10C11000134816F0A7F8589B6CA903F10B0201EB2A
:10C12000820E01EB830300250EAA43F88C2CB7EE98
:10C13000000A01213EA84EF8B45C5895FFF72AFB8F
:10C14000CDE500BF8CA10200E88D02002C9E02000C
:10C15000C48D0200C487020044A00200141CFF1F0B
:10C160002408FF1F58A00200A815FF1F0AD7233C70
:10C170006CA002000CA0020084A0020094A00200A7
:10C18000A0A00200ACA0020068A40200B8A00200B7
:10C19000DCBA0200C4A00200FCA302000122114686
:10C1A00010463C6BD7F82CB0DFF8E092AA4DF4F7BC
:10C1B00075FC0721A94815F0C5FB00230A22D7F812
:10C1C0009010A74816F05EF8A54816F04BF8D7F87F
:10C1D00090A0BAF1000F40F01C85D5ED0B6AD9EDA7
:10C1E0000A7AD9F82420D9F8203086EEA77A03FB02
:10C1F00002F307EE903AF8EE677A67EE877A17EE69
:10C20000900A18F0C7F8CDE900010D21954815F006
:10C2100099FBD9F8280018F0BDF841EC100B022169
:10C220008F4816F079F88E4816F01CF80A218E48CF
:10C2300015F088FB53460A22D9F82410884816F0D6
:10C2400021F8874816F00EF80B21884815F07AFB84
:10C2500053460A22D9F82010814816F013F8804876
:10C2600016F000F80921824815F06CFBE86A18F016
:10C2700091F841EC100B0221794816F04DF87848FE
:10C2800015F0F0FF06217B4815F05CFB9DED000BDF
:10C290000221734816F040F8714815F0E3FF0A21B7
:10C2A000754815F04FFB29696D4816F02BF86C485E
:10C2B00015F0D8FF0E21714815F044FBA9696848B4
:10C2C00016F020F8664815F0CDFF06216C4815F0F1
:10C2D00039FB5346696962480A2215F0D3FF60486A
:10C2E00015F0C0FFAA692B699FED667A03FB02F384
:10C2F00008EE103AF8EEC87A4FF0000927EE878A68
:10C300001EA8FDEEC87ACDF87C9017EE901A12F0B8
:10C31000CDF9696912F0BEF98246304618F028F866
:10C32000DDE9002318F08AF818F038FB0146504682
:10C3300012F0FAF90D214B4815F004FBB86A18F019
:10C3400029F841EC100B0221454815F0E5FF44485F
:10C3500015F088FF0A21444815F0F4FA4B460A22EA
:10C36000796A3F4815F08EFF3D4815F07BFF0B21A1
:10C370003E4815F0E7FA4B460A22396A384815F06C
:10C3800081FF374815F06EFF0921394815F0DAFAB8
:10C39000E86A17F0FFFF41EC100B0221304815F05E
:10C3A000BBFF2F4815F05EFF0621324815F0CAFA90
:10C3B0009DED000B02212A4815F0AEFF284815F02C
:10C3C00051FF0A212C4815F0BDFA2969244815F0BF
:10C3D00099FF234815F046FF0E21284815F0B2FAC0
:10C3E000A9691F4815F08EFF1D4815F03BFF0B2172
:10C3F000254815F0A7FA18EE100A17F0CBFF41EC0C
:10C40000100B0221164815F087FF154815F02AFF7A
:10C4100006211B4815F096FA4B46696910480A2216
:10C4200015F030FF0E4815F01DFF589BCDF86091B8
:10C430006CA903F10B0201EB820201EB83031EAD39
:10C4400043F88C5CB7EE000A01213EA842F8B49C88
:10C45000FFF7A0F943E400BFA815FF1FD0A002001A
:10C460002408FF1F84A0020094A00200A0A00200E4
:10C47000ACA0020068A40200B8A00200DCBA02006E
:10C48000FCA302000AD7233CC4A00200E815FF1F4A
:10C49000AB4DFC69D7F818B0012211460020F4F723
:10C4A000FDFAD5ED0D6AD7ED057A3A69FB6886EE9F
:10C4B000A77A03FB02F34FF00009CDF83C9007EE9A
:10C4C000903AF8EE677A67EE877A17EE900A17F0DF
:10C4D00061FFEA686B689FED9B7A03FB02F308EE4D
:10C4E000103AF8EEC87A0EAB27EE878ACDE9000144
:10C4F000FDEEC87A184617EE901A12F0D7F8A96820
:10C5000012F0C8F88246304617F032FFDDE900230A
:10C5100017F094FF18F042FA0146504612F004F961
:10C520003521894815F00EFA884815F09BFE032145
:10C53000864815F0E7FE854815F094FE0D218448E5
:10C5400015F000FA786917F025FF41EC100B022175
:10C550007E4815F0E1FE7D4815F084FE0A217D48F5
:10C5600015F0F0F94B460A223969784815F08AFE31
:10C57000764815F077FE0B21774815F0E3F94B4626
:10C580000A22F968714815F07DFE704815F06AFEC0
:10C590000921724815F0D6F9686B17F0FBFE41ECE3
:10C5A000100B0221694815F0B7FE684815F05AFED5
:10C5B00006216B4815F0C6F99DED000B022163487A
:10C5C00015F0AAFE614815F04DFE0A21654815F0E8
:10C5D000B9F969685D4815F095FE5C4815F042FEB2
:10C5E0000E21614815F0AEF9E968584815F08AFE49
:10C5F000564815F037FE0B215C4815F0A3F918EEEC
:10C60000100A17F0C7FE41EC100B02214F4815F03D
:10C6100083FE4E4815F026FE0621554815F092F986
:10C620004B46A96849480A2215F02CFE474815F0E8
:10C6300019FE589BCDF860916CA903F10B0201EB38
:10C64000820201EB83030EAD43F88C5CB7EE000A67
:10C6500001213EA842F8B49CFFF79CF8FFF73FBBCE
:10C660000122114602203C6DD7F84CB0344DF4F74E
:10C6700015FA7B6B95ED0C0A002B40F02883F4F73C
:10C680007DFB10EE100A17F085FECDE900016A6A05
:10C69000EB699FED2C7A03FB02F308EE103AF8EEFB
:10C6A000C87A4FF0000927EE878A2EA8FDEEC87AD7
:10C6B000CDF8BC9017EE901A11F0F8FF296A11F02E
:10C6C000E9FF8246304617F053FEDDE9002317F0FC
:10C6D000B5FE18F063F90146504612F025F80D2119
:10C6E0001B4815F02FF9786C17F054FE41EC100B35
:10C6F0000221164815F010FE144815F0B3FD0A216A
:10C70000144815F01FF94B460A22F96B0F4815F033
:10C71000B9FD0E4815F0A6FD0B210F4815F012F9D2
:10C720004B460A22B96B094815F0ACFD074815F0D5
:10C7300099FD0921094815F005F9286BFFF76EBA34
:10C74000A815FF1F0AD7233C0CA002002408FF1FD6
:10C7500084A0020094A00200A0A00200ACA00200ED
:10C7600068A40200B8A00200DCBA0200C4A0020063
:10C77000FCA302000122114610463C6BD7F82CB0F6
:10C78000DFF82493B04DF4F789F90721AF4815F08D
:10C79000D9F800230A22D7F89010AD4815F072FDA1
:10C7A000AB4815F05FFDD7F89030002B40F0438187
:10C7B000D9ED0A7AD5ED0E6AD9F82420D9F82030BF
:10C7C00086EEA77A03FB02F34FF0000907EE903ADA
:10C7D000F8EE677A67EE877A17EE900A17F0DAFDBF
:10C7E000AA692B699FED9B7ACDF87C9003FB02F33D
:10C7F00008EE103AF8EEC87ACDE9000127EE878AF4
:10C800001EA8FDEEC87A17EE901A11F04FFF696965
:10C8100011F040FF8246304617F0AAFDDDE9002303
:10C8200017F00CFE18F0BAF80146504611F07CFFE4
:10C830000D21894815F086F8B86A17F0ABFD41EC78
:10C84000100B0221824815F067FD814815F00AFDA2
:10C850000A21824815F076F84B460A22796A7C480C
:10C8600015F010FD7A4815F0FDFC0B217C4815F001
:10C8700069F84B460A22396A754815F003FD744879
:10C8800015F0F0FC0921774815F05CF8A86B17F05B
:10C8900081FD41EC100B02216D4815F03DFD6C4807
:10C8A00015F0E0FC0621704815F04CF89DED000BEA
:10C8B0000221674815F030FD654815F0D3FC0A21C8
:10C8C0006A4815F03FF82969614815F01BFD60487A
:10C8D00015F0C8FC0E21664815F034F8A9695C48CB
:10C8E00015F010FD5A4815F0BDFC0B21614815F0FC
:10C8F00029F818EE100A17F04DFD41EC100B02213B
:10C90000534815F009FD524815F0ACFC06215A4871
:10C9100015F018F869694E484B460A2215F0B2FC2A
:10C920004B4815F09FFC012211461046F4F7B6F86B
:10C930007BE53EA8FCF722FC01238BF80030FFF7D3
:10C94000FDB900904D482E2114F0FCFF404815F031
:10C9500089FC41A815F0F4FB009B4698409311F028
:10C96000E3FF479811F0E0FF454B01221A70FFF7F3
:10C97000F2B900902E214348E6E743490AA815F092
:10C980003FFE00210AA8F4F74FFE0AA815F0F8FDB3
:10C990003E49FFF7B5BAAB46FFF7A1B93C4A3D4D5A
:10C9A0002F9B3D48136009212B6014F0CBFF2968B1
:10C9B000274815F0A7FC264815F054FC2246002114
:10C9C0000220F4F76BF8FFF730BA3449314E0AA869
:10C9D00015F016FE29460AA8F4F726FE0AA815F057
:10C9E000CFFD2220F4F79EFF2D4B284693ED000A41
:10C9F000F4F73CFF2B490AA815F002FE29460AA8C5
:10CA0000F4F712FE0AA815F0BBFD214A1F9B22482D
:10CA100013600921336014F095FF31680C4815F05C
:10CA200071FC0B4815F01EFC224629462046F4F7FF
:10CA300035F8FFF7FAB9D9ED277AD5ED0E6AD9F8AE
:10CA40009820D9F89430BBE6A815FF1FD0A00200AB
:10CA50002408FF1F0AD7233C84A0020094A00200F0
:10CA6000A0A00200ACA0020068A40200B8A00200CE
:10CA7000DCBA0200C4A00200FCA30200A0A10200D4
:10CA8000E816FF1FD0A1020064A10200B08B0200D3
:10CA9000F812FF1FB412FF1F58A1020044A10200A8
:10CAA0002019FF1FC48D0200E815FF1F8C498D4C13
:10CAB0008D4E8E4D0AA815F0A3FD49460AA8F4F73D
:10CAC000B3FD0AA815F05CFD2220F4F72BFF884B7C
:10CAD000484693ED000AF4F7C9FE86490AA815F006
:10CAE0008FFD49460AA8F4F79FFD0AA815F048FDF6
:10CAF0000F9B81482360092114F024FF21687F489F
:10CB000015F000FC7D4815F0ADFB7D4B22687A489E
:10CB10001A60092114F016FF2168784815F0F2FB1D
:10CB2000764815F09FFB94ED007A3A69FB68D7EDE3
:10CB3000056A7449F8EEC77A03FB02F327EEA67A7A
:10CB400007EE903AF8EE677A0AA8C7EE276AC6EDB4
:10CB5000006A15F055FD49460AA8F4F765FD0AA8D4
:10CB600015F00EFD2220F4F7DDFE96ED000A484692
:10CB7000F4F77CFE2220F4F7D5FEFF20F4F7D2FE76
:10CB8000FF20F4F7CFFEFF20F4F7CCFE2B680993CB
:10CB9000099A2B680893089B544C9B1A042BF8D9CC
:10CBA00058490AA815F02CFD00210AA8F4F73CFD0D
:10CBB0000AA815F0E5FC2220F4F7B4FE96ED000A71
:10CBC0000020F4F753FE2220F4F7ACFEFF20F4F728
:10CBD000A9FEFF20F4F7A6FEFF20F4F7A3FE2368CA
:10CBE0000793079A2B680693069B9B1A042BF9D987
:10CBF000002108460122F3F751FFFFF716B9F4F7B9
:10CC000057F910EE100A17F0C5FBCDE90001FEF749
:10CC1000AEBFD5ED0B6AD9ED277AD9F89820D9F8AF
:10CC2000943086EEA77A03FB02F307EE903AF8EE13
:10CC3000677A67EE877A17EE900A17F0ABFBCDE9BB
:10CC400000011821304814F07DFE2C4815F00AFB35
:10CC50000D212E4814F076FED9F89C0017F09AFBAF
:10CC600041EC100B0221254815F056FB234815F026
:10CC7000F9FA0A21264814F065FE00230A22D9F8A1
:10CC800098101E4815F0FEFA1C4815F0EBFA0B211F
:10CC9000204814F057FE00230A22D9F894101748B0
:10CCA00015F0F0FA154815F0DDFA09211A4814F0CC
:10CCB00049FEE86A17F06EFB41EC100B02210F48A9
:10CCC00015F02AFB0D4815F0CDFAFFF70BBBF4F772
:10CCD000EFF810EE100A17F05DFBCDE90001D6E485
:10CCE00044A10200B412FF1FBC13FF1F141CFF1F3E
:10CCF0002419FF1FC48D020058A102002408FF1F41
:10CD0000F812FF1FE09D0200D8A0020084A00200DC
:10CD100094A00200A0A00200ACA002002DE9F04FF8
:10CD2000C9B041F28832052106460DF128081AA83B
:10CD3000DFF83890DFF838A0FCF72EFA00244046E0
:10CD400002220321CDF868A0359411F06DFCD9F8CA
:10CD500000300B94013B042B00F24382DFE813F018
:10CD60001D022102250229020A0000BF7015FF1FC3
:10CD7000C4870200C348C44C082114F0E3FD052118
:10CD8000C24814F0DFFDA168C14815F0BBFAC048E5
:10CD900015F068FAA06817F0EBFA41EC100B16F0EA
:10CDA0003BF851EC100B17F0F9FD019006FB00FB6E
:10CDB0000A21B848B84DB94CB94F14F0C3FD3146FB
:10CDC000B348B84E15F09EFAB14815F04BFA0C2155
:10CDD000B54814F0B7FD00230A222968AC4815F0C5
:10CDE00051FAAB4815F03EFA0B21B04814F0AAFDF9
:10CDF000A86817F0CFFA41EC100B0221A44815F0F7
:10CE00008BFAA34815F02EFA0B21A94814F09AFDCD
:10CE100000230A2269689E4815F034FA9C4815F0F0
:10CE200021FA0C21A34814F08DFD00230A22D5F825
:10CE30008410974815F026FA954815F013FA132137
:10CE40009D4814F07FFD00230A22D5F888109048F1
:10CE500015F018FA8E4815F005FA0E21974814F0CF
:10CE600071FD01998A4815F04DFA894815F0FAF9D3
:10CE7000D9F80410404611F019FCD9F80C104046BE
:10CE800011F008FC4046594611F04EFC10218C4828
:10CE900014F058FD59467E4815F034FA7C4815F0D8
:10CEA000E1F9012211460320F3F7F8FD349B48A96C
:10CEB00003F10B0201EB820201EB83034FF0000E42
:10CEC00043F88C8CB7EE000A01211AA842F8B4ECA2
:10CED000CDF8D0E0FEF75EFCDDF87080B8F1000F11
:10CEE00022D023680393039A23680293029B9B1A20
:10CEF000042BF9D9F5F7C6F8002807DB3868F5F7F1
:10CF0000B1F8C0B25328307000F057812368059300
:10CF1000059A23680493049B9B1A092BF9D9DDF821
:10CF20007080B8F1000FDCD16649674E674C06A8E7
:10CF300015F066FB414606A8F4F776FB06A815F047
:10CF40001FFB634906A815F05BFB414606A8F4F7F2
:10CF50006BFB06A815F014FB5E4906A815F050FB04
:10CF6000414606A8F4F760FB06A815F009FB5849EE
:10CF700006A815F045FB414606A8F4F755FB06A8A0
:10CF800015F0FEFA544906A815F03AFB414606A8EA
:10CF9000F4F74AFB06A815F0F3FA4D4906A815F078
:10CFA0002FFB414606A8F4F73FFB06A815F0E8FA68
:10CFB0004A4906A815F024FB414606A8F4F734FBBD
:10CFC00006A815F0DDFA424906A815F019FB4146FE
:10CFD00006A8F4F729FB06A815F0D2FA69682B68B1
:10CFE0000B9A95ED027ADFED3E6A03FB01F307EE43
:10CFF000903A06EE102AF8EE677AB8EEC66A67EE47
:10D00000877A3368374986EE277A0A6006A81A4479
:10D010003549326067EE267AC4ED007A15F0F0FAF1
:10D02000414606A8F4F700FB06A815F0A9FA22204D
:10D03000F4F778FC94ED000A4046F4F717FC2B490E
:10D0400006A815F0DDFA414606A8F4F7EDFA06A8A1
:10D0500015F096FA012241460320F3F71FFDD5F89B
:10D06000A430012B00F0B080214906A815F0C8FAC1
:10D07000414606A8F4F7D8FA06A815F081FA144933
:10D0800006A837E038A202005017FF1F0CA20200CA
:10D090002408FF1F08BD0200E815FF1F141CFF1F16
:10D0A0004807FF1FF413FF1F44A2020054A202000E
:10D0B00060A202006CA202007CA2020090A2020008
:10D0C000A0A20200B4A202006418FF1F9016FF1F66
:10D0D000B08B0200C8A20200DCA20200F0A2020093
:10D0E0000000B4436C15FF1FD09D0200C48D0200E8
:10D0F0001CA3020015F084FA414606A8F4F794FA3E
:10D1000006A815F03DFA394906A815F079FA414606
:10D1100006A8F4F789FA06A815F032FA344906A8E9
:10D1200015F06EFA414606A8F4F77EFA06A815F047
:10D1300027FA304906A815F063FA414606A8F4F725
:10D1400073FA06A815F01CFA2B4906A815F058FA30
:10D15000414606A8F4F768FA06A815F011FA27491F
:10D1600006A815F04DFA002106A8F4F75DFA06A806
:10D1700015F006FA224906A815F042FA002106A881
:10D18000F4F752FA06A815F0FBF91AA8CDF868A032
:10D19000FCF74CF849B0BDE8F08F082119481A4C4B
:10D1A000EBE5082119481A4CE7E5082119481A4C03
:10D1B000E3E5082119481A4CDFE51AA8FBF7DEFF62
:10D1C000184B01221A70A1E6174906A815F018FAA3
:10D1D000414606A8F4F728FA06A815F0D1F908493F
:10D1E000B3E74FF0000BCDF804B0E1E534A3020043
:10D1F000E88D02002C9E0200C48D020048A30200AC
:10D20000B08B020000A20200F016FF1F14A2020061
:10D210000817FF1F20A202002017FF1F2CA20200E8
:10D220003817FF1FE816FF1F04A302002DE9F04F77
:10D23000CC4FDFF88C93BB6CCB4AD9F81C40D9F8A3
:10D2400018602DED028BE5B00025012B05901560CF
:10D2500000F0A485C0F06485022B00F00584A84688
:10D260000395AB4604950195AA46E4B220460121F8
:10D27000F6B212F06DF83046012112F069F841F271
:10D280008832052136A8FBF787FF0025B74B369378
:10D290000222032116A8519511F0C6F95146019AB0
:10D2A000DFF8C0A226A811F0BFF93A683B699FEDEC
:10D2B000B07A03FB02F307EE903AF8EEE77A16A88D
:10D2C00067EE877AFDEEE77A17EE901A11F0EEF925
:10D2D000396A11F0DFF9FB6C1795002B00F0AC8474
:10D2E000012B40F0EA849AED0F6A9FEDA27AD9ED06
:10D2F000027ADAF848009AED0E0ADAF83050C6EEF3
:10D30000076A99E80C0003FB02F3043507EE103AB4
:10D31000B8EE477A9DED056A67EE277AB8EEC68AC1
:10D3200067EEA67A67EE887AFDEEE77ACDED017AB0
:10D33000F3F7EEFDDAF830305B0007EE903AF8EEE6
:10D34000E77A6B0080EE270A029320EE088AFDEE52
:10D35000C87A17EE905A3B218748DFF808A214F0EC
:10D36000F1FA864814F07EFF0D21854814F0EAFAA0
:10D370000199824814F0C6FF804814F073FF112110
:10D38000804814F0DFFA804B7C48196814F0BAFF2B
:10D390007A4814F067FF0A217C4814F0D3FA294632
:10D3A000764814F0AFFF754814F05CFF3B217248DB
:10D3B00014F0C8FA714814F055FF039926A811F02B
:10D3C00075F9414611F066F94FF000080E217048DA
:10D3D000CDF89C8014F0B6FA3968684814F092FFD2
:10D3E000664814F03FFF14216A4814F0ABFA39691B
:10D3F000624814F087FF614814F034FF0D2166483D
:10D4000014F0A0FA43460A22396A5C4814F03AFF45
:10D410005A4814F027FF1321604814F093FA43464A
:10D420000A22D9F80010554814F02CFF534814F084
:10D4300019FF11215A4814F085FA43460A22D9F8F7
:10D4400004104E4814F01EFF4C4814F00BFF12213C
:10D45000544814F077FAD9F8080016F09BFF41EC15
:10D46000100B0221454814F057FF444814F0FAFE0F
:10D47000FB6C002B00F0B183012B2DD110214A4809
:10D4800014F060FADAF83C0016F084FF41EC100B5F
:10D4900002213A4814F040FF384814F0E3FE0F210F
:10D4A000424814F04FFADAF8380016F073FF41ECF6
:10D4B000100B0221314814F02FFF304814F0D2FE37
:10D4C0000C213B4814F03EFADAF830102B4814F0E7
:10D4D00019FF2A4814F0C6FE0D21294814F032FA2B
:10D4E0000199264814F00EFF244814F0BBFE0A21CF
:10D4F000264814F027FA2946204814F003FF1F4855
:10D5000014F0B0FE0B212B4814F01CFA03991B48B1
:10D5100014F0F8FE194814F0A5FE1121264814F065
:10D5200011FA5946154814F0EDFE144814F09AFE0D
:10D530000A21224814F006FA0499104814F0E2FE79
:10D540000E4814F08FFE012203201146F3F7A6FACD
:10D55000B86C012800F0BC83C0F0B48302283CD131
:10D5600030E000BF8014FF1FF812FF1FC4870200C5
:10D570000AD7233C0000B44304A402002408FF1F80
:10D5800040A4020050A40200B412FF1F64A40200D1
:10D5900070A4020080A4020098A4020058AB02000C
:10D5A00078AB020098AB0200E8A40200FCA40200E1
:10D5B0000CA50200D0A30200E0A30200F8A3020021
:10D5C000E815FF1F01221146F3F768FA23212E48C0
:10D5D00014F0B8F92D4814F045FE029B042B40F3DB
:10D5E0008F80DFF8B0804FF0040A0AF0030B0521AA
:10D5F000274814F0A7F95946244814F083FE23481D
:10D6000014F030FEBBF1020F00F08882BBF1030F73
:10D6100000F0B482BBF1010F00F0B082D7F84CB03B
:10D62000BBF1000F00F04184BBF1010F41D1019922
:10D6300016A811F079F8509A64AB02F10B0E03EBC7
:10D640008E0E03EB820216A8002342F88C0C59467A
:10D650004EF8B43CB7EE000A36A85093FEF79AF89D
:10D66000D8F800300993099AD8F800300893089B3D
:10D670009B1A042BF8D9389B2046F3B9029B0AF178
:10D68000010A9A45B1D13BE01CA502002408FF1F06
:10D6900040A50200141CFF1FC14814F053F9C148F3
:10D6A00014F0E0FD002D1DDCF4F7ECFC002800F385
:10D6B0001D82389B2046002BE0D011F04FFE2E211A
:10D6C00083460028E8D0304611F048FE8346002803
:10D6D000EAD12E21B44814F035F9B24814F0C2FD55
:10D6E000002DE1DA39A814F02BFD3E98CDF8E0B01A
:10D6F00011F01AF93F9811F017F9AC4B01221A708A
:10D70000D9F80410D9F800302798179A99ED027AC1
:10D71000DFEDA76AA74CA84EA84D226003FB01F3DA
:10D7200007EE903A06EE102AF8EE677AB8EEC66A6F
:10D7300067EE877A07EE100AB8EEC70A86EE277AF8
:10D7400028609F4D67EE267AC6ED007AF2F700FF5B
:10D750009C4985ED000A12A814F052FF002112A87E
:10D76000F3F762FF12A814F00BFF2220F4F7DAF8A7
:10D7700096ED000A0020F4F779F8934912A814F006
:10D780003FFF002112A8F3F74FFF12A814F0F8FE94
:10D790008E4912A814F034FF002112A8F3F744FFB9
:10D7A00012A814F0EDFE2220F4F7BCF895ED000A63
:10D7B0000020F4F75BF8844912A814F021FF00213F
:10D7C00012A8F3F731FF12A814F0DAFE804912A86C
:10D7D00014F016FF002112A8F3F726FF12A814F088
:10D7E000CFFE7C4912A814F00BFF002112A8F3F71A
:10D7F0001BFF12A814F0C4FE774912A814F000FF12
:10D80000002112A8F3F710FF12A814F0B9FE714915
:10D8100012A814F0F5FE002112A8F3F705FF12A8D4
:10D8200014F0AEFE6D4912A814F0EAFE002112A811
:10D83000F3F7FAFE12A814F0A3FE664912A814F03A
:10D84000DFFE002112A8F3F7EFFE12A814F098FEF5
:10D85000634912A814F0D4FE002112A8F3F7E4FEE5
:10D8600012A814F08DFE5B4912A814F0C9FE002125
:10D8700012A8F3F7D9FE12A814F082FE0821594825
:10D8800014F060F82168474814F03CFD454814F056
:10D89000E9FC0521544814F055F8484B41481968F3
:10D8A00014F030FD3F4814F0DDFC504B22681A6044
:10D8B000002101220320F3F7F1F80021084601229C
:10D8C000F3F7ECF8012210460021F3F7E7F8012204
:10D8D00000210220F3F7E2F8D9F8A430012B00F080
:10D8E0009F82434912A814F08BFE002112A8F3F77F
:10D8F0009BFE12A814F044FE364912A814F080FED4
:10D90000002112A8F3F790FE12A814F039FE39494D
:10D9100012A814F075FE002112A8F3F785FE12A8D4
:10D9200014F02EFE344912A814F06AFE002112A849
:10D93000F3F77AFE12A814F023FE304912A814F06F
:10D940005FFE002112A8F3F76FFE12A814F018FE74
:10D950001D4912A814F054FE002112A8F3F764FE2A
:10D9600012A814F00DFE264912A814F049FE002159
:10D9700012A8F3F759FE12A814F002FE154912A8D6
:10D9800014F03EFE002112A8F3F74EFE12A814F088
:10D99000F7FD1C4912A814F033FE002112A833E051
:10D9A000A0A102002408FF1FD0A10200E816FF1F5B
:10D9B0000000B4436418FF1F9016FF1FB412FF1F2E
:10D9C000BC13FF1FD09D0200C48D0200E09D020029
:10D9D00064A50200B08B020078A502008CA50200AD
:10D9E000A0A502006CA802005CA402006C15FF1F39
:10D9F000DCA50200F0A50200E88D02002C9E0200CA
:10DA000004A6020018A60200F3F70EFE12A814F0F6
:10DA1000B7FDB24912A814F0F3FD002112A8F3F7E4
:10DA200003FE12A814F0ACFDAD4912A814F0E8FDF5
:10DA3000002112A8F3F7F8FD12A814F0A1FDA949DE
:10DA400012A814F0DDFD002112A8F3F7EDFD12A8D5
:10DA500014F096FDA44B369336A8FBF7E7FB65B0B0
:10DA6000BDEC028BBDE8F08FD7F81CB0FB689FEDD2
:10DA7000AB7AD7F82C809D48D9F85040D9F84C6043
:10DA8000CDF8108003FB0BF307EE903AF8EEE77A3F
:10DA90000F2167EE877A4FF0100AFDEEE77ACDEDA1
:10DAA000037A13F04FFFF968914814F02BFC90486B
:10DAB00014F0D8FB15218F4813F044FFF9698C4806
:10DAC00014F020FC8A4814F0CDFB0E218A4813F094
:10DAD00039FF2B460A22F96A854814F0D3FB8448A3
:10DAE00014F0C0FB17230193FFF7BFBB834B1868EB
:10DAF000F4F7B8FA824BC0B2532818707FF4D9AD4E
:10DB00001A21804813F01EFF794814F0ABFB36A8A9
:10DB1000FBF734FB7C4B01221A70F1E5D7F84CB0CF
:10DB2000BBF1000F00F0E481BBF1010F7FF4C1AD48
:10DB3000019B16A8594210F0F7FD509A64AB02F110
:10DB40000B0E03EB8E0E03EB820216A8002342F8A5
:10DB50008C0C59464EF8B43CB7EE000A36A85093E8
:10DB6000FDF718FED8F800301193119AD8F800305C
:10DB70001093109B9B1A042BF8D99AE5D7F84CB058
:10DB8000BBF1000F00F06F81BBF1010F7FF491AD8D
:10DB9000294626A810F0C8FD509A64AB02F10B0E7E
:10DBA00003EB8E0E03EB820226A8002342F88C0CB6
:10DBB00059464EF8B43CB7EE000A36A85093FDF72C
:10DBC000E9FDD8F800300D930D9AD8F800300C9389
:10DBD0000C9B9B1A042BF8D96BE50F214B4813F0D3
:10DBE000B1FEDAF8440016F0D5FB41EC100B02212F
:10DBF0003F4814F091FB3E4814F034FB1C2144488C
:10DC000013F0A0FEDAF8400016F0C4FB41EC100B54
:10DC10000221374814F080FB354814F023FB0D2116
:10DC20003C4813F08FFEDAF83410314814F06AFBE8
:10DC30002F4814F017FB4FE4DAF83420DAED116ABC
:10DC4000DFED355A99ED026A520007EE902AB8EEE0
:10DC5000E77A99E80A0086EE875A03FB01F307EE9C
:10DC6000903AC5EE256A02F108030293B8EE677A8E
:10DC700067EE067A9DED057A67EEA67AB8EEC78A5A
:10DC800067EE887A17EE900A16F084FB41EC100BD1
:10DC900015F0C2F851EC100B16F080FE9AED100A48
:10DCA0000190DAF84800F3F733F928EE000AFDEEA8
:10DCB000C07A17EE905AFFF74EBB082301950293E6
:10DCC000FFF749BB012211460020F2F7E7FE84E48A
:10DCD00002460146F2F7E2FE7FE400BFE88D020053
:10DCE0002C9E0200C48D0200C4870200CCA3020057
:10DCF0002408FF1FDCA30200F4A302004807FF1F53
:10DD0000F413FF1F48A50200E816FF1FA8A4020095
:10DD1000B8A40200D8A402000000B4430AD7233CF0
:10DD2000D7F814B07B681FED037AD7F824808248B7
:10DD3000CDF8108003FB0BF307EE903AF8EEE77A8C
:10DD40000F2167EE877A4FF0060AFDEEE77ACDEDF8
:10DD5000037A13F0F7FD7968784814F0D3FA77481E
:10DD600014F080FA1521764813F0ECFD79697348B8
:10DD700014F0C8FA714814F075FA0E21714813F0C6
:10DD8000E1FD2B460A22796A6C4814F07BFA6B4855
:10DD900014F068FA05230193FFF767BAD7F818B0B3
:10DDA000BB689FED697AD7F828806848D9F8304079
:10DDB000D9F82C60CDF8108003FB0BF307EE903AF6
:10DDC000F8EEE77A0F2167EE877A4FF0150AFDEE3D
:10DDD000E77ACDED037A13F0B5FDB968574814F032
:10DDE00091FA564814F03EFA1521594813F0AAFD4D
:10DDF000B969524814F086FA504814F033FA0E21EB
:10DE0000544813F09FFD2B460A22B96A4B4814F080
:10DE100039FA4A4814F026FA14230193FFF725BA79
:10DE20004D4912A814F0ECFB002112A8F3F7FCFBFB
:10DE300012A814F0A5FB494912A814F0E1FB002137
:10DE400012A8F3F7F1FB12A814F09AFB444912A8A8
:10DE500014F0D6FB002112A8F3F7E6FB12A814F089
:10DE60008FFB3E49ECE5019916A810F05DFC509A35
:10DE7000CDF840B164AB03EB8200024616AB40F82C
:10DE80008C3CB7EE000A42F888BC012136A8FDF7A9
:10DE900081FCD8F800300B930B9AD8F800300A9325
:10DEA0000A9B9B1A042BF8D903E4294626A810F0F4
:10DEB0003BFC509ACDF840B164AB03EB82000246C4
:10DEC00026AB40F88C3CB7EE000A42F888BC012132
:10DED00036A8FDF75FFCD8F800300793079AD8F80A
:10DEE00000300693069B9B1A042BF8D9FFF7E1BB81
:10DEF000694226A810F018FC509ACDF840B164ABE6
:10DF000003EB8200024626AB40F88C3CB7EE000AD9
:10DF100042F888BC012136A8FDF73CFCD8F8003057
:10DF20000F930F9AD8F800300E930E9B9B1A042B78
:10DF3000F8D9FFF7BEBB00BF5CA302002408FF1F97
:10DF40006CA3020084A302000AD7233C94A302001E
:10DF5000A4A30200BCA30200B4A50200B08B02007F
:10DF6000C8A502002DE9F04F2DED088BCBB0D14CA8
:10DF7000DFF8A0930090884608A8CF49F0EE408AC9
:10DF8000B0EE60BA14F03CFBE569A669D9F8007000
:10DF9000B8F1000F07D1012F00F0A082C0F01D8260
:10DFA000022F00F01A823021C44813F0CBFC39460E
:10DFB000C34814F0A7F9C24814F054F91721C14816
:10DFC00013F0C0FC18EE900A16F0E4F941EC1A0BBD
:10DFD0000221B0EE4A0AF0EE6A0AB94814F09CF940
:10DFE000B74814F03FF91521B74813F0ABFC1BEE0E
:10DFF000100A16F0CFF941EC190B0221B0EE490AD4
:10E00000F0EE690AAE4814F087F9AD4814F02AF929
:10E010001421AE4813F096FC0099A94814F072F947
:10E02000A74814F01FF91921A94813F08BFC4146A9
:10E03000A34814F067F9A24814F014F9012F00F076
:10E040002F82022F00F00E82002F00F0A8814FF0E7
:10E05000000908EE109A4B46CDF81090CDF80C90C0
:10E06000CDF80890CB46EDB228460121F6B20593D3
:10E0700011F06EF93046012111F06AF9B8EEC88A44
:10E08000DFED947A944C68EE277A0DF1300AFDEEBC
:10E09000E77A41F2883205211CA8CDED017AFBF721
:10E0A0007BF88E4B029A1C93594650464FF0000B5A
:10E0B000CDF8DCB010F0B8FADDED007A68EE8B8AAE
:10E0C000F8EEE77A68EEA77A17EE900A16F062F992
:10E0D00041EC100B14F0A0FE51EC100B16F0A6FC56
:10E0E000019908EE100A504610F0E0FA494610F087
:10E0F000D1FAFDEEC87A17EE901A10F015FB032145
:10E100007748CDF834B013F01DFC08A96C4814F022
:10E1100083F81921734813F015FC08A9684814F016
:10E120007BF803216E4813F00DFC654814F09AF853
:10E130000E216D4813F006FCB0EE4A0AF0EE6A0AB2
:10E1400002215F4814F0E8F85D4814F08BF80C21C8
:10E15000664813F0F7FBB0EE490AF0EE690A0221B7
:10E16000574814F0D9F8564814F07CF80B21604851
:10E1700013F0E8FB0099524814F0C4F8504814F02A
:10E1800071F80D215B4813F0DDFB18EE100A16F054
:10E1900001F941EC100B0221494814F0BDF8484840
:10E1A00014F060F80D21544813F0CCFB0199444859
:10E1B00014F0A8F8424814F055F80A214F4813F01B
:10E1C000C1FB03993E4814F09DF83D4814F04AF80D
:10E1D0000E214B4813F0B6FB0499394814F092F81D
:10E1E000374814F03FF81121464813F0ABFB059B6C
:10E1F0003348194614F086F8314814F033F80321F7
:10E20000414813F09FFB08A92D4814F005F8192187
:10E21000344813F097FB08A9294813F0FDFF0321A8
:10E22000394813F08FFB264814F01CF8369BCDF8C4
:10E23000D8B04AA903F10B0201EB820201EB830380
:10E240001CA8012143F88CACB7EE000A42F8B4BC1C
:10E25000FDF7A0FA1E99002900F0E280284611F08F
:10E260007DF8002840F0C6802921284813F06AFB79
:10E27000134813F0F7FF1FA813F062FF002424983F
:10E280001E9410F051FB259810F04EFB0125204BF9
:10E2900021462A4603201D70F2F700FC2A4621463B
:10E2A0002046F2F7FBFB2A4621462846F2F7F6FB0A
:10E2B00032E000BFE815FF1FB0A2020054A6020022
:10E2C0002408FF1F88A60200A0A60200B8A602002C
:10E2D000D0A602000AD7233C141CFF1FC4870200EB
:10E2E0003CA40200ECA6020008A7020018A7020046
:10E2F00028A7020068AC020034A702000C9F0200AD
:10E3000044A7020054A7020028AF0200B4A70200ED
:10E31000E816FF1F0814FF1F2A4621460220F2F7C5
:10E32000BDFB754D7548112113F00CFB296874482D
:10E3300013F0E8FF724813F095FFB8F1000F03D017
:10E340002A680D9B13442B6011216C4813F0FAFAD4
:10E3500029686B4813F0D6FF694813F083FF1A2130
:10E36000684813F0EFFA3946654813F0CBFF64486C
:10E3700013F078FF1721644813F0E4FA604813F0B3
:10E3800071FF624B1C931CA8FAF750FF08A814F009
:10E39000F7F820464BB0BDEC088BBDE8F08F5C4928
:10E3A00008A814F0B5F9012211463846E569A669B6
:10E3B000F2F774FBD9F8343003931A46D9F8443095
:10E3C000D9F85490CDF8109003FB02F208EE102A11
:10E3D000052202924FF0060B45E610214D4813F03E
:10E3E000B1FA0121464813F08DFF454813F03AFF7A
:10E3F0000127D8E5304610F0B1FF00283FF434AFD4
:10E40000F3F776FE70B923680793079A236806939B
:10E41000069B9B1A042BF9D91E9900297FF41EAF85
:10E420000C467EE717213C4813F08CFA344813F071
:10E4300019FF1CA8FAF7A2FE012200210320F2F71F
:10E440002DFB002108460122F2F728FB012210468D
:10E450000021F2F723FB012200210220F2F71EFB2C
:10E4600001245EE72D4908A814F052F90122114653
:10E470003846256DE66CF2F711FBD9F83C30039372
:10E480001A46D9F84C30D9F85C90CDF8109003FBBF
:10E4900002F208EE102A172202924FF0100BE2E56A
:10E4A0001F4908A814F034F93A4639463846256B16
:10E4B000E66AF2F7F3FAD9F8383003931A46D9F836
:10E4C0004830D9F85890CDF8109003FB02F208EECE
:10E4D000102A142202924FF0150BC4E510211148A6
:10E4E00013F030FA4146064813F00CFF044813F0CD
:10E4F000B9FE474657E500BFB412FF1F50A4020003
:10E500002408FF1F80A702009CA70200C487020006
:10E51000049B02002CA6020068A70200CC9B02000C
:10E5200078C6020040A602002DE9F0412DED068BD1
:10E53000C2B0322101909448944EDFF888829FED5A
:10E54000948A944FB0EE409AF0EE608A13F0FAF994
:10E55000914813F087FE012211460320F2F79EFA3C
:10E5600004AC41F28832052114A8FAF715FE002503
:10E57000204602220321CDF850802F9510F054F848
:10E58000326B336C03FB02F307EE903AF8EEE77A56
:10E59000204667EE887AFDEEE77A17EE901A10F0C3
:10E5A00085F8316D10F076F8326B336C7B4E03FBDF
:10E5B00002F307EE903AF8EEE77A204667EE887AA3
:10E5C000FDEEE77A17EE901A10F070F8DDED017AA3
:10E5D000059529EE287AF8EEE77A67EE277A17EEA6
:10E5E000900A15F0D7FE41EC100B14F015FC51EC1D
:10E5F000100B16F01BFA08EE100A1321684813F0EE
:10E60000A1F918EE100A15F0C5FE41EC1A0B022113
:10E61000B0EE4A0AF0EE6A0A5F4813F07DFE5E48EB
:10E6200013F020FE0C215F4813F08CF9B0EE4A0A7B
:10E63000F0EE6A0A0221584813F06EFE564813F0B5
:10E6400011FE0F21584813F07DF919EE100A15F04C
:10E65000A1FE41EC100B02214F4813F05DFE4E4825
:10E6600013F000FE0B21514813F06CF918EE900ADC
:10E6700015F090FE41EC100B0221474813F04CFEC0
:10E68000454813F0EFFD0A21494813F05BF9019961
:10E69000414813F037FE404813F0E4FDFDEEC87A20
:10E6A000204617EE901A10F03FF82E9B2E9542AAA6
:10E6B00002EB830242A90B3301EB830342F88C4C3B
:10E6C000B7EE000A43F8B45C14A80121FDF762F824
:10E6D000169B384CB3B1F3F7D5FC002806DB38683D
:10E6E000F3F7C0FCC0B25328307038D023680393CE
:10E6F000039A23680293029B9B1A042BF9D9169B59
:10E70000002BE8D12C4C2D48142113F01BF9216863
:10E71000214813F0F7FD204813F0A4FD2268059B63
:10E72000264813441421236013F00CF921681A4879
:10E7300013F0E8FD184813F095FD3121204813F03F
:10E7400001F9154813F08EFD14A8CDF85080FAF7A2
:10E750006DFD284642B0BDEC068BBDE8F08114A8E3
:10E76000FAF70CFD012200210320F2F797F90021AE
:10E7700008460122F2F792F9012210460021F2F731
:10E780008DF90125B2E700BFE0A702000814FF1FC2
:10E790000AD7233C4807FF1F2408FF1FF413FF1F5D
:10E7A00014A8020028A8020038A8020048A8020005
:10E7B00054A80200141CFF1F6418FF1F60A8020069
:10E7C00078A80200C48702002DE9F04FDFF86083CB
:10E7D000D8F81430012B14BF0820042087B0F2F7BA
:10E7E000D9FDD8F81030002B40F39281CB4CCC4DA2
:10E7F000A146AA460126CB4902A813F001FF002139
:10E8000002A8F2F711FF02A813F0BAFE2220F3F7D4
:10E8100089F807EE906A0020B8EEE70AF3F726F8C9
:10E82000C14902A813F0ECFE002102A8F2F7FCFE99
:10E8300002A813F0A5FED8F81430002B00F07A815E
:10E84000012B40F05F81B94F2068D7ED007A01932A
:10E85000F0EE080AB8EEE70AFFF766FE8346F3F724
:10E8600047FC002840F05481019BBBF1000F40F0B1
:10E870004F81D5ED007AD9F8000001931946B8EE22
:10E88000E70AF0EE000A4042FFF76CFB8346F3F71D
:10E890002FFC019B002840F03B81BBF1000F40F0B2
:10E8A0003781D7ED007AD9F800000193B8EEE70A76
:10E8B000F7EE000A4042FFF737FE8346F3F718FCF5
:10E8C000019B002840F02481BBF1000F40F0208123
:10E8D000DAED007AD9F800001946B8EEE70AF7EE4B
:10E8E000000AFFF73FFB8346F3F702FC002840F0E5
:10E8F0000F81BBF1000F40F00B812068D7ED007A4B
:10E900004042B8EEE70AF7EE000AFFF70DFE834635
:10E91000F3F7EEFB002840F0FB80BBF1000F40F066
:10E92000F7802068D5ED007A4042B8EEE70A012171
:10E93000F0EE000AFFF716FB8346F3F7D9FB002839
:10E9400040F0E680BBF1000F40F0E280774B20689A
:10E9500093ED000AF0EE080AB8EEC00AFFF7E4FDF6
:10E960008346F3F7C5FB002840F0D280BBF1000FCF
:10E9700040F0CE80D5ED007A2068B8EEE70A01219C
:10E98000F1EE000AFFF7EEFA8346F3F7B1FB002839
:10E9900040F0BE80BBF1000F40F0BA802068D5ED9A
:10E9A000007A4042B8EEE70A0121F2EE000AFFF7D2
:10E9B000D9FA8346F3F79CFB002840F0A980BBF10D
:10E9C000000F40F0A5802068D7ED007A4042B8EEF5
:10E9D000E70AF0EE080AFFF7A7FD8346F3F788FB86
:10E9E000002840F09580BBF1000F40F09180D5EDFC
:10E9F000007A2068B8EEE70A0121F0EE000AFFF77E
:10EA0000B1FA8346F3F774FB002840F08180BBF134
:10EA1000000F7DD1454B20681B68019307EE903AAB
:10EA2000F7EE000AB8EEE70AFFF77EFD8346F3F73C
:10EA30005FFB00286CD1BBF1000F69D12068D5EDD8
:10EA4000007A4042B8EEE70A0121F7EE000AFFF72C
:10EA500089FA8346F3F74CFB002859D1BBF1000F2C
:10EA600056D1324B206893ED000AF7EE000AB8EE5B
:10EA7000C00AFFF759FD8346F3F73AFB002847D158
:10EA8000BBF1000F44D1D5ED007A2068B8EEE70A5B
:10EA90000121F0EE000AFFF765FA8346F3F728FB41
:10EAA000B0BBBBF1000F33D197ED000A2068B8EE80
:10EAB000C00A4042F0EE080AFFF736FD0746F3F7BA
:10EAC00017FB28BB27BBD5ED007A2068B8EEE70A14
:10EAD0000121F1EE000AFFF745FA0746F3F708FBBC
:10EAE000B0B9AFB92068D5ED007A4042B8EEE70A78
:10EAF0000121F2EE000AFFF735FA0746F3F7F8FABC
:10EB000030B92FB9D8F810300136B342BFF673AE22
:10EB1000F2F7AEFD07B0BDE8F08F00BF4007FF1F62
:10EB20001C13FF1FF4930200C48D02008015FF1F09
:10EB30000814FF1FD5ED007A2068B8EEE70A01211E
:10EB4000F0EE080AFFF70EFA0746F3F7D1FA0028AD
:10EB5000DED1002FDCD1AB4FD9F80000D7ED007A21
:10EB60004042B8EEE70AF0EE000AFFF7DDFC83460C
:10EB7000F3F7BEFA0028CBD1BBF1000FC8D1D9F80A
:10EB80000000DAED007A4042B8EEE70A0121F7EE24
:10EB9000000AFFF7E7F98346F3F7AAFA0028B7D18E
:10EBA000BBF1000FB4D1D7ED007AD9F80000B8EE70
:10EBB000E70AF7EE000AFFF7B7FC8346F3F798FA87
:10EBC0000028A5D1BBF1000FA2D1D9F80000DAEDE1
:10EBD000007A4042B8EEE70A0121F7EE000AFFF79B
:10EBE000C1F98346F3F784FA002891D1BBF1000FF5
:10EBF0008ED12068D7ED007A4042B8EEE70AF0EEF9
:10EC0000000AFFF791FC8346F3F772FA00287FF4BD
:10EC10007FAFBBF1000F7FF47BAFD5ED007A2068AA
:10EC2000B8EEE70A0121F0EE080AFFF79BF98346E8
:10EC3000F3F75EFA00287FF46BAFBBF1000F7FF4AF
:10EC400067AF704B20681B68019307EE903AF1EEB6
:10EC5000000AB8EEE70AFFF767FC8346F3F748FAC5
:10EC600000287FF455AFBBF1000F7FF451AF654B27
:10EC7000206893ED000A4042B8EEC00AF2EE000AA6
:10EC8000FFF752FC8346F3F733FA00287FF440AFD6
:10EC9000BBF1000F7FF43CAF2068D5ED007A404215
:10ECA000B8EEE70A0121F0EE080AFFF75BF98346A8
:10ECB000F3F71EFA00287FF42BAFBBF1000F7FF4AF
:10ECC00027AFD7ED007A2068B8EEE70AF0EE000A29
:10ECD000FFF72AFC8346F3F70BFA00287FF418AFFE
:10ECE000BBF1000F7FF414AFD5ED007A2068B8EEC9
:10ECF000E70A0121F7EE000AFFF734F98346F3F73C
:10ED0000F7F900287FF404AFBBF1000F7FF400AFE8
:10ED10003C4B20681B68019307EE903A4042B8EEE6
:10ED2000E70AF7EE000AFFF7FFFB8346F3F7E0F987
:10ED300000287FF4EDAEBBF1000F7FF4E9AED5ED16
:10ED4000007A2068B8EEE70A0121F7EE000AFFF723
:10ED500009F98346F3F7CCF900287FF4D9AEBBF16B
:10ED6000000F7FF4D5AE274B206893ED000AF0EE3C
:10ED7000000AB8EEC00AFFF7D7FB8346F3F7B8F9ED
:10ED800000287FF4C5AEBBF1000F7FF4C1AE206850
:10ED9000D5ED007A4042B8EEE70A0121F0EE080A0C
:10EDA000FFF7E0F88346F3F7A3F900287FF4B0AE4D
:10EDB000BBF1000F7FF4ACAE97ED000A2068114F55
:10EDC000B8EEC00AF1EE000AFFF7AEFB8346F3F798
:10EDD0008FF900287FF49CAEBBF1000F7FF498AE52
:10EDE00097ED000A2068B8EEC00A4042F2EE000A31
:10EDF000FFF79AFB0746F3F77BF900283FF481AE53
:10EE000086E600BF8015FF1F2DE9F04FDFF8A883CD
:10EE1000D8F81430012B14BF0D20042087B0F2F76E
:10EE2000B9FAD8F81030002B40F3B382DD4CDE4D38
:10EE3000A146AA460127DD4902A813F0E1FB002103
:10EE400002A8F2F7F1FB02A813F09AFB2220F2F7D6
:10EE500069FD07EE907A0020B8EEE70AF2F706FDAA
:10EE6000D34902A813F0CCFB002102A8F2F7DCFB87
:10EE700002A813F085FBD8F81430002B00F0908224
:10EE8000012B40F08082CB4E2068D6ED007A0193B2
:10EE90004042B8EEE70A1946F7EE000AFFF762F8BB
:10EEA0008346F3F725F9002840F07382019BBBF1FC
:10EEB000000F40F06E82D5ED007AD9F80000019382
:10EEC000B8EEE70AF0EE080AFFF72EFB8346F3F7E9
:10EED0000FF9019B002840F05C82BBF1000F40F06D
:10EEE0005882D9F80000D6ED007A19464042B8EEB3
:10EEF000E70AF0EE000AFFF735F88346F3F7F8F873
:10EF0000002840F04682BBF1000F40F04282D9F861
:10EF10000000DAED007A4042B8EEE70AF7EE000AA8
:10EF2000FFF702FB8346F3F7E3F8002840F0318255
:10EF3000BBF1000F40F02D82D6ED007A2068B8EECC
:10EF4000E70A0121F7EE000AFFF70CF88346F3F712
:10EF5000CFF8002840F01D82BBF1000F40F019826D
:10EF60002068D5ED007A4042B8EEE70AF7EE000AD5
:10EF7000FFF7DAFA8346F3F7BBF8002840F009827E
:10EF8000BBF1000F40F005828A4B20681B6801939B
:10EF900007EE903A4042B8EEE70A0121F0EE080A87
:10EFA000FEF7E0FF8346F3F7A3F8002840F0F18175
:10EFB000BBF1000F40F0ED81D5ED007A2068B8EE8E
:10EFC000E70AF7EE000AFFF7AFFA8346F3F790F887
:10EFD000002840F0DE81BBF1000F40F0DA81754B74
:10EFE000206893ED000A0121B8EEC00AF7EE000A8E
:10EFF000FEF7B8FF8346F3F77BF8002840F0C9819D
:10F00000BBF1000F40F0C581D5ED007A2068B8EE65
:10F01000E70AF7EE000AFFF787FA8346F3F768F886
:10F02000002840F0B681BBF1000F40F0B2812068AB
:10F03000D6ED007A4042B8EEE70A0121F0EE000A70
:10F04000FEF790FF8346F3F753F8002840F0A181C4
:10F05000BBF1000F40F09D812068D5ED007A404261
:10F06000B8EEE70AF0EE080AFFF75EFA8346F3F718
:10F070003FF8002840F08D81BBF1000F40F08981FE
:10F080004C4B206893ED000A0121B8EEC00AF1EE66
:10F09000080AFEF767FF8346F3F72AF8002840F0D6
:10F0A0007881BBF1000F40F07481D5ED007A2068C3
:10F0B000B8EEE70AF1EE000AFFF736FA8346F3F7F7
:10F0C00017F8002840F06581BBF1000F40F0618126
:10F0D0002068D6ED007A4042B8EEE70A0121F1EE51
:10F0E0000C0AFEF73FFF8346F3F702F8002840F0D2
:10F0F0005081BBF1000F40F04C812068D5ED007AC3
:10F100004042B8EEE70AF0EE080AFFF70DFA834630
:10F11000F2F7EEFF002840F03C81BBF1000F40F019
:10F120003881244B20681B68019307EE903A4042D7
:10F13000B8EEE70A0121F0EE000AFEF713FF83465E
:10F14000F2F7D6FF002840F02481BBF1000F40F019
:10F150002081D5ED007A2068B8EEE70AF7EE000AC4
:10F16000FFF7E2F98346F2F7C3FF002840F0118170
:10F17000BBF1000F40F00D810E4B206893ED000AAB
:10F180000121B8EEC00AF7EE000AFEF7EBFE834657
:10F19000F2F7AEFF002840F0FC80BBF1000F40F01A
:10F1A000F8800BE04007FF1F8015FF1FF49302005B
:10F1B000C48D02001C13FF1F0814FF1FD5ED007A39
:10F1C0002068B8EEE70AF7EE000AFFF7ADF98346CC
:10F1D000F2F78EFF002840F0DC80BBF1000F40F01A
:10F1E000D8802068D6ED007A4042B8EEE70A0121C7
:10F1F000F0EE080AFEF7B6FE8346F2F779FF002824
:10F2000040F0C780BBF1000F40F0C3802068D5ED0F
:10F21000007A4042B8EEE70AF7EE000AFFF784F9F9
:10F220008346F2F765FF002840F0B380BBF1000F82
:10F2300040F0AF80594B206893ED000A0121B8EEF1
:10F24000C00AF7EE000AFEF78DFE8346F2F750FF84
:10F25000002840F09E80BBF1000F40F09A802068AB
:10F26000D5ED007A4042B8EEE70AF7EE000AFFF764
:10F270005BF98346F2F73CFF002840F08A80BBF13F
:10F28000000F40F086802068D6ED007A4042B8EE4C
:10F29000E70A0121F0EE000AFEF764FE8346F2F76A
:10F2A00027FF002875D1BBF1000F72D1D5ED007A90
:10F2B0002068B8EEE70AF0EE080AFFF735F9834652
:10F2C000F2F716FF002864D1BBF1000F61D1334B78
:10F2D00020681B68019307EE903A0121B8EEE70A17
:10F2E000F1EE040AFEF73EFE8346F2F701FF002826
:10F2F0004FD1BBF1000F4CD1284B206893ED000A91
:10F300004042B8EEC00A0121F1EE080AFEF72AFEDB
:10F310008346F2F7EDFE00283BD1BBF1000F38D158
:10F320002068D5ED007A4042B8EEE70AF1EE000A17
:10F33000FFF7FAF88346F2F7DBFE50BBBBF1000F94
:10F3400027D196ED000A2068144EB8EEC00A0121BC
:10F35000F1EE0C0AFEF706FE8346F2F7C9FEC0B9CD
:10F36000BBF1000F15D196ED000A2068B8EEC00A77
:10F3700040420121F1EE0C0AFEF7F4FD0646F2F7D9
:10F38000B7FE30B92EB9D8F810300137BB42BFF6FE
:10F3900052ADF2F76DF907B0BDE8F08F1C13FF1FF7
:10F3A0002068D5ED007A4042B8EEE70AF7EE000A91
:10F3B000FFF7BAF80646F2F79BFE0028E9D1002EC7
:10F3C000E7D1DF4ED9F80000D6ED007AF0EE080A5A
:10F3D000B8EEE70A0121FEF7C5FD8346F2F788FE85
:10F3E0000028D6D1BBF1000FD3D1D9F80000DAED57
:10F3F000007A4042B8EEE70AF0EE000AFFF794F810
:10F400008346F2F775FE0028C3D1BBF1000FC0D1CF
:10F41000D9F80000D6ED007A4042B8EEE70A0121A3
:10F42000F7EE000AFEF79EFD8346F2F761FE002824
:10F43000AFD1BBF1000FACD1DAED007AD9F8000002
:10F44000B8EEE70AF7EE000AFFF76EF88346F2F728
:10F450004FFE00289DD1BBF1000F9AD12068D6ED58
:10F46000007A4042B8EEE70A0121F7EE000AFEF703
:10F4700079FD8346F2F73CFE00288AD1BBF1000FEC
:10F4800087D12068D5ED007A4042B8EEE70AF0EE69
:10F49000080AFFF749F88346F2F72AFE00287FF4AE
:10F4A00078AFBBF1000F7FF474AFA54B20681B68E9
:10F4B000019307EE903A0121B8EEE70AF7EE000A51
:10F4C000FEF750FD8346F2F713FE00287FF461AF8C
:10F4D000BBF1000F7FF45DAFD5ED007A2068B8EE88
:10F4E000E70AF7EE000AFFF71FF88346F2F700FE7F
:10F4F00000287FF44EAFBBF1000F7FF44AAF904B72
:10F50000206893ED000A0121B8EEC00AF7EE000A68
:10F51000FEF728FD8346F2F7EBFD00287FF439AFB4
:10F52000BBF1000F7FF435AF2068D5ED007A404283
:10F53000B8EEE70AF0EE000AFEF7F6FF8346F2F7B0
:10F54000D7FD00287FF425AFBBF1000F7FF421AF7A
:10F550002068D6ED007A4042B8EEE70A0121F0EECD
:10F56000080AFEF7FFFC8346F2F7C2FD00287FF48D
:10F5700010AFBBF1000F7FF40CAFD5ED007A20681F
:10F58000B8EEE70AF1EE080AFEF7CEFF8346F2F77F
:10F59000AFFD00287FF4FDAEBBF1000F7FF4F9AEA4
:10F5A000674B206893ED000A0121B8EEC00AF1EE26
:10F5B000000AFEF7D7FC8346F2F79AFD00287FF495
:10F5C000E8AEBBF1000F7FF4E4AE2068D5ED007A21
:10F5D0004042B8EEE70AF1EE0C0AFEF7A5FF8346BB
:10F5E000F2F786FD00287FF4D4AEBBF1000F7FF464
:10F5F000D0AE2068D6ED007A4042B8EEE70A01218D
:10F60000F0EE080AFEF7AEFC8346F2F771FD002823
:10F610007FF4BFAEBBF1000F7FF4BBAE2068D5ED29
:10F62000007A4042B8EEE70AF0EE000AFEF77CFFEF
:10F630008346F2F75DFD00287FF4ABAEBBF1000F0F
:10F640007FF4A7AE3E4B20681B68019307EE903A0B
:10F650000121B8EEE70AF7EE000AFEF783FC8346C5
:10F66000F2F746FD00287FF494AEBBF1000F7FF463
:10F6700090AED5ED007A2068B8EEE70AF7EE000A02
:10F68000FEF752FF8346F2F733FD00287FF481AE88
:10F69000BBF1000F7FF47DAE294B206893ED000A8B
:10F6A0000121B8EEC00AF7EE000AFEF75BFC8346C4
:10F6B000F2F71EFD00287FF46CAEBBF1000F7FF463
:10F6C00068AE2068D5ED007A4042B8EEE70AF0EE69
:10F6D000080AFEF729FF8346F2F70AFD00287FF4A7
:10F6E00058AEBBF1000F7FF454AE2068D6ED007A1F
:10F6F0004042B8EEE70A0121F7EE000AFEF732FCBD
:10F700008346F2F7F5FC00287FF443AEBBF1000F0F
:10F710007FF43FAED5ED007A2068B8EEE70AF7EE49
:10F72000000AFEF701FF8346F2F7E2FC00287FF4AF
:10F7300030AEBBF1000F7FF42CAE014B206801E02E
:10F740001C13FF1F93ED000A4042B8EEC00A0121CE
:10F75000F7EE000AFEF706FC8346F2F7C9FC002824
:10F760007FF417AEBBF1000F7FF413AE2068D5ED28
:10F77000007A4042B8EEE70AF0EE000AFEF7D4FE47
:10F780008346F2F7B5FC00287FF403AEBBF1000F0F
:10F790007FF4FFAD96ED000A2068384EB8EEC00A3F
:10F7A0000121F0EE080AFEF7DDFB8346F2F7A0FC2C
:10F7B00000287FF4EEADBBF1000F7FF4EAADD5ED8C
:10F7C000007A2068B8EEE70AF1EE040AFEF7ACFE14
:10F7D0008346F2F78DFC00287FF4DBADBBF1000F10
:10F7E0007FF4D7AD2068D5ED007A4042B8EEE70A45
:10F7F000F1EE080AFEF798FE8346F2F779FC00283E
:10F800007FF4C7ADBBF1000F7FF4C3AD96ED000AE6
:10F810002068B8EEC00A40420121F1EE000AFEF76E
:10F82000A1FB0646F2F764FC00287FF4B2AD002E7F
:10F830007FF4AFADD5ED007A2068B8EEE70AF1EEBF
:10F840000C0AFEF771FE0646F2F752FC00287FF420
:10F85000A0AD002E7FF49DAD2068D5ED007A40422A
:10F86000B8EEE70AF1EE0C0AFEF75EFE0646F2F786
:10F870003FFC00283FF486AD8BE500BF1C13FF1F43
:10F880002DE9F04FDFF8F082D8F81430012B14BFC7
:10F890000420032087B0F1F77DFDD8F81030002B4D
:10F8A00040F3C680B04DDFF8D4922F46CA460124FB
:10F8B000AE4902A812F0A4FE002102A8F1F7B4FE9E
:10F8C00002A812F05DFE2220F2F72CF807EE904A13
:10F8D0000020B8EEE70AF1F7C9FFA54902A812F027
:10F8E0008FFE002102A8F1F79FFE02A812F048FE49
:10F8F000D8F81430002B00F0A080012B40F092804B
:10F900009C4E2868D6ED007A0193F0EE080AB8EE16
:10F91000E70AFEF709FE8346F2F7EAFB002840F00B
:10F920008780019BBBF1000F40F08280D9ED007A07
:10F93000386801931946B8EEE70AF0EE080A40422B
:10F94000FEF710FB8346F2F7D3FB019B00286FD133
:10F95000BBF1000F6CD1D6ED007A38680193B8EE98
:10F96000E70AF0EE000A4042FEF7DEFD8346F2F7BA
:10F97000BFFB019B00285BD1BBF1000F58D1DAED32
:10F98000007A38681946B8EEE70AF7EE000AFEF783
:10F99000E9FA8346F2F7ACFB002849D1BBF1000F2E
:10F9A00046D196ED000A2868724EB8EEC00AF7EE0E
:10F9B000000AFEF7B9FD8346F2F79AFBC0BBBBF124
:10F9C000000F35D1D9ED007A2868B8EEE70A012199
:10F9D000F7EE000AFEF7C6FA8346F2F789FB38BB5A
:10F9E000BBF1000F24D196ED000A2868B8EEC00ADA
:10F9F0004042F0EE000AFEF797FD0646F2F778FB6C
:10FA0000B0B9AEB92868D9ED007A4042B8EEE70A3D
:10FA10000121F0EE080AFEF7A5FA0646F2F768FBA8
:10FA200030B92EB9D8F810300134A342BFF640AF38
:10FA3000F1F71EFE07B0BDE8F08FD9ED007A286817
:10FA4000B8EEE70A0121F0EE080AFEF78BFA064647
:10FA5000F2F74EFB0028EBD1002EE9D1454E386875
:10FA6000D6ED007A4042B8EEE70AF0EE080AFEF75B
:10FA70005BFD8346F2F73CFB0028D9D1BBF1000FB8
:10FA8000D6D13868DAED007A4042B8EEE70A0121B3
:10FA9000F0EE000AFEF766FA8346F2F729FB00282B
:10FAA000C6D1BBF1000FC3D1D6ED007A3868B8EEED
:10FAB000E70AF7EE000AFEF737FD8346F2F718FB78
:10FAC0000028B5D1BBF1000FB2D1DAED007A386869
:10FAD000B8EEE70A0121F7EE000AFEF743FA834683
:10FAE000F2F706FB0028A3D1BBF1000FA0D196EDE1
:10FAF000000A28681F4EB8EEC00AF7EE000AFEF7AB
:10FB000013FD8346F2F7F4FA002891D1BBF1000F00
:10FB10008ED12868D9ED007A4042B8EEE70A01217B
:10FB2000F0EE000AFEF71EFA8346F2F7E1FA00282B
:10FB30007FF47EAFBBF1000F7FF47AAF96ED000A41
:10FB40002868B8EEC00A4042F0EE080AFEF7ECFC66
:10FB50000646F2F7CDFA00283FF463AFF1F788FDCF
:10FB600007B0BDE8F08F00BF4007FF1FF49302000D
:10FB7000C48D02008015FF1F0814FF1F1C13FF1FF8
:10FB80002DE9F04FDFF81083D8F81430012B14BFA3
:10FB90000820032087B0F1F7FDFBD8F81030002BC8
:10FBA00040F36B81B74CB84DA146AA460126B74930
:10FBB00002A812F025FD002102A8F1F735FD02A8E8
:10FBC00012F0DEFC2220F1F7ADFE07EE906A002075
:10FBD000B8EEE70AF1F74AFEAD4902A812F010FDAF
:10FBE000002102A8F1F720FD02A812F0C9FCD8F804
:10FBF0001430002B00F05281012B40F03881A54FCA
:10FC00002068D7ED007A0193F0EE080AB8EEE70A13
:10FC1000FEF78AFC8346F2F76BFA002840F02D814C
:10FC2000019BBBF1000F40F02881D5ED007AD9F897
:10FC3000000001931946B8EEE70AF0EE080A4042C8
:10FC4000FEF790F98346F2F753FA019B002840F043
:10FC50001481BBF1000F40F01081D7ED007AD9F884
:10FC600000000193B8EEE70AF0EE000A4042FEF70A
:10FC70005BFC8346F2F73CFA019B002840F0FD80D4
:10FC8000BBF1000F40F0F980DAED007AD9F80000FE
:10FC90001946B8EEE70AF7EE000AFEF763F9834665
:10FCA000F2F726FA002840F0E880BBF1000F40F0A0
:10FCB000E480D7ED007A2068B8EEE70AF7EE000A94
:10FCC000FEF732FC8346F2F713FA002840F0D580A5
:10FCD000BBF1000F40F0D180D5ED007A2068B8EE7E
:10FCE000E70A0121F7EE000AFEF73CF98346F2F736
:10FCF000FFF9002840F0C180BBF1000F40F0BD804B
:10FD0000644B20681B68019307EE903A4042B8EEBE
:10FD1000E70AF0EE000AFEF707FC8346F2F7E8F97F
:10FD2000002840F0AA80BBF1000F40F0A6802068B8
:10FD3000D5ED007A4042B8EEE70A0121F1EE040A5F
:10FD4000FEF710F98346F2F7D3F9002840F09580CA
:10FD5000BBF1000F40F091804E4B206893ED000AFC
:10FD6000F0EE000AB8EEC00AFEF7DEFB8346F2F7BB
:10FD7000BFF9002840F08180BBF1000F7DD1D5EDA7
:10FD8000007A2068B8EEE70A0121F7EE000AFEF7D4
:10FD9000E9F88346F2F7ACF900286ED1BBF1000F09
:10FDA0006BD12068D7ED007A4042B8EEE70AF7EE53
:10FDB000000AFEF7B9FB8346F2F79AF900285CD1F6
:10FDC000BBF1000F59D1D5ED007A2068B8EEE70AF3
:10FDD0000121F7EE000AFEF7C5F88346F2F788F92D
:10FDE00000284AD1BBF1000F47D12A4B206893ED80
:10FDF000000AF0EE000AB8EEC00AFEF795FB834653
:10FE0000F2F776F9C8BBBBF1000F36D12068D5ED0B
:10FE1000007A4042B8EEE70A0121F0EE080AFEF748
:10FE2000A1F88346F2F764F938BBBBF1000F24D187
:10FE300097ED000A2068B8EEC00A4042F0EE080ACA
:10FE4000FEF772FB0746F2F753F9B0B9AFB9206875
:10FE5000D5ED007A4042B8EEE70A0121F7EE000A3C
:10FE6000FEF780F80746F2F743F930B92FB9D8F812
:10FE700010300136B342BFF69AAEF1F7F9FB07B086
:10FE8000BDE8F08F4007FF1F1C13FF1FF493020013
:10FE9000C48D02008015FF1F0814FF1FD5ED007AE6
:10FEA0002068B8EEE70A0121F0EE080AFEF75AF8DA
:10FEB0000746F2F71DF90028DFD1002FDDD1974F5B
:10FEC000D9F80000D7ED007A4042B8EEE70AF0EE2C
:10FED000080AFEF729FB8346F2F70AF90028CCD17D
:10FEE000BBF1000FC9D1D9F80000DAED007A404229
:10FEF000B8EEE70A0121F0EE000AFEF733F8834678
:10FF0000F2F7F6F80028B8D1BBF1000FB5D1D7ED64
:10FF1000007AD9F80000B8EEE70AF7EE000AFEF71B
:10FF200003FB8346F2F7E4F80028A6D1BBF1000FEB
:10FF3000A3D1DAED007AD9F80000B8EEE70A012182
:10FF4000F7EE000AFEF70EF88346F2F7D1F8002824
:10FF500093D1BBF1000F90D1D7ED007A2068B8EEB5
:10FF6000E70AF7EE000AFEF7DFFA8346F2F7C0F879
:10FF7000002882D1BBF1000F7FF47FAF2068D5ED60
:10FF8000007A4042B8EEE70A0121F0EE000AFDF7E0
:10FF9000E9FF8346F2F7ACF800287FF46EAFBBF1BF
:10FFA000000F7FF46AAF5D4B20681B68019307EE7A
:10FFB000903A4042B8EEE70AF1EE040AFEF7B4FACE
:10FFC0008346F2F795F800287FF457AFBBF1000F96
:10FFD0007FF453AFD5ED007A2068B8EEE70A01212F
:10FFE000F0EE000AFDF7BEFF8346F2F781F8002825
:10FFF0007FF443AFBBF1000F7FF43FAF474B206866
:020000021000EC
:1000000093ED000AF7EE000AB8EEC00AFEF78CFA8C
:100010008346F2F76DF800287FF42FAFBBF1000F95
:100020007FF42BAF2068D5ED007A4042B8EEE70AA6
:100030000121F7EE000AFDF795FF8346F2F758F825
:1000400000287FF41AAFBBF1000F7FF416AFD7ED95
:10005000007A2068B8EEE70AF7EE000AFEF764FAC5
:100060008346F2F745F800287FF407AFBBF1000F95
:100070007FF403AFD5ED007A2068B8EEE70A0121DE
:10008000F0EE000AFDF76EFF8346F2F731F8002824
:100090007FF4F3AEBBF1000F7FF4EFAE1F4B20688F
:1000A00093ED000A4042B8EEC00AF0EE080AFEF7EF
:1000B0003BFA8346F2F71CF800287FF4DEAEBBF172
:1000C000000F7FF4DAAE2068D5ED007A4042B8EE3A
:1000D000E70A0121F0EE080AFDF744FF8346F2F734
:1000E00007F800287FF4C9AEBBF1000F7FF4C5AE5E
:1000F00097ED000A2068B8EEC00A4042F7EE000A09
:10010000FEF712FA0746F1F7F3FF00283FF4AEAE10
:10011000F1F7AEFA07B0BDE8F08F00BF8015FF1F02
:100120002DE9F04FA54FDFF8B4927B69012B14BF86
:100130000320022087B0F1F72DF91421A04811F017
:1001400001FCD9F800109F4812F0DCF89D4812F02D
:1001500089F83B69002B40F3B880DFF884820124E2
:1001600046461221984811F0EDFB2146954812F0C1
:10017000C9F8944812F076F8944902A812F040FAAF
:10018000002102A8F1F750FA02A812F0F9F9222092
:10019000F1F7C8FB07EE904A0020B8EEE70AF1F746
:1001A00065FB8B4902A812F02BFA002102A8F1F797
:1001B0003BFA02A812F0E4F9D7F814A0BAF1000F44
:1001C00000F08880BAF1010F7AD114218148824D64
:1001D00011F0B8FBD9F800107A4812F093F879487A
:1001E00012F040F8D5ED007AD8F80000B8EEE70A32
:1001F000F0EE000AFEF798F98346F1F779FF002840
:1002000063D1BBF1000F60D1744B30681B68019360
:1002100007EE903A4042B8EEE70A5146F0EE000A87
:10022000FDF7A0FE8346F1F763FF00284DD1BBF137
:10023000000F4AD13068D5ED007A4042B8EEE70AA7
:10024000F7EE000AFEF770F98346F1F751FF002838
:100250003BD1BBF1000F38D1604B306893ED000A01
:100260005146B8EEC00A4042F7EE000AFDF77AFEAA
:100270008246F1F73DFF40BBBAF1000F25D195ED65
:10028000000AD8F80000B8EEC00A4042F7EE000AB3
:10029000FEF74AF90546F1F72BFFB0B9ADB9D8F82A
:1002A0000000D9ED007A4042B8EEE70A0121F0EEF5
:1002B000000AFDF757FE0546F1F71AFF28B925B9E0
:1002C0003B690134A342BFF64CAFF1F7D1F907B057
:1002D000BDE8F08FD9ED007AD8F80000DFF8FCA077
:1002E000B8EEE70A0121F0EE000AFDF73BFE0546F5
:1002F000F1F7FEFE0028E8D1002DE6D1364D30683A
:10030000D5ED007A4042B8EEE70AF0EE000AFEF7BB
:100310000BF98346F1F7ECFE0028D6D1BBF1000FB4
:10032000D3D13068DAED007A4042B8EEE70A012115
:10033000F7EE000AFDF716FE8346F1F7D9FE002816
:10034000C3D1BBF1000FC0D1D5ED007A3068B8EE53
:10035000E70AF7EE000AFEF7E7F88346F1F7C8FE72
:100360000028B2D1BBF1000FAFD19AED000A30687E
:10037000B8EEC00A40420121F7EE000AFDF7F2FD97
:100380008246F1F7B5FE00289FD1BAF1000F9CD14B
:1003900095ED000AD8F80000B8EEC00A4042F0EE31
:1003A000000AFEF7C1F80546F1F7A2FE002886D044
:1003B000F1F75EF907B0BDE8F08F00BF0814FF1F2A
:1003C000ACA802002408FF1FC4A80200F493020096
:1003D000C48D0200D8A802008015FF1F1C13FF1F48
:1003E0004007FF1F2DE9F04FDFF8C092D9F8143015
:1003F000012B14BF0620022087B0F0F7CBFFD9F8FD
:100400001030002B40F34281A34CA44DA04601269E
:10041000A34902A812F0F4F8002102A8F1F704F9A8
:1004200002A812F0ADF82220F1F77CFA07EE906AEC
:100430000020B8EEE70AF1F719FA9A4902A812F07B
:10044000DFF8002102A8F1F7EFF802A812F098F8FF
:10045000D9F814A0BAF1000F00F02A81BAF1010F07
:1004600040F00E81904F2068D7ED007AF7EE000A39
:10047000B8EEE70A5146FDF775FD8346F1F738FE01
:10048000002840F00381BBF1000F40F0FF80D8F856
:100490000000D7ED007A4042B8EEE70A5146F7EE89
:1004A000000AFDF75FFD8346F1F722FE002840F0C9
:1004B000ED80BBF1000F40F0E980D8F80000D5EDE9
:1004C000007A4042B8EEE70AF0EE000AFEF72CF898
:1004D0008346F1F70DFE002840F0D880BBF1000FF5
:1004E00040F0D480D8F80000D7ED007A5146404261
:1004F000B8EEE70AF0EE000AFDF734FD8346F1F7A7
:10050000F7FD002840F0C280BBF1000F40F0BE8034
:100510002068D5ED007A4042B8EEE70AF0EE000A16
:10052000FEF702F88346F1F7E3FD002840F0AE80C5
:10053000BBF1000F40F0AA80D7ED007A2068B8EE3A
:10054000E70A0121F7EE000AFDF70CFD8346F1F7FB
:10055000CFFD002840F09A80BBF1000F40F096805C
:100560002068D5ED007A4042B8EEE70AF7EE000ABF
:10057000FDF7DAFF8346F1F7BBFD002840F08680E7
:10058000BBF1000F40F08280474B206893ED000ADA
:100590004042B8EEC00A0121F0EE080AFDF7E2FC85
:1005A0008346F1F7A5FD002870D1BBF1000F6DD196
:1005B000D5ED007A2068B8EEE70AF7EE000AFDF7FD
:1005C000B3FF8346F1F794FD00285FD1BBF1000F24
:1005D0005CD197ED000A2068334FB8EEC00A0121C4
:1005E000F7EE000AFDF7BEFC8346F1F781FD002817
:1005F0004CD1BBF1000F49D1D5ED007A2068B8EE9F
:10060000E70AF7EE000AFDF78FFF8346F1F770FD6A
:1006100000283BD1BBF1000F38D12068D7ED007A1C
:100620004042B8EEE70A0121F0EE000AFDF79AFC1D
:100630008346F1F75DFD48BBBBF1000F26D1206872
:10064000D5ED007A4042B8EEE70AF0EE000AFDF779
:100650006BFF8346F1F74CFDC0B9BBF1000F15D11C
:1006600097ED000A2068B8EEC00A40420121F7EE7B
:10067000000AFDF777FC0746F1F73AFD30B92FB9CC
:10068000D9F810300136B342BFF6C2AEF0F7F0FF32
:1006900007B0BDE8F08F00BF4007FF1F8015FF1FA8
:1006A000F4930200C48D02001C13FF1F0814FF1FE7
:1006B000D5ED007A2068B8EEE70AF7EE000AFDF7FC
:1006C00033FF0746F1F714FD0028DFD1002FDDD1FD
:1006D000844BD8F800001B68019307EE903A404223
:1006E000B8EEE70AF7EE000AFDF71EFF0746F1F73E
:1006F000FFFC0028CAD1002FC8D17B4FD8F80000DA
:10070000D7ED007AF0EE000AB8EEE70A0121FDF716
:1007100029FC8346F1F7ECFC0028B7D1BBF1000FB0
:10072000B4D1704BD8F800001B68019307EE903AE3
:100730004042B8EEE70AF0EE000AFDF7F5FE834608
:10074000F1F7D6FC0028A1D1BBF1000F9ED1D8F85B
:100750000000D7ED007A4042B8EEE70A0121F7EE3B
:10076000000AFDF7FFFB8346F1F7C2FC00288DD19C
:10077000BBF1000F8AD1D5ED007A2068B8EEE70A08
:10078000F7EE000AFDF7D0FE8346F1F7B1FC002832
:100790007FF47CAFBBF1000F7FF478AF2068D7ED1A
:1007A000007ADFF844A14042B8EEE70A0121F7EEF3
:1007B000000AFDF7D7FB8346F1F79AFC00287FF487
:1007C00065AFBBF1000F7FF461AF2068D5ED007A13
:1007D0004042B8EEE70AF0EE080AFDF7A5FE8346B0
:1007E000F1F786FC00287FF451AFBBF1000F7FF4D6
:1007F0004DAF9AED000A2068B8EEC00A0121F7EE6D
:10080000000AFDF7AFFB8346F1F772FC00287FF486
:100810003DAFBBF1000F7FF439AFD5ED007A206812
:10082000B8EEE70AF7EE000AFDF77EFE8346F1F721
:100830005FFC00287FF42AAFBBF1000F7FF426AFE6
:1008400097ED000A2068284FB8EEC00A0121F7EEA4
:10085000000AFDF787FB8346F1F74AFC00287FF486
:1008600015AFBBF1000F7FF411AF2068D5ED007A12
:100870004042B8EEE70AF0EE000AFDF755FE834667
:10088000F1F736FC00287FF401AFBBF1000F7FF4D5
:10089000FDAE97ED000A2068B8EEC00A4042012183
:1008A000F0EE000AFDF75EFB0746F1F721FC002899
:1008B0007FF4ECAE002F7FF4E9AE2068D5ED007A2E
:1008C0004042B8EEE70AF7EE000AFDF72DFE0746B4
:1008D000F1F70EFC00283FF4D2AEF0F7C9FE07B0E6
:1008E000BDE8F08F8015FF1F1C13FF1F2DE9F0439B
:1008F000EBB0044641F2883205213CA8F8F74CFCE5
:10090000DFF8C482CDF8F0800023052206210CA870
:1009100057930DF089FE142215211CA80DF084FEBA
:10092000172210212CA80DF07FFE1D219448954F11
:1009300011F008F8944811F095FC1821934811F033
:1009400001F8934B9048196811F0DCFC8E4811F0C7
:1009500089FC12218F4810F0F5FF39688A4811F0A0
:10096000D1FC894811F07EFC052C4ED80123A34010
:1009700013F0240F00F02A813B68874A2D931368F7
:100980000593059913680493049B5B1A132BF9D9FB
:100990000C218248824D10F0D5FF2D997A4811F034
:1009A000B1FC794811F05EFCE96E2CA80DF07EFEDA
:1009B000296F0DF06FFE00210DF09CFE1621794885
:1009C00010F0C0FF296F704800230A2211F05AFC72
:1009D0006D4811F047FC012211460220F0F75EF845
:1009E000569B6AA903F10B0201EB820201EB830320
:1009F00000252CAE43F88C6CB7EE000A01213CA810
:100A000042F8B45C5695FAF7C5FE3E9B664E674DBC
:100A1000DFF88491CBB1F1F735FB002807DB3068B4
:100A2000F1F720FBC0B25328287000F0A480D9F859
:100A300000300793079AD9F800300693069B9B1A5B
:100A4000092BF8D93E9B002BE5D1052C0ED80122AD
:100A500002FA04F414F0240140F0098114F01203A6
:100A600040F05D8114F0090F40F0528108A8504910
:100A700011F0C6FD08A80021F0F7D6FD08A811F076
:100A80007FFD08A84B4911F0BBFD08A80021F0F735
:100A9000CBFD08A811F074FD08A8454911F0B0FD80
:100AA00008A80021F0F7C0FD08A811F069FD08A80A
:100AB000404911F0A5FD08A80021F0F7B5FD08A8F0
:100AC00011F05EFD08A83C4911F09AFD08A800212C
:100AD000F0F7AAFD08A811F053FD08A8354911F058
:100AE0008FFD08A80021F0F79FFD08A811F048FD30
:100AF00008A8324911F084FD08A80021F0F794FD00
:100B000008A811F03DFD08A82A4911F079FD08A8B0
:100B10000021F0F789FD08A811F032FD08A8284946
:100B200011F06EFD002108A8F0F77EFD08A811F075
:100B300027FD2220F0F7F6FED7ED007A0020B8EE70
:100B4000E70AF0F793FE08A81E4911F059FD0021AD
:100B500008A8F0F769FD08A811F012FD00233CA8D1
:100B60001D93CDF8F0800D933B602D93F8F75EFB5D
:100B70006BB0BDE8F0833CA8F8F700FB57E700BF77
:100B8000F0A80200B412FF1F2408FF1F10A90200E2
:100B9000F812FF1F2CA90200141CFF1F90A90200CD
:100BA000E815FF1FA0A902004807FF1FF413FF1F4D
:100BB00008A10200B08B0200F4A00200B8A9020054
:100BC000E09D0200C48D0200C487020013F0120FE2
:100BD00054D113F0090F3FF418AF3B68534A0D93FB
:100BE00013680193019913680093009B5B1A132B00
:100BF000F9D90C214E484F4D10F0A4FE0D994E48E6
:100C000011F080FB4C4811F02DFBE96D0CA80DF0A4
:100C10004DFD296E0DF03EFD00210DF06BFD1621FE
:100C2000464810F08FFE296E434800230A2211F037
:100C300029FB414811F016FB012211460020EFF775
:100C40002DFF569B6AA903F10B0201EB820201EB17
:100C5000830300250CAE43F88C6CB7EE000A01212B
:100C60003CA842F8B45C5695FAF794FDCDE61946D7
:100C700002202D9B3B60EFF711FFF7E63B682B4A04
:100C80001D9313680393039913680293029B5B1AE5
:100C9000132BF9D90C212A48264D10F053FE1D992B
:100CA000254811F02FFB244811F0DCFA696E1CA8CE
:100CB0000DF0FCFCA96E0DF0EDFC00210DF01AFD0D
:100CC0001621204810F03EFEA96E1B4800230A2280
:100CD00011F0D8FA184811F0C5FA01221146104651
:100CE000EFF7DCFE569B6AA903F10B0201EB8202CF
:100CF00001EB830300251CAE43F88C6CB7EE000AB1
:100D000001213CA842F8B45C5695FAF743FD7CE615
:100D10000D99396018461946EFF7C0FEA6E61D9BEF
:100D20003B601046EFF7BAFEA0E600BF141CFF1FA1
:100D300040A90200E815FF1F2408FF1F50A9020068
:100D400068A9020078A902002DE9F04FDFF8A8B3E6
:100D5000DFF8A883DBF80020D14ED8F81C40D8F883
:100D600018502DED028B0023012AD9B0336008EE14
:100D7000900A08EE101A00F0AE82C0F08782022AB4
:100D800000F023821F460293994601930393E4B235
:100D9000EBB21D462046012100930EF0D9FA2846F9
:100DA00001210EF0D5FA0AAD41F2883205212AA8B8
:100DB000F8F7F2F94FF0000ABA4B2A930222032106
:100DC0002846CDF814A10DF02FFC039B019A1AAE12
:100DD000194630460DF028FC98ED027ADBED0F7ACB
:100DE000DBF80420DBF824309FEDAF6A67EE877AEA
:100DF00098ED007AF8EE476A03FB02F307EE103A2B
:100E000067EEA67AD8ED016AB8EEC77AB8EE668AC0
:100E100027EE067A67EE887AF8EEE88A284627EE0B
:100E2000A88AFDEEC77A17EE901A0DF03FFCDBF8AA
:100E300008100DF02FFCFDEEC87A17EE901A0DF099
:100E400073FC029930460DF031FC39460DF022FC5E
:100E500049460DF069FC0821944810F073FD534693
:100E60000A22DBF80010924811F00CFA904811F0B9
:100E7000F9F908218F4810F065FD0D218E4810F01A
:100E800061FD18EE100A13F085FA41EC100B0221F7
:100E9000874811F041FA864811F0E4F908218548A5
:100EA00010F050FD0C21854810F04CFDDBF83C00A3
:100EB00013F070FA41EC100B02217D4811F02CFA6E
:100EC0007B4811F0CFF90821784810F03BFD09214B
:100ED0007B4810F037FDDBF8380013F05BFA41EC8B
:100EE000100B0221724811F017FA714811F0BAF98B
:100EF00008216E4810F026FD0D216F4810F022FDEC
:100F000049466B4811F0FEF9694811F0ABF901222E
:100F100003201146EFF7C2FDDBF80000012800F0C6
:100F2000B081C0F0A881022803D101221146EFF759
:100F3000B5FD37216348644F10F004FD5C4811F0A3
:100F400091F9449B58AA02EB830158A803F10C02C3
:100F500000EB8202002341F8886C41F88C5CB7EE0C
:100F6000000A42F8B43C02212AA84493FAF712FC82
:100F70002C9B564E002B30D020460EF0EFF98246C7
:100F8000002840F047812E21514810F0DBFC4848F2
:100F900011F068F9B9F1000F00F35E816A681B9BDC
:100FA0003A603360F1F76EF8002809DB494B1868A6
:100FB000F1F758F8484BC0B25328187000F045813B
:100FC000464A13680593059913680493049B5B1ABA
:100FD000092BF9D92C9B002BCED1DBF80090404B8C
:100FE0006A681B991A60B9F1010F316000F08A83B9
:100FF000C0F08A82B9F1020F00F0AE8106AC4FF06A
:101000000009012249460320C5F80490CDF86C90F0
:10101000EFF744FD0821274810F094FC3968244874
:1010200011F070F9224811F01DF905212D4810F03A
:1010300089FC31681E4811F065F91D4811F012F95C
:10104000D8F8A430012B00F035842749204611F050
:10105000D7FA49462046F0F7E7FA204611F090FA11
:101060002249204611F0CCFA49462046F0F7DCFA36
:10107000204611F085FA1E49204611F0C1FA494672
:101080002046F0F7D1FA204611F07AFA19492046A5
:1010900011F0B6FA49462046F0F7C6FA30E000BF34
:1010A000F812FF1FC48702000AD7233CCCA9020014
:1010B0002408FF1F009F0200D8A90200E8A902002F
:1010C000ACA00200F8A902006418FF1FB412FF1FB1
:1010D000A0A102004807FF1FF413FF1F141CFF1FED
:1010E0006C15FF1F2C9F0200BCAA0200B08B0200EF
:1010F000D0AA0200E88D02001418FF1FE815FF1F98
:10110000204611F03DFA8849204611F079FA494607
:101110002046F0F789FA204611F032FA834920463A
:1011200011F06EFA49462046F0F77EFA204611F09B
:1011300027FA7F49204611F063FA49462046F0F726
:1011400073FA204611F01CFA7A49204611F058FA39
:1011500049462046F0F768FA204611F011FA764920
:10116000204611F04DFA49462046F0F75DFA204638
:1011700011F006FA7149204611F042FA494620461C
:10118000F0F752FA204611F0FBF96749204611F0BA
:1011900037FA49462046F0F747FA204611F0F0F9B1
:1011A0006249204611F02CFA49462046F0F73CFAF5
:1011B000204611F0E5F9624B2A932AA8F8F736F891
:1011C00059B0BDEC028BBDE8F08FDBF81C00DBF8FA
:1011D00030209FED5C7AD8F83410D8F85040D8F819
:1011E0004C50DBF8207002FB00F207EE902AF8EE7C
:1011F000E77A67EE877AFDEEE77ACDED027A00298D
:1012000000F07B83012900F089839946172301931D
:101210001023BBE500980EF0A1F800287FF4BEAEC5
:1012200001902E21484810F08DFB484811F01AF823
:10123000B9F1000F019BBFF6B1AE2DA8009310F0DD
:101240007FFF009B32982C930CE02AA8F7F76AFFE7
:101250003F4B01221A70B3E62DA810F071FF3298AF
:10126000CDF8B0A00DF060FB33980DF05DFB384B6E
:1012700001221A70B1E6012250461146EFF70EFC2A
:1012800057E602460146EFF709FC52E6DBF80C1080
:10129000DBF828209FED2B7A9BED0E0ADBF810700F
:1012A00002FB01F207EE902AF8EEE77A184667EEA5
:1012B000877A0523FDEEE77A0193CDED027AEFF709
:1012C00027FEB8EEC88A062328EE000AFDEEC07A93
:1012D00017EE909A5AE5DBF81410DBF82C309FEDEE
:1012E000197A9BED0E0AD8F83040D8F82C50DBF86C
:1012F000187003FB01F307EE903AF8EEE77A142337
:1013000067EE877A1046FDEEE77A0193CDED027A1B
:10131000EFF7FEFDB8EEC88A152328EE000AFDEEB1
:10132000C07A17EE909A31E52C9E0200C48D02001F
:10133000E4AA0200B08B0200F8AA0200E88D0200C5
:10134000C48702000AD7233CD0A102002408FF1F53
:10135000E816FF1F0000B443D8F80420D8F8003086
:1013600098ED027AD7ED006A1FED066ADFF888A3D0
:10137000DFF888B303FB02F307EE903AF8EE677AE2
:10138000F8EEE66A67EE877A484686EEA77A06ACFC
:1013900007EE901AB8EEE70A67EE067ACAED007A11
:1013A000EFF7BAFC2046CB498BED000A11F028F983
:1013B00000212046F0F738F9204611F0E1F822200C
:1013C000F0F7B0FA9AED000A0020F0F74FFA204645
:1013D000C14911F015F920460021F0F725F9204602
:1013E00011F0CEF82046BD4911F00AF9002120463F
:1013F000F0F71AF9204611F0C3F82220F0F792FA1C
:101400009BED000A0020F0F731FA2046B24911F0B6
:10141000F7F820460021F0F707F9204611F0B0F860
:101420002046AF4911F0ECF820460021F0F7FCF817
:10143000204611F0A5F82046AA4911F0E1F820460F
:101440000021F0F7F1F8204611F09AF82046A6495D
:1014500011F0D6F820460021F0F7E6F8204611F00A
:101460008FF820469F4911F0CBF820460021F0F775
:10147000DBF8204611F084F820469C4911F0C0F8B2
:1014800020460021F0F7D0F8204611F079F82046E8
:10149000944911F0B5F820460021F0F7C5F8204630
:1014A00011F06EF82046924911F0AAF8204600216A
:1014B000F0F7BAF8204611F063F82046894911F098
:1014C0009FF820460021F0F7AFF8204611F058F8B9
:1014D0002046884911F094F820460021F0F7A4F83E
:1014E000204611F04DF820467E4911F089F820463B
:1014F0000021F0F799F8204611F042F84846012201
:101500000021EFF7CBFA7AE5D8F80400D8F80030DC
:1015100098ED027AD7ED006AD8F81040D8F80C2080
:1015200098ED055ADFED765ADFF8CCA1DFF8CC91C3
:1015300003FB00F307EE903AF8EE677AB8EEE66A3E
:1015400067EE877A07EE101A02FB04F2F8EEC76A1C
:1015500086EE277A06AC5F49204607EE902A66EEB3
:10156000856AF8EE677A27EE257A86EEA76A8AED15
:10157000007A89ED006A11F043F800212046F0F767
:1015800053F8204610F0FCFF2220F0F7CBF99AED3B
:10159000000A0020F0F76AF920464F4911F030F8B0
:1015A00020460021F0F740F8204610F0E9FF2046E1
:1015B0004A4911F025F800212046F0F735F8204679
:1015C00010F0DEFF2220F0F7ADF999ED000A0020BF
:1015D000F0F74CF92046404911F012F8204600215E
:1015E000F0F722F8204610F0CBFF20463C4911F0DE
:1015F00007F820460021F0F717F8204610F0C0FF4A
:101600002046384910F0FCFF20460021F0F70CF886
:10161000204610F0B5FF2046334910F0F1FF204678
:101620000021F0F701F8204610F0AAFF20462D49CE
:1016300010F0E6FF20460021EFF7F6FF204610F0FD
:101640009FFF2046294910F0DBFF20460021EFF7DD
:10165000EBFF204610F094FF2046224910F0D0FF07
:1016600020460021EFF7E0FF204610F089FF2046DA
:101670001F4910F0C5FF20460021EFF7D5FF204697
:1016800010F07EFF2046174910F0BAFF20460021D7
:10169000EFF7CAFF204610F073FF2046154910F0FF
:1016A000AFFF20460021EFF7BFFF204610F068FF94
:1016B00020460C4910F0A4FF20460021EFF7B4FFAC
:1016C000204610F05DFF002108460122EFF7E6F901
:1016D00095E400BFD09D0200C48D0200E09D020091
:1016E00030AA0200B08B020044AA020058AA0200ED
:1016F00080AA02006CAA02009016FF1FBC13FF1FF5
:101700000000B443D8F80420D8F8003098ED027AED
:10171000D7ED006A1FED066ADFF838A2DFF838B2AD
:1017200003FB02F307EE903AF8EE677AF8EEE66A0A
:1017300067EE877A07EE101AB8EEC70A86EEA77A28
:1017400006AC67EE067ACAED007AEEF701FF204696
:1017500075498BED000A10F053FF00212046EFF78A
:1017600063FF204610F00CFF2220F0F7DBF89AED23
:10177000000A0020F0F77AF820466C4910F040FF8C
:1017800020460021EFF750FF204610F0F9FE2046DA
:10179000674910F035FF00212046EFF745FF20464E
:1017A00010F0EEFE2220F0F7BDF89BED000A0020BD
:1017B000F0F75CF820465D4910F022FF204600213A
:1017C000EFF732FF204610F0DBFE2046594910F0BB
:1017D00017FF20460021EFF727FF204610F0D0FE2C
:1017E0002046554910F00CFF20460021EFF71CFF62
:1017F000204610F0C5FE2046504910F001FF20465B
:101800000021EFF711FF204610F0BAFE20464A49AA
:1018100010F0F6FE20460021EFF706FF204610F0FC
:10182000AFFE2046464910F0EBFE20460021EFF7C0
:10183000FBFE204610F0A4FE20463F4910F0E0FEDB
:1018400020460021EFF7F0FE204610F099FE2046DA
:101850003C4910F0D5FE20460021EFF7E5FE20467A
:1018600010F08EFE2046344910F0CAFE20460021BA
:10187000EFF7DAFE204610F083FE2046324910F0E2
:10188000BFFE20460021EFF7CFFE204610F078FE85
:101890002046294910F0B4FE20460021EFF7C4FE8F
:1018A000204610F06DFE4A4648460021EFF7F6F854
:1018B000FFF7A5BB2549204610F0A2FE4946204669
:1018C000EFF7B2FE204610F05BFE1B49204610F0F9
:1018D00097FE49462046EFF7A7FE204610F050FE3F
:1018E0001B49204610F08CFE49462046EFF79CFE2F
:1018F000204610F045FE104953E49BED0E0AEFF729
:101900003DFAB8EEC88A172328EE000A0193FDEECF
:10191000C07A102317EE909AFFF738BA9BED0E0AA3
:10192000EFF7C6FAEDE700BFD09D0200C48D0200BC
:10193000E09D020030AA0200B08B020044AA02001F
:1019400058AA02006CAA020080AA020094AA02000F
:10195000A8AA02009016FF1FBC13FF1F2DE9F04F2D
:10196000DFF84C83DFF89C93D8F84830CD4AD9F89B
:101970001C40D9F818602DED028BD9B00025012B41
:101980000090156000F0C085C0F04885022B00F083
:101990001384AA460295AB4603952F46E4B220462F
:1019A0000121F6B20DF0D4FC304601210DF0D0FC3F
:1019B00041F2883205212AA8F7F7EEFBBA4B2A93A9
:1019C0000222002303210AA8459301930CF02CFE68
:1019D0003A4629461AA80CF027FED8F80010D8F885
:1019E00010209FEDB27AB24D02FB01F307EE903A60
:1019F000F8EEE77A0AA867EE877AFDEEE77A17EE47
:101A0000901A0CF053FED8F820100CF043FED8F8D2
:101A10004C70002F00F02E84012F40F0FA8495EDD9
:101A20000F6A9FEDA47AD9ED027A2A6BA86C95ED26
:101A30000E0AC6EE076A99E80A0003FB01F352009A
:101A4000019207EE103AB8EE477A9DED006A67EE14
:101A5000277AB8EEC68A67EEA67A67EE887AFDEE38
:101A6000E77ACDED007AEFF753FA2B6B5B0007EEC8
:101A7000903AF8EEE77A80EE270A20EE088AFDEE2B
:101A8000C87A17EE905A3B218B48894F0FF05AFFC6
:101A90008A4810F0E7FB0D2189480FF053FF0099A9
:101AA000864810F02FFC854810F0DCFB112185489A
:101AB0000FF048FF844B8148196810F023FC7F48E1
:101AC00010F0D0FB0A2181480FF03CFF29467B48EB
:101AD00010F018FC794810F0C5FB3B2176480FF058
:101AE00031FF764810F0BEFB02991AA80CF0DEFD1B
:101AF00051460CF0CFFD0E2175480FF023FFD8F8AA
:101B000000106E4810F0FEFB6C4810F0ABFB142187
:101B100070480FF017FFD8F81010684810F0F2FB6B
:101B2000664810F09FFB0D216B480FF00BFF002360
:101B30000A22D8F82010614810F0A4FB5F4810F08A
:101B400091FB132165480FF0FDFE00230A22D9F80E
:101B500000105A4810F096FB584810F083FB1121F2
:101B60005F480FF0EFFE00230A22D9F80410534813
:101B700010F088FB514810F075FB122159480FF006
:101B8000E1FED9F8080012F005FC41EC100B02212F
:101B90004A4810F0C1FB494810F064FBD8F84C30BB
:101BA000002B00F00984012B2AD110214E480FF0A0
:101BB000C9FEF86B12F0EEFB41EC100B02213F481E
:101BC00010F0AAFB3D4810F04DFB0F2147480FF0E5
:101BD000B9FEB86B12F0DEFB41EC100B0221374866
:101BE00010F09AFB354810F03DFB0C2140480FF0F7
:101BF000A9FE396B314810F085FB304810F032FBFC
:101C00000D212F480FF09EFE00992C4810F07AFB12
